:100000000C94890F0C94A80F0C94A80F0C94A80FB3
:100010000C9489290C94A80F0C94A80F0C94C62A50
:100020000C94A80F0C94A80F0C94A80F0C94A80F74
:100030000C94A80F0C94A80F0C94A80F0C94A80F64
:100040000C94A80F0C94A80F0C94A80F0C94A80F54
:100050000C94A80F0C94A80F0C94B42F0C94A80F18
:100060000C94A80F0C94A80F0C94A80F0C94A80F34
:100070000C94A80F0C94A80F0C94A80F0C941323A5
:100080000C94A80F0C94A80F0C94A80F0C94A80F14
:100090000C94A80F0C94A80F0C94A80F0C94A80F04
:1000A0000C94A80F5645523A323430393230009B06
:1000B0001354153C156E156512A41549112E1551D2
:1000C00011DE116C1F8915491149117520C6131CC9
:1000D0001054153C156E156512A415C2142E150882
:1000E00014DE116C1F8915B31149117520C613490F
:1000F0001154153C156E156512A4157E122E15545B
:1001000012DE116C1F8915B91149117520C61349EA
:100110001154153C156E156512A415E0122E1557D5
:1001200012DE116C1F89151E1549117520C6137337
:100130001154153C156E156512A41549112E155B49
:1001400012DE116C1F8915C21349117520C6137375
:100150001154153C156E156512A415A7112E15F432
:1001600013DE116C1F8915D71549117520C613733D
:100170001154153C156E156512A415AD112E1537C9
:1001800014DE116C1F8915531149117520C61373A4
:100190001149114911491165124911BC15491164E0
:1001A00011DE116C1F49114911491175204911497E
:1001B0001154153C156E156512A41549112E156ABA
:1001C00013DE116C1F8915651349117520C613497B
:1001D0001154153C156E156512A41514122E159C9C
:1001E00013DE116C1F8915BF1149117520C6134903
:1001F0001154153C156E156512A4151C122E15A070
:1002000013DE116C1F8915491149117520C6134958
:100210001154153C156E156512A41521122E15B535
:100220000FDE116C1F8915921449117520C61349F0
:100230001154153C156E156512A41549112E15AAF9
:100240000FDE116C1F8915A41349117520C61349BF
:100250001154153C156E156512A415E9112E15875C
:1002600014DE116C1F8915F91549117520C6134943
:100270001154153C156E156512A415F5112E15CCEB
:1002800015DE116C1F8915031549117520C6134918
:1002900011E611E414751365123A12001246124A5F
:1002A00011DE116C1F4911D0114911752049119CA3
:1002B000ACCCB6F400C111214191A131B171F19CD6
:1002C000ACCCB6F4367491A1C111214131F1714425
:1002D0004547000055534552000052414400005329
:1002E0004849465400005052474D0000414C504888
:1002F000410000000302050003050104060204C0DA
:10030000C1C2FFC4C5C618808182C3848586877038
:1003100071728374757677303132733435363710B5
:10032000111213141516170304050A08060BFF0211
:1003300009070D010C00FF464B3A3A494A483A3A40
:100340003A3A3A4C4F3A3A3A3A3A3A3A3A3A3A3AE6
:100350003A3A3A3A4D3A3A30000030000030000064
:10036000200000300418355D80300C902000083BE0
:10037000AEBC359D9C318C9C2AAAA83BAEBC359D59
:100380009C318C9C2AAAA8300018355580300090EA
:10039000200008300418355D8030009020000830BF
:1003A00000183555803000002000000057C007FFBE
:1003B000C402FFC000028000FFC005FFD402FFE0BE
:1003C000002E000001F41557F82D100002800030B7
:1003D000000030000030000020000007FFF40B5048
:1003E0003C057FF40A00283FFFFC000F00157D400C
:1003F0002AAA800007FC00783C07897C2800280096
:100400003C00557D55AABEAA003C00000000555591
:1004100055AABEAA003C003FFFFC30000C30000C87
:1004200030000C3FFFFC31554C32AA8C30000C3FA1
:10043000FFFC31554C32AA8C33FFCC30000C30001D
:100440000C30000C35555C31554C32AA8C30000C08
:1004500035555C31554C32AA8C33FFCC35555C2A6E
:10046000FFA800000000000000000000000055543C
:1004700000AABC00003C00003C00557C00AAA8007B
:10048000000000003C00003D55002AAA00000000CA
:100490000000001555003EAA003C00003C00003C56
:1004A00000003C00003C00003C00557C00AABC0061
:1004B000003C0001414403C7E007E3C02282800002
:1004C0003C00003D55003EAA003C00003C00557D2C
:1004D00055AAAAAA000000000000000000000000C9
:1004E0000000000000003FFF3C0000000000003F53
:1004F000C0000000001540002A800017D7D42BEB65
:10050000E83FFFFC02828007F4D01F7DF40F3DF02E
:10051000020A803C0078001E8007A0142800281FD3
:1005200047F43C343C2F8AF80002080000001440D5
:10053000002A000000000007FFD03E00BC20000899
:1005400000000034001C2F55F802AA8000000002B1
:100550004C60017F50006E40020820003C0003FF09
:10056000C0003C000000000000000003D8000000B4
:10057000000000003C00003C00003C00002800009F
:1005800000000000F0000000000000000078001EE5
:100590008007A0002800001FFFF43C1E3C3DF57CB6
:1005A0000AAAA005003C3FFFFC00003C0000001F21
:1005B00001FC3C1FBC3DF83C0A80281F00F43C14A1
:1005C0003C3D7D7C0A82A0007F00078F003FFFFC3E
:1005D000000A003FF0F43CF03C3CF57C282AA01FC8
:1005E000FFF43C3C3C3C3D7C280AA03C00003C1F06
:1005F000FC3DF8002A80001FD7F43C3C3C3D7D7C4C
:100600000A82A01FF4F43C3C3C3D7D7C0AAAA00079
:100610000000014140028280000000000000014112
:10062000440282A0000000001D0001E2D00E002C58
:1006300000000001414003C3C003C3C00000000428
:1006400000040B407800B7800008001F00003C1F2A
:100650003C3D78000A800006AAA431AA4C24AA4C8A
:1006600002AA0007FFFC3E0F002F5F5402AAA83F1A
:10067000FFFC3C3C3C3D7D7C0A82A01FFFF43E0019
:10068000BC3D007C0A00A03FFFFC3C003C2F55F81D
:1006900002AA803FFFFC3C3C3C3C283C2800283F11
:1006A000FFFC3C3C003C28002800001FFFF43C00FD
:1006B0003C3C0F7C080AA03FFFFC003C00157D5429
:1006C0002AAAA83C003C3FFFFC3C003C0000001470
:1006D00000F43C003C3FFFF82800003FFFFC003CDA
:1006E0000017C3D42800283FFFFC00003C00003C5A
:1006F0000000283FFFFC0B40001F55542AAAA82FDA
:10070000FFFC02D000157D542AAAA81FFFF43C006C
:100710003C3D557C0AAAA03FFFFC3C3C003D7C00D0
:100720000AA0001FFFF43C053C3D57FC0AAAA03F6D
:10073000FFFC3C3D003D7EF40AA0281FF4343C3C05
:100740003C3C3D7C080AA03C00003FFFFC3C000014
:100750000000003FFFF400003C15557C2AAAA03F92
:10076000FF400000B41555E02AAA003FFFF800073B
:10077000801557D02AAAA83D417C02BE8017EBD431
:100780002800283FD400003FFC3FE8000000003C68
:1007900001FC3C1E3C3DE03C2A00281555543EAA75
:1007A000BC3C003C0000002D000002B400000AD058
:1007B0000000281400143C003C3FFFFC0000000136
:1007C000E0001E00000B400000A00000003C000004
:1007D0003C00003C0000282D000002D0000000007A
:1007E0000000000051F400F33C00F774002AA83F19
:1007F000FFFC00F03C00F57C002AA0007FF400F034
:100800003C00F03C002020007FF400FC3C157D7C87
:100810002AAAA8007FF400F33C00F73C002A200538
:100820007D543EBEA83D28000A0000007D1400F360
:100830003C00F77C002AA03FFFFC00780000F55444
:10084000002AA80050003CFFFC000000000000004F
:1008500000F400503C3CFFF80000000FFFFC0007D4
:10086000D000382C0000081400003FFFFC000000FE
:1008700000000000FFFC002D00007D5400AAA8002D
:10088000BFFC00F80000BD54002AA8007FF400F06F
:100890003C00F57C002AA000FFFC007AD000F5F0B7
:1008A000002A80007FD000F0F0007FD400AAA800CA
:1008B000FFFC00780000F400002800007D3C00F3FD
:1008C0003C00F37C00A0A015F5502AFABC00007C87
:1008D0000000A000FFF400003C00557C00AAA0002E
:1008E000FF400000B40055E000AA0000FFFC00013A
:1008F000E00055F400AAA800F47C002BA0007EF4D0
:1009000000A02800FD14000F3C005F7C00AAA0009E
:10091000F07C00F3BC00FE3C00A028000000057D38
:10092000503A82AC000000000000555555AAAAAA12
:1009300000000000000035415C0ABEA00000003F3E
:1009400041FC3CBE3C3D007C2A00A83FFFFC003C33
:1009500000003C00002800005FFF07A0057807FEAC
:10096000F03E00F03FFFBD2AAA0AF555FFD4005023
:100970002B40BFC2F007C0BCFF007CABC0A05F80B3
:10098000001FFFFFFFFFFFFF800FFF000FFF400F63
:10099000FFFFFF2FFFFFFFFFFCFFFFFCF00000F059
:1009A0000000F00000FFFFFCFFFFFCFFFFFFFFFF68
:1009B000FFFF003FFF003FFF407FFFFFFF2FFFE0F3
:1009C000FFFFFCFFFFFCC003FCC003FCD007FCFFE3
:1009D000FFFCBFFFE01FFFFFFFFFFFFF8000FF00E6
:1009E00000FF4000FFF0002FF000FFFFD0FFFFFCF2
:1009F000000BFC0003FC0007FC00FFFC00FFE0FF15
:100A0000FFFFFFFFFFFF0000FF0000FF40003FFF70
:100A1000FF0AFFFFFFFFFCFFFFFC0003FC0003FCDD
:100A20000007FCFFFFF0FFFE80FFFFFFFFFFFFFF5F
:100A3000003FFF003FFF003FFF0000FF0000FFFFFF
:100A4000FCFFFFFCC003FCC003FCC003FC0003FC74
:100A50000003FCFFFFFFFFFFFFFF003FFF003FFF22
:100A6000002AFF0000FF0000FFFFFCFFFFFCC000AA
:100A700000C000008000000000000000001FFFFF19
:100A8000FFFFFFFF8000FF0000FF4000FFF0002F8E
:100A9000F000FFFFD0FFFFFC000BFC0003FCFF0792
:100AA000FCFFFFFCFFFFE0FFFFFFFFFFFF00003F39
:100AB00000003F00003FFFFFFFFFFFFFFFFFFCFFC5
:100AC000FFFCC00000C00000C00000FFFFFCFFFFF3
:100AD000FCFF0000FF0000FF5555FFFFFFFFAAAA23
:100AE000FF0000FF00000003FC0003FC5557FCFF63
:100AF000FFFCAAABFC0003FC0003FC0000000000AC
:100B000000FF0000FF0000FFFFFFFFFFFFFF0000EE
:100B100000FFD000FFFC000BFC0007FCFFFFFCFF08
:100B2000FFE0000000FFFFFFFFFFFF00003F0001AC
:100B3000FF001FF8FFFF80FFF800FFFFFCFFFFFC36
:100B4000D00000FD0000BFD0000BFFFC00BFFCFF89
:100B5000FFFFFFFFFF00000000000000000000009A
:100B600000000000FFFFFCFFFFFC0003FC0003FC93
:100B70000003FC0003FC0003FCFFFFFFFFFFFF0A74
:100B8000FF50000FFF05FFA0FFFFFFFFFFFFFFFF6C
:100B9000FCFFFFFC000000000000000000FFFFFC65
:100BA000FFFFFCFFFFFFFFFFFF2BFF50002BFF00AD
:100BB000002BFFFFFFFFFFFFFFFFFCFFFFFC00001C
:100BC00000500000FF5000FFFFFCFFFFFC1FFFFF75
:100BD000FFFFFFFF8000FF0000FF4000FFFFFF2F2F
:100BE000FFFFFFFFD0FFFFFC000BFC0003FC000732
:100BF000FCFFFFFCFFFFE0FFFFFFFFFFFFFF003FE9
:100C0000FF003FFF407FFFFFFF2FFFFEFFFFFCFFC6
:100C1000FFFCC00000C00000C00000C000000000D9
:100C20000017FFFF7FFFFFFF8000FF0000FF400075
:100C3000BFFFFF2BFFFFFFFF50FFFFF0000BFC0F7C
:100C4000F6FC0AFF6CFDBFF4FFDBFCFFFFFFFFFFBC
:100C5000FFFF003FFF003FFF407FFFFFFF2FFFFE32
:100C6000FFFFFCFFFFFCFF0000FFD000EFFD00C214
:100C7000FFFC002FFC17FFF57FFFFFFF80BFFF0089
:100C80003FFF403FBFF02F2BF00A003F50403FF4A2
:100C9000C00BFCC003FCD007FCFFFFF8FFFFA0FF68
:100CA0000000FF0000FF5555FFFFFFFFAAAAFF004D
:100CB00000FF0000000000000000555554FFFFFC3D
:100CC000AAAAA8000000000000FFFFFFFFFFFF002E
:100CD0000000000000000000FFFFFFFFFFFFFFFF1C
:100CE00050FFFFF4000BFC0003FC0007FCFFFFF8C3
:100CF000FFFFA0FFFFFFFFFFFF000000000000005C
:100D00000000FFFFFFFFFFFFFFD000FFFD0000BF5F
:100D1000D0000FFC007FE0FFFE00FFE000FFFFFFC0
:100D2000FFFFFF000000000000000000FFFFFFFFCA
:100D3000FFFFFFFFFCFFFFFC017FA03FF00002BFB1
:100D400050FFFFFCFFFFFCFF5000FFFF5000AFFF14
:100D500000003F005FFFFFFFA0FFA0000017FC178F
:100D6000FFFCFFE800F00000FFD4002BFFFC002B8D
:100D7000FCFFFFD0FFFFFD0000BF00000F00007F61
:100D8000FFFFFEFFFFE0000000000000D55554FF0C
:100D9000FFFCEAAAA8000000000000FF0000FF001E
:100DA00000FF0007FF007FFF07FFFFFFFEFFFFE0E0
:100DB00007FFFC7FFFFCFFE3FCFE03FCE003FC00FD
:100DC00003FC0003FCFFFFFFFFFFFFFF0000FF002D
:100DD00000FF0000FF0000FF0000FFFFFCFFFFFC22
:100DE0000003FC0003FC0003FC0003FC0003FC14F4
:100DF00000003FD4002BFFD4002BFF00002B00008D
:100E000000000000000000000000000000D400000E
:100E1000FFD4002BFFC0002BC0FF0000FF0000FF2D
:100E20000000FF0000FF0000FFFFFFFFFFFF0003C7
:100E3000FC0003FC0003FC0003FC0003FCFFFFFCC0
:100E4000FFFFFC001F0001FF001FFFFFFFFFFF2F40
:100E5000FFFF02FF00002F00000000000000FFFF66
:100E6000FCFFFFFCFFFFFC00000000000000000092
:100E70000000000000000000000000000000000072
:100E800000000003FC0003FC0003FC0003FC000363
:100E9000FC0003FC0003FC00000000000000000058
:100EA0000000000000000000000000000000000042
:100EB0000000000000000000000000000000000032
:100EC00000000000000000555555FFFFFFAAAAAA28
:100ED000000000000000000000000000554154FF29
:100EE000C3FCAA82A8000000000000555500FFFFC7
:100EF00000AAAA00000000000000FFFF00FFFF00A2
:100F000000000000000000000000000000000000E1
:100F10000000000000000FF00FFFFF0FFFFF000FA9
:100F2000F00FFFFF0FFFFF000FF03FC000FFFFC0FB
:100F3000FFFFC03FC000FFFFC0FFFFC03FC0000079
:100F4000555407FFFF0FE02FFFFFFFAFEAAF0FF48D
:100F50000F02FC0200540040FF40C02FC0FFFFFC06
:100F6000EAAFE8F57FC0FFFE0001540003FC000279
:100F7000A80100017F017FFE3FFE803E800000014E
:100F800040017FC07FFE80FE800080000003FC00E7
:100F900003FC0000000101551F1FFFFF3E03FF3F40
:100FA000DFE00AFA00000003FFFD40EAAFF0400274
:100FB000FCF500FCBFF5F802FFD0FFFAB00000001E
:100FC000FFFF00FFFF000000000000000000000025
:100FD0000000000000000000000000000000000011
:100FE000000000000000000000000007FF01FFFFFC
:100FF0000FFA007E0000A80000000000000000FFC3
:101000004000FFFD0002BFC00002F40000A8000085
:1010100000000000F400003F40000BFD5500BFFF42
:101020000002AF00000000000000007C0007F05547
:10103000FF80FFF800EA0000000000003D0F000BF9
:10104000DF0015FF003FFF002AFF0007EF003E0F03
:10105000F07C00F7E000FF5400FFFC00FFA800FB5D
:10106000D000F0BC0000000F00000F00155F003F33
:10107000FF002AAF00000F00000FF00000F000009A
:10108000F55400FFFC00FAA800F00000F00000009A
:10109000000700000F00000F00005B0007CF01FAFF
:1010A0000F00000B400000C00000C00000940000D2
:1010B000CF4000C2BD0080000000000500000F000E
:1010C000000F00000F00000F00000F00000F500085
:1010D00000F00000F00000F00000F00000F0000060
:1010E000F0000000000702F50F000BCF0000A70082
:1010F000000F00000F00000B400000C17E00CF80F9
:1011000000680000C00000C0000080000000000077
:1011100000000000000100017F017FFE3FFE803ED5
:101120008000000140017FC07FFE80FE80008000C3
:101130000000000000000017FFFF7FFFFFFF80019D
:10114000FF001FFF41FFBFFFFF2BFFFFFFFF50FF0F
:10115000FFF4FF8BFCF803FC8007FCFFFFF8FFFFA8
:10116000A000000007FC007FFD55FFFFFFAAAAAA10
:101170000000000000000003FC0003FC5557FCFFCA
:10118000FFFCAAABFC0003FC0003FC1FF0007FF097
:1011900000FF8000FF0001FF401FFFFFFF2FFFF84F
:1011A000001FFC01FFFC1FFBFCFF83FCF803FC801D
:1011B00003FC0003FC1FF000FFF000FF8000FF00B5
:1011C0003FFF407FFFFFFF2FFFE0003FD0003FFCCD
:1011D000000BFCC003FCD007FCFFFFFCBFFFE000DE
:1011E000007F0007FF007FF807FF807FFD55FFFFAE
:1011F000FFAAAAAAFF0000FF0000FF0000FF0000F6
:10120000FF5554FFFFFCFFAAA8FFFFFDFFFFFFFFF4
:1012100000FFFF00FFFF00FFFF00FFFF002F003F68
:10122000D0003FFC000BFC0003FC4007FCFFFFFC70
:10123000FFFFE01FFFFFFFFFFFFF807FFF00FFFFBB
:1012400000FFFF00FFAA002FFFFFD0FFFFFC800B75
:10125000FC0003FC4007FCFFFFFCFFFFE055000023
:10126000FF0000FF0000FF0001FF001FFFFFFFFF66
:10127000FFF8000000000000155554FFFFFCFAAA1B
:10128000A88000000000001FFFD0FFFFFFFF80BF0D
:10129000FF003FFF407FFFFFFF2FFFE27FFFD0FFF8
:1012A000FFFCE00BFCC003FCD007FCFFFFFCFFFFD2
:1012B000E01FFFF5FFFFFFFF80BFFF003FFF407F04
:1012C000FFFFFF2FFFFF003FD0403FFCC00BFCC0E3
:1012D00003FCC007FCFFFFFCFFFFE06FFFF9F455C4
:1012E0000FFC0A8FFCFFF3FC054FFCAA0FE7FFF68B
:1012F000BFFFE4C1547CCA80FC3FFCFCC540FCC27B
:10130000A8FC7FFF6C00000700000F00000F00002A
:101310000B000000000000000000400000C01500AD
:10132000C7E8009E00000000000000000000000070
:10133000000700007F0007F8007F8007F8003F806B
:1013400000380000400000F40000BF40000BF40033
:1013500000BF40000BF00000B0000FF0000FF000E5
:101360000FF0000FF0000FF0000FF0000FF00FF083
:10137000000FF0000FF0000FF0000FF0000FF00072
:101380000FF0003400003F40000BF40000BF4000AD
:101390000BF40000BF00000B0000700007F0007F9E
:1013A0008007F8007F8000F8000080000017FC0034
:1013B0007FFC00FF8001FF001FFF41FFBFFFF82BF4
:1013C000FF80000000000000555154FFF3FCAAA26A
:1013D000A80000000000002FFFF902AA8F00000FF4
:1013E00000000B000000000000000000BFFFE0CA8A
:1013F000AA00C00000800000000000000000000003
:1014000000000000003FC0003FC0003FC0003FD0D0
:10141000003FFF000BFF1FFFD0FFFFFCFF8BFCFF17
:1014200003FCFF03F8FFFFFCFFFFFC0FFFFF0FFFB4
:10143000FF00001F00003F00003F00003F00000BC6
:10144000FFFFFCFFFFFCF80BFCC003FCD007FCFF18
:10145000FFFCFFFFE000007F0003FF0003FE00032E
:10146000FC0003FD0003FF0000BFFFFFD0FFFFFCF7
:10147000000BFC0003FC0007FC000FFC000FE00069
:10148000000100001F00003F00003F00002F0FFF81
:10149000FF0FFFFFFFFFD0FFFFFCE00BFCC003FCD2
:1014A000D007FCFFFFFCFFFFFC00007F0003FF00F4
:1014B00003FE0003FC0003FD0003FF0000BFFFFF6D
:1014C000D0FFFFFC3FCBFC3FC3FC3FC3FCFFC3FC92
:1014D000FFC3FC400000F40000FC0000FC0000FC26
:1014E0000000FC0000E00000000000000000000020
:1014F00000000000000000000000000000400000AC
:10150000F40000FC0000FDFFF4FCAAA0FC0000E0D9
:1015100000000000000000000000000000000000CB
:1015200000000000000000400000F40000FC00008B
:10153000FDFFFDFCAAA8FC0000E000000000000088
:10154000150007E800AA00000000000000000000ED
:1015500000400000F40000FC0000FDFFFDFCAAA814
:10156000FC0000E0000000000000150007E800AAF1
:101570000000AF400002BD00000000400001F40088
:101580000FFC000FFDFFF7FCAAA0FC0000E000002C
:10159000000000C01500C7E8002A0000AF400002AC
:1015A000BD00000000400001F4000FFC000FFDFF33
:1015B000F7FCAAA7FC000FE0000B000000C015001C
:1015C000C7E8002A00006F4000C2BD008000000094
:1015D000001500003F00000000000500000F0000A3
:1015E00000000000555550FFFEA000BF00555F00F1
:1015F000FFFF00001600000000000FF0000FF000D9
:101600000FF0000FF5000FFF15FFF03FAFF00FF5E3
:10161000FC0FFFA85FF000FFF0000FF0000FF000DC
:101620000FF000FD4000FFFD40FC2BFDFC002FFDF6
:101630000002FFC000FFC0000005FC05FFFCFFA08A
:10164000FCE000FC0001FC000FFC000FFC000000AF
:101650000000000000000000070001FE007F800F76
:10166000E0000001FC007FFC1FE0FCFF00FC0BD051
:10167000FC00BFFC0000FC00000100000F00003F68
:1016800000003F00003F00003F00003EF001F0C1BD
:101690007FF0DFFA00E00550DFFFF0EA03F0000A18
:1016A0000000000500007F0003FF0003F80003FDB9
:1016B0000001FF0003FAFFFF40FFFFF0A00FF00062
:1016C0001FE057FF50FFFFF0AA03F017FFFF3FEAAC
:1016D000AAFE0054FC00FCFF01FD3FFFFF0BFE8F44
:1016E000FFFFFFABFEAA00FF0000FF0001FF00FFAD
:1016F000FE00FFF80000000114001FFC007FFC004A
:10170000FCFD403F3FFFFF0ABFFF5FF500FFFFF01A
:101710008002FC0003F8517FE0FFFE00EA80000039
:101720001FD401FFFD07F82F0FF00F0FF00F0FF080
:101730000A02FC001FFD00FFFFD0F00BF4E003FCE9
:10174000C003FC8003FC000FF000001500003F0701
:10175000FFFF3FFFFFFE003FFC002ABF0000000329
:10176000FC015FFCFFFFFCFEA3FC0003FC0003FC8C
:101770000003FC0000FC005FFF0FFEFE3F80FCFE4C
:1017800000FCFD00FC3F4000FC0000FFD400FEFF19
:10179000C0FC0BF0FC02FCFC01FC0007E0000014A4
:1017A0000001F80013F007F3C0FE83F0A002FF0071
:1017B000000A0155001FFFD07E02FCFC00FCFC0764
:1017C000E0FFFFFCAAAAA800001F0001FE0173F0C1
:1017D0005FE3F0F803F50000BF00000AFFFF40FEE2
:1017E000AFF4FC02FCFC00FCFC01FCFC03F0A800D4
:1017F000000000500000F0007CF51FE0FF3E0000FC
:101800000000000000000000FC0000FC5555FCFF3B
:10181000FFFC0000FC0000FC00000000005F000175
:10182000FE01F3F05FA3F0F802FF00002B000000C0
:10183000FFFD40AAAFF40002FC0001FC555FF8FF79
:10184000FE800000000003FF0010AA45F0003F806A
:10185000002801FF0002AA000000FFFFD0AAABFC95
:101860000000FC0005F8FFFFFCAAAAA80000000089
:10187000000000000005FFFF3FFFFFFE00003C00EE
:101880000000000000001F00003FFFFFFFFFFFE817
:10189000000000000000000000001FE0003FC0004A
:1018A0003FD0000FF00003FC0003FC001FF07F801E
:1018B00000FF0000FF00003FC0000FF0000FF0002D
:1018C0007F80000000FF07F0FF0F007E0BD3F007C2
:1018D000F3FD0F80FF00002FFFFFFCFFFFFC000067
:1018E00000000000000000FFFFFCFFFFFC0017FFEE
:1018F00001FFEA0FE8000FC0000FD40002FFD5007F
:101900002BFFFF50FCAFFDFC000BFC0000000007AC
:10191000FC5FFEFCFA80FC400000F40000FC0000CC
:10192000FDFFF4FCAAA0FC0000E0000000000000A5
:1019300000000000000000000000000000000000A7
:10194000000000000003FC0003FC0003FC0003FD9A
:101950000003FF0000BF07FFD03FFFFC3F8BFC3FB1
:1019600003FC3F03F8FFFFFCFFFFFC0FFFFF0FFF2F
:10197000FF00001F00003F00003F00003F00000B81
:10198000FFFFFCFFFFFCF80BFCC003FCD007FCFFD3
:10199000FFFCFFFFE000000700003F00003F0000E9
:1019A0003F00003F00003F00000BFFFFD0FFFFFCA7
:1019B000E00BFCC003FCC003FCF00FFCF00FE000E8
:1019C000000100001F00003F00003F00002F0FFF3C
:1019D000FF0FFFFFFFFFD0FFFFFCE00BFCC003FC8D
:1019E000D003FCFFFFFCFFFFFC00000100001F0014
:1019F000003F00003F00003F00003F00000B555536
:101A000040FFFFF4EFEFFC0FC3FC4FC3FCFFC3FC30
:101A1000FFC3FC000003007FFF03FFFF03FE03037F
:101A2000FD0303FFC000BFC0FC0000FFFFFCFFFF81
:101A3000FCFC0000FC000000000000000000007F33
:101A40000003FF0003FE0003FC0003FD0003FF0092
:101A500000BFFD03F4FFC3FF2FC0BF0FC03F1FC077
:101A60007FFFFFFFFFFFF803FFFF03FFFF000007FB
:101A700000000F00000F00000F000002FFFFFCFF3E
:101A8000FFFCF80000F00000F40000FFFFFCFFFF87
:101A9000FC00000000000000001500FF3F00FF3FB9
:101AA000000000000000000000000000400000FFF7
:101AB000FFFCFFFFFC000000000000000000000031
:101AC0000000000000000000001500FF3F00FF3F85
:101AD0000003F40003FF0000BF00003F40007FFF51
:101AE000FFFFFFFFF800FFFF00FFFF000000000006
:101AF0000100003F00003E000000FFFFFCFFFFFC74
:101B00001FF400FEBF40E00BFC0000BC0000000022
:101B10000000000000000000003FFF003FFF000049
:101B200000000000000000000000000000FFFFFCBB
:101B3000FFFFFC00000000000000000700003F0065
:101B4000003F00000F00003F00003F00000BFFFFC0
:101B5000FCFAAAA8D40000FFC000E80000F5555424
:101B6000FFFFFC00003F00003F00001F00003F009F
:101B7000003F00003F00000BFFFFFCFFFFFCE00008
:101B800000C00000C00000FFFFFCFFFFFC000007DA
:101B900000003F00003F00003F00003F00003F000A
:101BA000000BFFFFD0FFFFFCE00BFCC003FCD007E5
:101BB000FCFFFFFCFFFFE0003FFF003FFF0007FED0
:101BC000000FF0000FF4000FFF0002FFFFFFFCFF0B
:101BD000FFFC02FD0000FF0001FF00FFFF00FFF817
:101BE0000000007F0007FF000FF8000FF0000BF46B
:101BF000003FFF003FFFFFF400FFFF0002FF000077
:101C0000FF0001FE00FFFFFCFFFFFC00003F0000A3
:101C10003F00000700003F00003F00003F00000BB6
:101C2000FFFFFCFFFFFCFE0000E00000D00000FC16
:101C30000000FC000000001F0000FF0000FE00008C
:101C4000FC0000FC0000FF0000BFFD0FD0FFCFFC38
:101C50002FC2FC0FC0FC0FD1FC0FFFFC02FFE00005
:101C6000000301555703FFFF02AAAB000003000069
:101C700000000000FC0000FD5540FFFFF4FEABFC3F
:101C8000FC01FC003FFC003FE000003F00003F0083
:101C9000000000000000000000003F00003FFFFFC8
:101CA000D0FFFFFC000BFC0003FC0007FCFFFFFC67
:101CB000FFFFE000003F00003F00000000000000C8
:101CC000000000003F00003FFFD000FFFD0002FFCA
:101CD000D0003FFC01FFE0FFFE00FFE00000003FFE
:101CE00000002A00000000000000000000001500B5
:101CF000003FFFFFD0AAAFFC0007FC03FFF0000B82
:101D0000FC555FFCFFFFE000003F00002B000000DF
:101D100000000000000000001700003F4001FCF43C
:101D20001FE8BFFE000FF0007FFD00F82FD48002F7
:101D3000FC00003F00003F00000000000000001514
:101D400000003F00003FFD03F4FFC3FC2FC0BC1F99
:101D5000C03CFF807CFFFFFCFFFFF800003F00005D
:101D60003F00003F00003F00003F00003F00003FF9
:101D7000C001FCC01FFCC1FFFCDFFFFCFFE3FCFE59
:101D800003FCE003FC00000000000301400F7FFFA4
:101D9000FFFEAAA8F00000A00000000000C00000A4
:101DA000F00140FFFFFD2AAABF00000F00000A005B
:101DB0000000000000555555FFFFFFAAAAAA000029
:101DC00000000000000000000000555554FFFFFC1B
:101DD000AAAAA8000000000000000000F00000FC1B
:101DE0000000FFFFFD2BEAAF00000300000200002F
:101DF0000000000F00001F1FFFFFFAABE8E000002B
:101E0000800000FD4000FFFD40FC2BFDFC002FFD8D
:101E10000002FFC000FFC0000005FC05FFFCFFA0A2
:101E2000FCE000FC0001FC000FFC000FFC1FFFFFAA
:101E3000FFFFFFFF800FFF000FFF400FFFFFFF2F8F
:101E4000FFFFFFFFD0FFFFFCC00BFCC003FCC0077F
:101E5000FCFFFFFCFFFFE0000000000000000000AE
:101E60000000000000000000000000000000000072
:101E700000000001540003FC0002A80550000FF010
:101E8000000AA000000550000FF0000AA0000000AA
:101E9000000000000000001547003FFE002AA001DE
:101EA0000101FF02EB0202D76802D10102C08007E4
:101EB000C128282828140005C20000000002CB1702
:101EC0000BB4E577F1FFFF4FF1FFFF4F02B0640164
:101ED0001101FF03C7A6E9023620023A1102B80930
:101EE00002D01F0120012902B9E301FF02B9230238
:101EF00072000139004255494C543A205365702014
:101F0000323020323032342031303A35383A3035C0
:101F1000000011241FBECFEFCDBFDFE7DEBF10E40E
:101F2000A0E0B0E4E6EAFFE700E00BBF02C00790E4
:101F30000D92A231B107D9F72DE7A2E1B0E401C0BB
:101F40001D92AB3EB207E1F70E94AE3C0C94D13F2C
:101F50000C9400009091367D81E098279093367D17
:101F6000809307408093064008951092367D81E06B
:101F7000809307408093054080930640089581E058
:101F80008093EA7D10927F42109280428093D569BF
:101F9000E6E3F2E411921586138E11A617AA82E4E5
:101FA000E434F807B9F710928B4210928C421092E9
:101FB0008D4210928F42109290421092CE691092F0
:101FC000CF6910927C4210927D4210927E4280E155
:101FD00080938E421092FB691092D3691092D1695E
:101FE000089580917E42813019F08CE792E4089543
:101FF0008DE792E408958031910508F0C097E6E3FB
:10200000F2E427E0289FB001299F700D112490E091
:1020100080E0DC01A60FB71FAF56BD4B258D30E128
:10202000239FA0011124248D242B2C9301963296FA
:102030008730910571F708958091D169833009F057
:1020400045C08091584290E0982F88279295907FC4
:1020500020915742922B20915542822B209156423B
:1020600040E1249F90011124822B932B292F22954C
:102070002F70283059F59F70FC01EF52FA4A2091D9
:10208000534230E1239FA001112420915242242B7E
:102090002083FC01F695E795F695E795EF52FA490E
:1020A000880F867023E030E0082E01C0220F0A94CA
:1020B000EAF72095908129232083909154429370D0
:1020C00001C0990F8A95EAF7292B20830895CF93B1
:1020D000DF93DC01EB013EE049914D933A95E1F746
:1020E000DF91CF910895CF93DF93342FDC01EB0183
:1020F000231BA30FB11DC30FD11D49914D932A95E9
:10210000E2F7DF91CF910895242FDC01261BA60F63
:10211000B11D1D922A95EAF70895CF93DF93342FCE
:10212000DC01EB01231BA30FB11DC30FD11D4C918B
:1021300058815D9349932A95D2F7DF91CF91089505
:10214000CF93DF93DC01022E000C330B51E0E42F20
:10215000F0E02E173F071CF4DF91CF91089580E047
:102160006115710521F0EB01CE0FDF1F8881EA0FA9
:10217000FB1F9081C091D5699C0F980F908380912F
:102180008E42981730F0981B90835093D5694F5F1B
:10219000DECF1092D569FBCF0F93FC0131E002171F
:1021A00014F40F91089590E06115710531F0DB0191
:1021B000A20FB11D27FDBA959C9180E041155105F4
:1021C00031F0DA01A20FB11D27FDBA958C91981B51
:1021D0008091D569981B97FF0FC080918E42980F10
:1021E0003093D569309731F0DF01A20FB11D27FD83
:1021F000BA959C932F5FD3CF1092D569F3CFCF932D
:10220000DF93242FEC01C60FD11D261B4981499372
:102210002A95E2F71A92DF91CF910895CF93DF9339
:10222000DC011092D5692417A4F0E42F042E000CD1
:10223000FF0B90E06115710521F0EB01CE0FDF1F60
:102240009881EA0FFB1F8081891731F081E080932C
:10225000D569DF91CF9108954F5FE5CFA3E8B2E450
:102260008D919C911197E5E8F2E4208131812D93C5
:102270003C93A7E8B2E42D913C91119720833183E0
:10228000E9E8F2E4208131812D933C9310821182A0
:10229000089508950E942E1180937F42909380426A
:1022A00008950C942E110E942E11E6E3F2E4292FDA
:1022B00022952F7022A39F7091A3982F92959F70C3
:1022C00090A38F70878F0895E6E3F2E482A1829550
:1022D00091A1892B90A19295278D922BEFE7F2E4A3
:1022E0009083818308958295837090E09C01220FF2
:1022F000331F227095958795822B90918242292FCA
:1023000022952F7030E096E1929FF001939FF00D9F
:102310001124E25DFF4B9589EEE2F0E444E0840293
:1023200090011124458949130CC0DF01A20FB31F8E
:102330004D915D916D917C91452B462B472B09F07A
:10234000848B769641E4EE38F40761F7089562E5F0
:1023500072E480E692E40C94671060E672E482E531
:1023600092E40C94671062E572E48EE692E40C94B9
:1023700067106EE672E482E592E40C946710E6E37F
:10238000F2E4968D858D8295807F248D822B8093BB
:10239000F9699093FA691092A7411092A8410895A3
:1023A000E6E3F2E4858D20E1829FC0011124248DB3
:1023B000822B8093A7419093A841089582958F70B6
:1023C0008093D06985E08093FB69089510928F42D5
:1023D0000895E6E3F2E4858D90E1899F9001112450
:1023E000848D822B80938F420895E6E3F2E48091FE
:1023F0008F42982F9F70948F82958F70858F08954C
:10240000E6E3F2E4AFE8B2E48C91958D40E1949F6D
:1024100090011124948D922B9C93982F9F70948FF0
:1024200082958F70858F089580918F4280938D4221
:1024300080EA80930704089580918D4280938F42B3
:10244000089580918F4290918D4290938F42809316
:102450008D4280EA8093070480910240811109C077
:1024600088ED9DE1809303409093044081E0809348
:10247000024008950E94F10FFC019081911103C068
:102480008DE0808308959150908308950E94F10F0C
:10249000FC0190819F5F90830E94F10FFC012081DD
:1024A0002E3008F01082089510927E42089581E047
:1024B00080937E42089590917C4280917D42981352
:1024C00003C081E08093D5690895CF93C82F0E94FF
:1024D000F10FDC01EC91F0E0EA5CFD4BC295CF70AE
:1024E000C48F0E94F10FFC019081911104C08DE016
:1024F0008083CF91089591509083FBCFCF93DF934A
:102500000E94F10FDC01EC91D0918C42C0918B4282
:10251000ED30B1F480911440982F9F7B953B11F0E2
:10252000873F49F4C0935F42D0938B42C0938C4263
:10253000DF91CF910895D0935F42C0935242F8CF7C
:10254000809113408D3079F580911440853F61F082
:10255000982F9F70973039F582958F70982F977FBD
:10256000973009F18B30F9F0D0938B42C0938C42B5
:102570000E94F10FDC01EC91F0E0EA5CFD4BC58FAD
:102580000E94F10FDC01EC91F0E0EA5CFD4BD48F8E
:102590000E94F10FDC01EC91F0E0EA5CFD4B858DCF
:1025A00080935242C5CFF0E0EA5CFD4BD58F0E948C
:1025B000F10FDC01EC91F0E0EA5CFD4BC48FB8CF89
:1025C000CF93DF930E94F10FDC018C91C0918B427D
:1025D0008D3001F59091144080915F42292F2F7B1F
:1025E000253B11F0973F49F480938C4280938B42B6
:1025F000C0935F42DF91CF91089590918C422091DA
:10260000524220938B4280938C4290935F42C093BE
:102610005242F0CF20911340D0918C4290E02D3067
:1026200099F520911440253F61F0322F3F703730EB
:1026300059F522952F70322F377F373029F12B3003
:1026400019F18A5C9D4BFC01858D80938C420E9420
:10265000F10FDC01EC91F0E0EA5CFD4B848D80939E
:102660008B420E94F10FFC0190915242E081F0E018
:10267000EA5CFD4B958F0E94F10FDC01EC91F0E0DC
:10268000EA5CFD4BD48FC3CF8A5C9D4BFC01858DEA
:1026900080938C420E94F10FDC01EC91F0E0EA5C47
:1026A000FD4B848D80938B420E94F10FDC01EC91F5
:1026B000F0E0EA5CFD4BD58F0E94F10FDC01EC915C
:1026C000F0E0EA5CFD4BC48F95CF8091354280935A
:1026D0007F42089580913542E6E3F2E4982F929587
:1026E0009F7090A38F70878F08958091377D909110
:1026F000387D892B91F08091377D9091387D0197BD
:102700008093377D9093387D81E09091A64191111F
:1027100001C080E08093D56908958091D3698230AB
:1027200099F71092D3691092A64110923542809188
:10273000284290E0E5CF089580E180938E4208958D
:102740008AE080938E420895E6E3F2E482A18295C6
:1027500091A1892B90A19295278D922B90932C403B
:1027600080932D4082E08093FB690895E6E3F2E4D4
:10277000968F982F92959F70958F8F70848F10925F
:10278000FB69089583E08093FB690895CF93DF93FD
:10279000CDB7DEB72E97CDBFDEBF82958F70E82F05
:1027A000F0E0E95DFC4FE491DE0111969E01215FAE
:1027B0003F4FBD0181E08E0F0E2E000CFF0BEA5C37
:1027C000FD4B948D9D93E0E08E300CF4E82FA21722
:1027D000B30781F782E592E40E9467102E96CDBF81
:1027E000DEBFDF91CF91089580912A422AE0829F37
:1027F000C00111242091467D3091477D82179307B7
:1028000020F081E08093D56908951092D5690895EC
:1028100084E08093FB690895F89480910E6A882380
:10282000B9F0E0910C6AF0E0E450F64980819091B3
:102830000C6A9F5F90930C6A90910C6A9F709093C2
:102840000C6A90910E6A915090930E6A7894089554
:1028500080E0FCCF9091240895FFFCCF8093220864
:1028600008952EE0FC0111922A95E9F7089586E378
:1028700092E40E94311484E492E40E94311482E5CF
:1028800092E40C943114E1E9F2E48DE397E2DF0184
:102890009C011D9221503040E1F70895CF93DF93C2
:1028A000DC01FC013B966B3061F41B968C911B970D
:1028B00092919183EA17FB07D9F78083DF91CF913B
:1028C00008958C91ED0199819993CE17DF07D9F77F
:1028D0001B968C93F3CF9C014097C09788F02115ED
:1028E00082E0380769F0C901805F9240419740F06B
:1028F0008091D16980FD06C081E0203F334030F0F7
:1029000080E004C081E0203F3240D0F708958091FC
:102910003442882331F00E942E1180937F4290939D
:1029200080420895CF93DF938091A7419091A84171
:10293000009731F08D3F910589F0DF91CF91089597
:10294000C091F969D091FA69CE010E946B14882375
:10295000A1F3CE01DF91CF910C94FB0F2091544253
:102960008091534230E1839FC0011124922B20912A
:102970005242822B8093327D9093337D81E080930D
:102980000640DBCF0E94F10FDC01EC91ED30A1F4A9
:102990009091144080915F42292F2F7B253B11F0AD
:1029A000973F39F490918C4290938B4280938C4264
:1029B000089590915242F8CFF0E0EA5CFD4B848D8F
:1029C00080938B42858DF2CF8091377D9091387DB9
:1029D000892B51F08091377D9091387D01978093BC
:1029E000377D9093387D08958091D3698130D9F7F0
:1029F0008091B6418111F7CF82E08093D3698091B5
:102A0000284290E0ECCF8EE0815078F480913442FF
:102A1000882351F08091D2698D3031F480915242F7
:102A200080935F42809343420895E82FF0E0EA5C90
:102A3000FD4B948D20819223948FE6CFCF93DF932B
:102A4000A2E5B2E4CEE6D2E43EE04C9158815D933B
:102A500049933A95D1F7DF91CF910895CF9382951D
:102A60008F70E82FF0E0E95DFC4FC4910E94F10FF8
:102A7000FC01C083CF91089582958F70E82FF0E01C
:102A8000E95DFC4FE491AFE8B2E421E030E002C040
:102A9000220F331FEA95E2F78D919C911197822BBB
:102AA000932B8D939C93089582958F70E82FF0E07F
:102AB000E95DFC4FE491AFE8B2E481E090E002C050
:102AC000880F991FEA95E2F7809590952D913C919A
:102AD0001197822393238D939C93089582958F70F1
:102AE000E82FF0E0E95DFC4FE49181E090E002C066
:102AF000880F991FEA95E2F720918F42309190421A
:102B00008223932321E0892B09F420E02093D569C7
:102B100008952091CE693091CF6982958F70E82F0A
:102B2000F0E0E95DFC4FE49181E090E002C0880FA5
:102B3000991FEA95E2F78223932321E0892B09F478
:102B400020E02093D5690895CF93C82F0E94F10FFC
:102B5000C295CF70EC2FF0E0E95DFC4FE491DC0111
:102B60008C910E2E000CFF0B8E171F0619F481E0BE
:102B70008093D569CF910895CF93DF93A2E5B2E416
:102B8000C0E6D2E43EE04C9158815D9349933A957A
:102B9000D1F7DF91CF91089580913442811106C021
:102BA0000E942E1180937F42909380420895E6E325
:102BB000F2E482A1829591A1892B90A19295278D13
:102BC000922BE7E8F2E4208131812093894230930F
:102BD0008A42A5E8B2E42D913C911197208331837C
:102BE000E3E8F2E4208131812D933C93908381834B
:102BF00008958EE0815078F480913442882351F01A
:102C00008091D2698D3031F48091524280935F423D
:102C1000809343420895E82FF0E0EA5CFD4B948DE9
:102C20002081922B948FE6CFE0E4F4E081818D60E7
:102C30008183E0E0F4E0818180648183E0E6F9E073
:102C400084E0818381E38083089580936409809187
:102C5000630987FFFCCF08951F93CF93DF93C0E0F4
:102C6000D4E010E41E830E9425161D83DF91CF91CE
:102C70001F91089527E731E0829FF001839FF00DB7
:102C80001124E15FF54920E0818192819695969526
:102C900030E4839FA0011124942B92839081869528
:102CA000869530E4939FA0011124842B818396950F
:102CB000969590832F5F33962D3731F7089527E748
:102CC00031E0829FF001839FF00D1124E15FF5490F
:102CD0002DE781819081990F990F382F3295369584
:102CE00036953370932B90839281880F880F392FFC
:102CF0003295369536953370832B8183990F990FD2
:102D00009283215033962111E4CF0895EFE0FAE643
:102D10008DE190E1DF019C011D9221503040E1F7EF
:102D20000895EFE0FAE69191DF01119798279C93BF
:102D30009AE7EC32F907B9F7089527E731E0829F67
:102D4000F001839FF00D1124E15FF5499F012251AD
:102D50003D4F8191DF01119786768C93E217F3073F
:102D6000C1F7089527E731E0829FF001839FF00DBE
:102D70001124E15FF549629FD001639FB00D1124DA
:102D8000A15FB549CF0189589E4F21912D93E81736
:102D9000F907D9F7089570E027E731E0482F429FFF
:102DA000C001439F900D112447E751E0815F954991
:102DB0000C94CA3FFF920F931F93CF93DF93182F6A
:102DC000F62E8AE20E942C1689E1810F0E942516B8
:102DD00089E18F0D810F0E9425168BE20E942C162F
:102DE00080E00E9425168CE70E9425168CE20E9446
:102DF0002C1687E791E0189FE001199FD00D112450
:102E0000C15FD549F89E8001F99E100D11240C0F69
:102E10001D1FC017D10731F4DF91CF911F910F9182
:102E2000FF90089589910E942516F3CFCF93DF93E9
:102E30008F773CE0839FC0011124895A9C4FC62F95
:102E4000C695E7E7F1E04E9FD0014F9FB00D1124EA
:102E5000A15FB54933E0C39FE00111248A1B9B0B9E
:102E600060FF30C0AE014D5F5F4FCA0FDB1FA40F84
:102E7000B51F3CE0841B950BFC01EA0FFB1F2636B7
:102E8000F1F0E491E22748814A7A48834C914575F4
:102E90004C93F0E0AF0155954795542F55754881F7
:102EA000452B4993EE0FFF1FEA7A4C91E42BED93EB
:102EB000315011F788E0860FDF91CF910895E491AA
:102EC000E676E1CFAC0FBD1F3CE08C1B9D0BFC01F7
:102ED000EA0FFB1F263641F0E491E227EC933150D4
:102EE00011963111F4CFE6CFE491E676F7CFFF9259
:102EF0000F931F93CF93DF938C01D42FF22EC0E05A
:102F0000F801EC0FF11D8081811107C0862FDF9140
:102F1000CF911F910F91FF9008952F2D4D2F0E945B
:102F20001617682FCF5FECCFFF920F931F93CF93AD
:102F3000DF938C01D42FF22EC0E0F801EC0FF11DCD
:102F40008491811107C0862FDF91CF911F910F913E
:102F5000FF9008952F2D4D2F0E941617682FCF5FD9
:102F6000ECCFCF92DF92EF92FF920F931F93CF930C
:102F7000DF93C42FD22F00E318E721E03327680145
:102F80007901C80ED91EE11CF11C10E0D701C60161
:102F9000810F911DA11DB11DABBFFC018791811156
:102FA0000AC0862FDF91CF911F910F91FF90EF9074
:102FB000DF90CF9008952D2F4C2F0E941617682F69
:102FC0001F5FE4CF5F926F927F928F929F92AF923A
:102FD000BF92CF92DF92EF92FF920F931F93CF9306
:102FE000DF93CDB7DEB72597CDBFDEBF89836A8378
:102FF0004B832C830D83EEE3F7E7A6E8B7E7108257
:10300000118212821C9211961C92119712961C9298
:103010001297E55BFF4FA55BBF4F28E7E53BF20743
:1030200071F76AE089E00E94B216CE0101965C0158
:1030300010E000E096E0692E22E3822E912C80E3DE
:1030400098E7A1E0BB27F501C1905F01C69C600134
:1030500011240D2C000CEE08FF088C0D9D1DAE1DDB
:10306000BF1DAC01BD014D5A5E4F6F4F7F4F6BBF0F
:10307000FA0177906C017D01F4E5CF0EF1E0DF1EDF
:10308000E11CF11CB40128E0729E60197109112441
:1030900077FF02C06F5F7F4F75956795600F711F57
:1030A000512C57101BC00E5C1F4F0A3F110509F031
:1030B000C6CF89E02596CDBFDEBFDF91CF911F91AE
:1030C0000F91FF90EF90DF90CF90BF90AF909F90C7
:1030D0008F907F906F905F900C943A16EBBEF60144
:1030E00087912FEF49E00E941617682F53948FEFB6
:1030F000C81AD80AE80AF80AD4CF99E1899F802D26
:10310000112461E0282F260F30E0A901440F551F3C
:10311000240F351F215F3549F901E15DF24F9081A0
:10312000492F440F440FD901A05DB24F9C91929555
:10313000969596959370942B90839C91492F440F6C
:10314000440F329690819295969596959370942B14
:103150009C93408194E0499FA001112443604083E7
:103160002A55314FF90110826F5F683159F6089581
:103170002F923F924F925F926F927F928F929F9287
:10318000AF92BF92CF92DF92EF92FF920F931F9375
:10319000CF93DF9380E090E8A1E0BB276C017D0135
:1031A00028E7D20EE11CF11C0E94861630E020E0D8
:1031B00087E7882E99249394A1E0B0E05524539496
:1031C00050E040E0289D3001299D700C389D700C26
:1031D000112426C0EBBEF60117918FEFC81AD80A4A
:1031E000E80AF80A90E0EBBEF6018791EFEFCE1AFD
:1031F000DE0AEE0AFE0A980F092F0095C92FC81B98
:10320000811111C015259A3F70F3625071096E3F0C
:103210008FEF7807F9F64F5F5F4F4330510539F173
:1032200066E070E0D7CF113001F5C695D0E0FE0121
:10323000EE0FFF1FEC0FFD1FE60DF71DE15FF549D7
:10324000E40FF51FC02FC80FC0FBAA24A0F8B12CB3
:10325000E501C60FD71F1D0102C0220C331CCA9501
:10326000E2F7E101D081CD2BC0838150C7CF2F5F22
:103270003F4F2B30310509F0A3CFDF91CF911F9144
:103280000F91FF90EF90DF90CF90BF90AF909F9005
:103290008F907F906F905F904F903F902F90089508
:1032A000BF92CF92DF92EF92FF920F931F93CF9333
:1032B000DF93362F9AE2899F80011124095A164F15
:1032C00083E0689F70011124B0E0A0E085E1B82E92
:1032D00050E097E7C92EDD24D3948A2FAA32B10596
:1032E00061F487E0830FDF91CF911F910F91FF90E1
:1032F000EF90DF90CF90BF900895FD01E00FF11F98
:10330000E4916B2D0E947C3EBA01680F711D6C9D8B
:10331000E0016D9DD00D7C9DD00D1124CE0DDF1DE3
:10332000C90FD11DC15FD549E227E8831196D5CFDA
:10333000CF92DF92EF92FF920F931F93CF93DF9381
:10334000D62E92E1899FE0011124C95AD14E83E023
:10335000689F8001112430E020E089E0C82E50E011
:1033600097E7E92EFF24F394822F2231310559F497
:1033700083E08D0DDF91CF911F910F91FF90EF9022
:10338000DF90CF900895F901EC0FFD1FE4916C2DB3
:103390000E94883EBA01680F711D6E9DD0016F9D1D
:1033A000B00D7E9DB00D1124A00FB11FA90FB11D4E
:1033B000A15FB549EC932F5F3F4FD6CFCF92DF92FD
:1033C000EF92FF920F931F93CF93C42F00E318E760
:1033D00021E0332768017901C80ED91EE11CF11CD8
:1033E000EBBEF6018791811109C0862FCF911F9105
:1033F0000F91FF90EF90DF90CF90089520E04C2F39
:103400000E94501963E0680F8FEFC81AD80AE80AC3
:10341000F80AE6CF80E10C942C1681E10C942C166E
:10342000262F2150330BF901ED50FD4FE49191E02F
:10343000633008F090E0891B282F26952695280FE9
:103440003327331F64E60E947C3EB901681B710973
:10345000CB018E0F911D840F911D67E070E00E94DB
:10346000AA3E8F5F0895823021F4637081F48DE16C
:1034700008958150990B67E070E00E94AA3E62E0D7
:1034800070E00E94AA3E9FE1981B892F08958CE16D
:1034900008958D3010F08C500895811101C08CE09A
:1034A0000895CF93DF931092367D85E080931C4280
:1034B000E0E2F0E4CAE3DDE7ABEEB9E6119219927F
:1034C0001D9280E4EC32F807C9F71092327D109219
:1034D000337DDF91CF91089560E089E00E94CB16A3
:1034E0008091327D80FF07C020E049E060ED8CEEE6
:1034F00092E00E9494178091327D81FF07C020E006
:1035000049E06AEA86EE92E00E9494178091327D4B
:1035100082FF06C020E049E06CE984E30E941617B0
:103520008091327D83FF06C020E049E064E983E3B7
:103530000E9416178091327D84FF06C020E049E08A
:103540006CE882E30E9416178091327D85FF06C0E9
:1035500020E049E064E881E30E9416178091327D03
:1035600086FF06C020E049E06CE780E30E94161762
:103570008091327D87FF07C020E049E06EE48FED47
:1035800092E00E9494178091327D9091337D90FF5C
:1035900007C020E049E060E38AED92E00E949417C2
:1035A0008091327D9091337D91FF06C020E049E00B
:1035B00068E287E40E9416178091327D9091337DF6
:1035C00092FF07C020E049E062E084ED92E00E94B3
:1035D00094178091327D9091337D88279370892B49
:1035E00039F420E049E060E38FEC92E00E94941708
:1035F00089E00E943A1661E089E00C94DA160F9394
:103600001F93CF93DF938091367D882331F107EFAD
:1036100019E62AE33DE7C0E2D0E4EEE8F1E46BEE20
:1036200079E6D9011B969C91D8018E918D01B4E069
:103630008B9FA0011124892F8370842B8295807F1A
:103640004B85840F868B96959695978B21503109E3
:10365000219732976017710721F7DF91CF911F9162
:103660000F9108951F93CF93DF93182F88E1EEE811
:10367000F1E4AAE1BDE701900D928A95E1F760E0DF
:10368000812F0E94CB1660E081E0810F0E94CB1653
:10369000CEE8D1E485E020E0412F682F8E890E949A
:1036A0005019412F682F8F890E949819229791E411
:1036B000C637D90781F78091327D9091337D837031
:1036C0009927892B49F420E048E061E088E5DF9103
:1036D000CF911F910C941617DF91CF911F910895F0
:1036E000EEE8F1E4AAE1BDE791918D91981306C04F
:1036F00081E4E53AF807C1F781E0089580E0089594
:10370000DC011E96FB013E963E912291321305C0CC
:10371000A817B907C9F781E0089580E00895FC0172
:10372000108211821282138214820895DC01159690
:10373000FB0135963E912291231728F0321728F08D
:10374000A817B907B9F781E0089580E008956F924E
:103750007F928F929F92AF92BF92CF92DF92EF9221
:10376000FF920F931F93CF93DF938B01DB011D9289
:103770001D921D921C921397EC0122963C01BEE013
:103780006B0E711CC12CD12C7601C394A991B0E0B1
:10379000A70196010E94F03EF80180809180A280EE
:1037A000B380DC01CB01880D991DAA1DBB1D808350
:1037B0009183A283B383AAE0B0E00E94F03E6B0144
:1037C0007C016C167D0611F7DF91CF911F910F914F
:1037D000FF90EF90DF90CF90BF90AF909F908F9031
:1037E0007F906F900895AC0190E070E0292F092E32
:1037F000000C330B261737070CF00895240F351FE4
:10380000F90110829F5FF2CF4F925F926F927F9289
:103810008F929F92AF92BF92CF92DF92EF92FF92E0
:10382000CF93DF9300D000D0CDB7DEB7F894BE01C0
:103830006F5F7F4F88EC91E40E94A71B7894C9804A
:10384000DA80EB80FC808CE3882E912CA12CB12CAB
:10385000C701B601A50194010E94BE3E60932242B9
:10386000CA01B901A50194010E94BE3E60932142A4
:10387000C701B60120E13EE040E050E00E94BE3EBC
:10388000CA01B90128E130E040E050E00E94BE3EAC
:1038900060932042809120420E94491A80932D42D9
:1038A000C701B60120E831E541E050E00E94BE3E8C
:1038B00069017A01C982DA82EB82FC82CA01B9010C
:1038C0006C557C498F4F9F4F22E0660F771F881FF2
:1038D000991F2A95D1F721EB3AE342E050E00E948C
:1038E000BE3E215F3F4F4F4F5F4F82EAC80E8FEDC4
:1038F000D81E84E2E81EF11CC20ED31EE41EF51E83
:1039000062E056954795379527956A95D1F7C21A83
:10391000D30AE40AF50AA4E1B0E0A70196010E94E7
:10392000F03E2B013C012AE8421A29E0520A6108C4
:103930007108C301B20129E83CE140E050E00E9477
:10394000BE3E49015A01ADE6B1E00E94F03EC61A02
:10395000D70AE80AF90AC301B20124E232E740E0DB
:1039600050E00E94BE3EC21AD30AE40AF50AA8EE4D
:10397000B3E0A70196010E94F03E29E837E740E056
:1039800050E00E94BE3E29013A018EE1289FC018F6
:103990001124A9E5B2E00E94F03E28EE33E040E0B9
:1039A00050E00E94BE3EC21AC09225422EE042164E
:1039B00051046104710480F58CE6881A82E1980A4A
:1039C000A108B10821E0421A51086108710880E39A
:1039D000880E809223424092244240912542609179
:1039E0002442809123420E94101A80932E4281E04B
:1039F000809317402496CDBFDEBFDF91CF91FF901B
:103A0000EF90DF90CF90BF90AF909F908F907F907E
:103A10006F905F904F9008958BE6881A82E1980A24
:103A2000A108B1082DE0421A510861087108CFCFF2
:103A30002F923F924F925F926F927F928F929F92BE
:103A4000AF92BF92CF92DF92EF92FF920F931F93AC
:103A5000CF93DF93CDB7DEB72997CDBFDEBFC09040
:103A600023420C2C000CDD0820E3C21A28EFD20AF6
:103A70000D2C000CEE08FF0830912442232E022C5E
:103A8000000C330829823A8291012330310548F431
:103A9000245F3F4F29833A8331E0C31AD108E108FC
:103AA000F10810912542ADE6B1E0A70196010E9410
:103AB000F03E4601570122E0B694A794979487946C
:103AC0002A95D1F7860E971EA81EB91EC701B6010A
:103AD00020E931E040E050E00E94BE3E820E931E9D
:103AE000A41EB51EC701B60124E630E040E050E058
:103AF0000E94BE3E821A930AA40AB50A29813A811D
:103B00002F5F3F4FC901880F991F820F931F65E0F8
:103B100070E00E94963E2EE129803A80229DC001ED
:103B2000239D900D1124810F911D17FD9A95FB0186
:103B3000E80FF91F9F0150E040E060E070E0CB012A
:103B4000E9833A834B835C836D837E838F8398877D
:103B50009401A50160E070E080E090E0A980BA8067
:103B6000C12CD12CE12CF12C00E010E00E94B23FDE
:103B70002A5E36494A405109610971098109910952
:103B8000E0E8AE2EF1E5BF2ECC24C3940E94FB3EAC
:103B900059016A017B018C01A09120424091214290
:103BA000409022420A2E000CBB0B20E13EE00E9416
:103BB000E93E042C000C550866087708DC01CB01AF
:103BC000840D951DA61DB71D3CE34302A0011124E1
:103BD000840F951FA11DB11D1C012D01612C712C9D
:103BE00043013A82AB835C826D827E828F829886AB
:103BF0009C01AD0160E070E080E090E00E94B23F87
:103C000029014A01698779831C01F8941092D469CB
:103C1000AAEC6A2EA1E47A2E8AE0A82EB12CC12C3F
:103C2000D12CE12CF12C00E010E09201A401698577
:103C30007981C1010E94533FF30121933F01920119
:103C4000A40169857981C1010E94553F29014A017A
:103C5000698779831C0126ED31E426153705E1F6E5
:103C600068EC71E480E092E40E94671078942996F1
:103C7000CDBFDEBFDF91CF911F910F91FF90EF90ED
:103C8000DF90CF90BF90AF909F908F907F906F907C
:103C90005F904F903F902F900895FC0195E020E0B9
:103CA0008191980FDF0111979A3060F49C9390E016
:103CB000211101C09E5F2F5F2E3011F09111F0CFC6
:103CC000892F08959A509C9391E0F2CFCF93803141
:103CD00008F04AC0E82FF0E0E059F14E0C94E03EC5
:103CE000801E8D1EA51EB61EEE1E051FB41E1B1FB8
:103CF000211F341F451F4D1F551F5D1F651F691F65
:103D00008091C7412EE0829FC001112462E572E4D8
:103D100088539E4BCF910C9467108091C741CEE0A1
:103D20008C9FC001112462E572E488539E4B0E946F
:103D30006710E091C741CE9FF0011124E954FE4B7A
:103D4000118A128ACF910C94041C8091C7412EE0F5
:103D5000829FC001112462E572E48C519E4B0E9447
:103D6000671081E080931740CF9108958091C741FB
:103D7000811126C09091B7412091534280E1289F44
:103D80009001112480915242806C822B8923809370
:103D9000B7418091B7418F7339F78091CE69909187
:103DA000CF699F7D8093CE699093CF698091CE69D2
:103DB0009091CF699F7E8093CE699093CF69D4CF45
:103DC00023E040E063E572E489EB91E40E94731024
:103DD0008091BC4181708093BC41C6CF8091C74126
:103DE0002EE0829FC001112462E572E480509E4B58
:103DF0000E94671080910F4282FD04C081E0809391
:103E00001F42B2CF10921F42AFCF24E040E062E5E4
:103E100072E482EC91E40E9473108DEB91E40E94B5
:103E20008F1B8091B7419091B84194608093B741C6
:103E30009093B84199CF8091B7419091B8419B7FC1
:103E4000F5CF4091B7415091B8412091C741255FCE
:103E500081E090E002C0880F991F2A95E2F78095D3
:103E6000909584239523E2CF4091B7415091B8417A
:103E70002091C741255F81E090E002C0880F991F23
:103E80002A95E2F7842B952BD1CF4091B7415091E1
:103E9000B8412091C741285FDBCF4091B741509195
:103EA000B8412091C741285FE6CF4091B74150917A
:103EB000B8412091C7412A5FCBCF4091B741509183
:103EC000B8412091C7412A5FD6CF81E08093C74196
:103ED0004BCF1092C74148CF7F928F929F92AF9263
:103EE000BF92CF92DF92EF92FF920F931F93CF93E7
:103EF000DF93082F02950F70C02FD0E0E090F96992
:103F0000F090FA6920EFE22223E0F222E02AFD2A73
:103F1000E092F969F092FA69C7010E946B14182FB8
:103F2000882381F0C701DF91CF911F910F91FF90FE
:103F3000EF90DF90CF90BF90AF909F908F907F9049
:103F40000C94FB0F8091A7419091A8418B3F910564
:103F500009F469C08D3F910541F5C154DD4FFE0163
:103F6000C49180E0C7FD8BE0FC2FFF709F2E00E026
:103F70002C2F2071822EDBE0D81B90E0FC01E05E4C
:103F8000FF4B7F01FC2FF0727F2E9C01265C324894
:103F90006901C074FC01E551F6495F01901213C03C
:103FA00081E08093074080930540DF91CF911F917E
:103FB0000F91FF90EF90DF90CF90BF90AF909F90C8
:103FC0008F907F900895882069F06D2F80E290E4B3
:103FD0000E944E14E12FF0E0EA5CFD4B848DF70166
:103FE00080831F5F772069F06D2F8AE39DE70E9431
:103FF0004E14E12FF0E0EA5CFD4B848DF6018083E6
:104000001F5FCC2371F06D2F8BEE99E60E944E144A
:10401000E12FF0E0EA5CFD4B848D8170F501808337
:104020001F5F0F5FBBCF802FDF91CF911F910F914B
:10403000FF90EF90DF90CF90BF90AF909F908F90C8
:104040007F900C94661E8230A1F038F08430E9F144
:10405000C8F0853009F442C008956091C7418EE0F0
:10406000689FB001112468537E4B82E592E40C9462
:1040700067106091C7418EE0689FB00111246C51B8
:104080007E4BF3CF8091C741811117C08091B7411A
:104090008F70809352428091B74182958F70809348
:1040A00053428091B8418F70809354428091B841BF
:1040B0008295817080935542089523E040E069EB3A
:1040C00071E483E592E40C9473106091C7418EE033
:1040D000689FB001112460507E4BC7CF24E040E0C0
:1040E00062EC71E482E592E4EECF6F927F928F9260
:1040F0009F92AF92BF92CF92DF92EF92FF920F9377
:104100001F93CF93DF93182F12951F7082E592E4CF
:104110000E9431148091A7419091A8418B3F910555
:1041200009F4B9C08D3F910509F440C0892B79F598
:10413000112359F08091F9699091FA69807F937009
:10414000812B8093F9699093FA690091F969109134
:10415000FA69C8010E946B148823C9F00031110567
:1041600010F00053110987E0809FE001819FD00D7E
:104170001124CF56DD4BA2E5B2E467E04991542FFC
:1041800052955F704F704D935D936A95B9F7DF91CB
:10419000CF911F910F91FF90EF90DF90CF90BF9044
:1041A000AF909F908F907F906F900895153001F59C
:1041B0008091327D9091337D909354429C0194E0A4
:1041C000369527959A95E1F72F70209353428F707B
:1041D000809352428091367D8823C9F21330B8F221
:1041E0001530A9F281E08093074080930540CFCF3E
:1041F000E12FF0E0E155FD4FC4910BE0C7FF00E077
:104200002C2F2F70822ED0E0912C3C2F3071732EEA
:10421000802F90E0DC01A05EBF4B7D01BC2FB0720F
:104220006B2E9C01265C32486901C074DC01A551EB
:10423000B6495D01891471F2772069F0ED2FF0E045
:10424000EA5CFD4BD7018C91848FDF5F602F80E2A9
:1042500090E40E944E14662069F0ED2FF0E0EA5CD5
:10426000FD4BD6018C91848FDF5F602F8AE39DE741
:104270000E944E14CC2369F0ED2FF0E0EA5CFD4B78
:10428000D5018C91848FDF5F602F8BEE99E60E94C1
:104290004E149394CFCF812FDF91CF911F910F9127
:1042A000FF90EF90DF90CF90BF90AF909F908F9056
:1042B0007F906F900C9423206EE088EC91E40E9434
:1042C000F31B6EE084EE91E40E94F31B6EE080E04D
:1042D00092E40E94F31B6EE086ED91E40E94F31BD2
:1042E0006EE082EF91E40E94F31B6EE08EE092E4B8
:1042F0000E94F31B64E089EB91E40E94F31B8DEBB9
:1043000091E40E948F1BE7EBF1E4108A8081918198
:104310008064808391838081918191608083918387
:104320004AE050E069E070E085EF91E40E94CA3F06
:1043300088E080930F420C94181D6F927F929F9299
:10434000AF92BF92CF92DF92EF92FF920F931F93A3
:10435000CF93DF93EEE2F0E480E691E0DF019C0191
:104360001D9221503040E1F7E8E4FDE782EADF01E9
:104370001D928A95E9F740E058EFDF0120E066E002
:10438000A62E00E014E176E1B72E99249394FA0169
:1043900034913196D4913196C4913196E49111962D
:1043A0003C9311971796CC9317971896EC93189700
:1043B000303108F051C0822F6A2D0E947C3E909FC0
:1043C0006001919FD00C11240D2C000CEE08FF0809
:1043D000813009F456C0823009F458C060E070E8BA
:1043E00080E09927C60ED71EE81EF91E1296CD92C0
:1043F000DD92ED92FC921597632F70E06D2E712C7B
:104400002630D0F49C92B69E7001B79EF00C112419
:10441000C301880F991F880F991F8E0D9F1D825D04
:104420009F4B1296CD90DD90ED90FC901597FC017E
:10443000C082D182E282F3821696DC931697B69EF2
:10444000C001B79E900D1124825D9F4BF301E80FD0
:10445000F91F208BFC01C58B2F5F4C5F5F4F1996B6
:10446000223109F094CFDF91CF911F910F91FF90EE
:10447000EF90DF90CF90BF90AF909F907F906F9024
:10448000089560E370E081E09927ACCF60E070E8C8
:1044900081E09927A7CFE62FE69527E0AC01249F7E
:1044A000C001259F900D11248A5C9D4BE80FF92FC8
:1044B000F11DE55AFF4F808160FD82958F70089550
:1044C000CF92DF92EF92FF92BC01672F7727629520
:1044D0006F7026E1269FA001279F500D1124FA013D
:1044E000E25DFF4B248934E0239FF0011124E40FA7
:1044F000F51FE25DFF4BC080D180E280F380C114E4
:10450000D104E104F10409F43FC09F709C01369589
:10451000279536952795DC01AA0FBB1FA670BB27F0
:104520004091D1694330C1F468307105A9F48F52CC
:104530009A4AFC0180812F523A49F901408150E0AA
:1045400002C055954795AA95E2F74370942FFF90C6
:10455000EF90DF90CF900895B701A601480F591F43
:10456000611D711D6BBFFA014791842FA90170E095
:1045700060E0505F6F4F7F4F4C0D5D1D6E1D7F1DC6
:104580006BBFFA014791DBCF80E090E0E0CF8091F4
:104590000E6A8823E1F30E940C1490ED980F9A3074
:1045A00030F09FE9980F963020F499EA980F892F00
:1045B00008959FEB980F963010F499ECF7CF803266
:1045C00031F390E0F4CF8A3310F08755089580538B
:1045D0000895F894ECEFF9E6108A118A128A78941B
:1045E0000895F89490910E6A9031B1F0E0910D6ABF
:1045F000F0E0E450F649808380910D6A8F5F8093EC
:104600000D6A80910D6A803110F010920D6A8091D0
:104610000E6A8F5F80930E6A7894089580912408C3
:1046200086FFFCCF08951F920F920FB60F921124B0
:104630000BB60F928F93EF93FF93E0910D6AF0E02A
:1046400080912008E450F649808380910D6A8F5F45
:1046500080930D6A80910D6A8F7080930D6A8091AE
:104660000E6A8F3028F480910E6A8F5F80930E6AF5
:10467000FF91EF918F910F900BBE0F900FBE0F9097
:104680001F901895CF92DF92EF92FF92CF93DF9316
:1046900040E050E061E077276A017B01C80ED91E37
:1046A000E11CF11CD0E0D701C6018D0F911DA11DA9
:1046B000B11DABBFFC01C7918C2F0E942A14DF5F94
:1046C000CA3089F7DF91CF91FF90EF90DF90CF90C4
:1046D0000895813408F0875F8F70089547E0489F00
:1046E0009001499F300D11242A5C3D4BBC016C5F49
:1046F0007F4F8617970710F080E0089550E040E064
:10470000FA01E55AFF4FE20FF31FE081E11109C002
:104710004F5F5F4F4730510599F70196295F3F4F33
:10472000E8CF81E0089582EC8093354281E0809368
:10473000A6418093D3698091284290E08093377D91
:104740009093387D089527E731E0829FD001839FC1
:10475000B00D1124A15FB549629FF001639FF00D78
:104760001124E15FF5498EEE92E001900D920197E0
:10477000E1F7089597E0899FB001112430E020E02F
:10478000A901460F571FFA01EA52F6494F565D4BF1
:10479000DA019C9190832F5F3F4F2730310581F7DD
:1047A000089527E0829FC001112430E020E0A90194
:1047B000480F591FFA01EA52F6494F565D4B608186
:1047C000FA014081641307C02F5F3F4F2730310546
:1047D00071F781E0089580E00895CF93DF93DC01C5
:1047E000362F4423C1F06A30B0F4E0E0222311F008
:1047F0002C93E1E0ED01CE0FD11D832F6AE00E94E2
:104800007C3E905D9883EF5FEA0FFB2FF11D1082D5
:10481000DF91CF910895832F6AE00E947C3E805DF6
:104820008C93E7CF1F93CF93DF93CDB7DEB7259758
:10483000CDBFDEBF182F6091254220E041E0CE01C0
:1048400001960E94ED2380912E4224E08202C00155
:1048500011242FEF40E0612FC7960E94B1172FEF70
:1048600040E0682F8DE20E941617682F8091F64273
:1048700080FF20C02FEF40E0CE0101960E94771705
:104880002FEF40E0682F8DE20E941617E09124423E
:1048900094E0E902F00111242FEF40E0682FCF01EE
:1048A00007960E94B1172596CDBFDEBFDF91CF914D
:1048B0001F9108958091244224E08202C0011124B6
:1048C0002FEF40E007960E94B1172FEF40E0682FCE
:1048D0008DE20E9416172FEF40E0682FCE0101965F
:1048E0000E947717E0CF1F93CF93DF93CDB7DEB74A
:1048F0002597CDBFDEBF182F80911F42813009F070
:1049000040C060912D4220E241E0CE0101960E941C
:10491000ED232FEF40E0612FCE0101960E94771723
:104920002FEF40E0682F8AE30E941617182F60913E
:10493000214220E040E0CE0101960E94ED232FEFBE
:1049400040E0612FCE0101960E947717682F809179
:104950001F42813079F4809120422FEF40E08C306B
:10496000ACF080E50E9416172FEF40E0682F8DE431
:104970000E9416172596CDBFDEBFDF91CF911F9104
:1049800008956091204220E240E0BFCF81E4EACF69
:10499000CF93DF93EC01FB016AE070E00E94963E4A
:1049A0009B01805D82836A30710590F0CE0164E6E0
:1049B00070E00E94963E605D6083C9016AE070E02D
:1049C0000E94963E805D81831382DF91CF9108958E
:1049D0004083672B91F74183F7CFCF93DF93EC01AF
:1049E000FB016AE070E00E94963E9B01805D83833C
:1049F0006A30710570F0CE0164E670E00E94963E68
:104A0000605D6083C9016AE070E00E94963E805D4F
:104A100004C080E38083672BA9F782838EE28183C1
:104A200086E584831582DF91CF91089581E080939C
:104A3000000624E090E080E031E030930A064091E7
:104A40000D0640FFFCCF4091100650911106840FD7
:104A5000951F215091F796958795969587956AE0D1
:104A600070E00E94963E059710F06F5F7F4F1092A6
:104A70000006CB010895E62FE69527E0829FC0014E
:104A800011248A5C9D4BE80FF92FF11DE55AFF4F69
:104A9000808160FD82958F70089527E0289FD00166
:104AA000299FB00D112430E020E0F901EA0FFB1F2F
:104AB000EF56FD4B9081492F4F70FB01408392953B
:104AC0009F7091832F5F3F4F6E5F7F4F273031057F
:104AD00061F708958F929F92BF92CF92DF92EF92EB
:104AE000FF920F931F93CF93DF93CDB7DEB76897F5
:104AF000CDBFDEBFD42E8E010F5F1F4FAE01435FCF
:104B00005F4F780120E2D7012D937D011B961C9207
:104B10001B974A175B07B9F7382F4C0120E072E06A
:104B2000CC24C39483E0B82E882D831B8617D8F439
:104B3000D401ED914D01822F90E0E7FD54C0E036A5
:104B400018F4E03488F1E054800F911FDC01EC93FD
:104B5000F4018081982F9D7F9C3219F08A3309F0EF
:104B600040C02C3008F385E020E04D2D682FD8019F
:104B70008D918D010E9450194D2D682FF80183856C
:104B80000E9498190E151F0579F76896CDBFDEBFF4
:104B9000DF91CF911F910F91FF90EF90DF90CF9019
:104BA000BF909F908F900895E03238F0EA3349F437
:104BB000840F951FDC017C9314C0F0E0E95CFC4F8E
:104BC000E491EE3251F0EA3B99F3EC3209F0BCCFBC
:104BD000840F951FFC01B08204C0840F951FFC0157
:104BE000C0822F5FBECFEAE3AFCF4F925F926F924A
:104BF0007F928F929F92AF92BF92CF92DF92EF926D
:104C0000FF920F931F93CF93DF93CDB7DEB7A69795
:104C1000CDBFDEBF8C014B018430910510F40E94A2
:104C2000BA23BE016F5F7F4F7B013E017DE0670EBF
:104C3000711C570180E2D5018D935D011B961C927A
:104C40001B97A615B705B9F787E0809F9001819F54
:104C5000300D1124F901E956FD4B8081803109F0B6
:104C600089C085E090E0682FF901E80FF91FEF5641
:104C7000FD4B4081411103C00197A8F76FEF6F5FB3
:104C800090E0462F50E087E0809FD001819FB00DDB
:104C90001124AA5CBD4B292F092E000C330B2417BD
:104CA0003507FCF00430110508F045C0402F440FD3
:104CB0004F5FCE0149960E946A25A696CDBFDEBF02
:104CC000DF91CF911F910F91FF90EF90DF90CF90E8
:104CD000BF90AF909F908F907F906F905F904F901C
:104CE0000895FA01E21BF30BEA0FFB1FE65AFF4F90
:104CF000808187FD1EC0803280F48823C1F07EEF62
:104D0000780F7230B0F079EF780F753090F072EF65
:104D1000780F7F3070F08E3160F4E9E1F0E0EC0F55
:104D2000FD1F2E0F3F1FF90180839F5FB4CF8AE0E4
:104D3000F4CF82E0F2CF8BE0D4018C9380E2119625
:104D40008C9320E0822F022E000C990BFC013296EE
:104D5000E80DF91D8417950714F01082AECF69E1B4
:104D600070E06C0F7D1F860F971FDC018C91808394
:104D70002F5FE8CF6E01B9E1CB0ED11CB601C8019F
:104D80000E944D255090F64241E0A3E04A2E53FC8C
:104D900003C043E0442443949091F44292959C7064
:104DA000A091F542AF705A2F898D2A8DF82FEAE035
:104DB0002E9FF00D11242F2F3B8D3323F9F034E675
:104DC0003F1B232F31E09830D9F4E22F022E000C44
:104DD000FF0B6A2F70E06F5F7F4F6E177F070CF439
:104DE0005AC031E0E617F70721F49DA131E0953074
:104DF00018F098E02A3024F090E002C09830C9F30F
:104E00006EA1662311F06DE26983943009F4D4C079
:104E1000983009F442C0911121C1332311F08DE281
:104E20008A87822F6AE00E94883E90E3980F9B87D2
:104E300090E3920FF6EF8F9F900D11249C874E8781
:104E4000A83008F0B6C0F601EA1BF109A1E083859D
:104E5000853008F4A0E0B1E0B50F6DE070E08B2F75
:104E60000B2E000C990BFB01E81BF90BEC0DFD1D43
:104E7000E081EA0FA0E0EA3010F0E0E0A1E08E0D62
:104E80009F1DF0E37F2E7E0EFC017082B15039F73A
:104E90002111EAC039C031E0AFCF313009F04EC046
:104EA000AF5F8A2F821BF601E81BF10987FDF3959E
:104EB00051E08485853008F450E01EA2022E000CDB
:104EC000330B8DE090E06701C20ED31E6A2F0A2ECD
:104ED000000C770BFB01E21BF30BF7FD0BC0FC0191
:104EE000E61BF70BEC0DFD1DE08DE50F50E0EA3001
:104EF00010F051E0E0E06E0D7F1DB0E3BE0FFB014E
:104F0000B083A15019F74E870430110508F0DCC0BA
:104F1000000F0F5F85E020E0402F682FF70181919F
:104F20007F010E945019402F682FD7011B968C914A
:104F30000E949819AE14BF0471F7BFCE8F5F8A0F1D
:104F40008A3034F551E0F601E81BF10987FDF3954D
:104F50009485953008F450E0082E000C990BF6016A
:104F6000E81BF90B3D961816B4F0E1E0E20FE60DF0
:104F7000F72DF11D4083225052FEC6CF121624F6A3
:104F8000F301E20FF11D27FDFA9540822350F6CF81
:104F9000532F8AE0E1CF6191650F532F6A3010F0F3
:104FA000632F51E0D701A80FB91F605D6C93019783
:104FB000DACFA0E057E04FCFA83008F046C0F601A6
:104FC000EA1BF109A1E08385853008F4A0E0B1E097
:104FD000B50F6DE070E08B2F0B2E000C990BFB01D1
:104FE000E81BF90BEC0DFD1DE081EA0FA0E0EA30B3
:104FF00010F0A1E0E0E08E0D9F1DF0E35F2E5E0E4D
:10500000FC015082B15039F7332309F1121614F420
:105010008DE28A872E5FE3E0822F6E2F0E94883E0A
:10502000E91B291BE60DF72DF11D4083822F6AE055
:105030000E94883E90E3980F9B8790E3920FF6EFD3
:105040008F9F900D11249C8723CF57E0BFCF822FD5
:1050500063E00E94883EE1E0E90FE3CF222309F4F8
:1050600053CF983009F450CF8A81803309F04CCF68
:105070002336A9F461E0252F550F330B2F5F3F4FE7
:1050800059E305C08E0D9F1DDC015C936F5F862F79
:10509000062E000C990B28173907A4F735CF81E3AA
:1050A0008A83332379F02150822F6AE00E94883E60
:1050B00090E3980F9B87205DB6EF8B9F200D112406
:1050C0002C8722CF2F5FF0CF80E09CE22EE2F70109
:1050D00031917F01F401E80FF11D3083E1E0E80F29
:1050E000D7011B963C91341310C0E80DF92DF11D2A
:1050F000413049F420838E5FAE14BF0441F7880E1F
:10510000911CF4012ACE9083F6CF8E2FF5CFF89420
:10511000E9EAF1E411861086128613861486158654
:10512000789408958F708A3010F0895A0895805DC0
:105130000895CF93C82F82958F700E9492280E9465
:105140002A148C2F8F700E949228CF910C942A14CD
:105150001F93CF93DF9327E0289FE001299FD00D75
:105160001124C856DD4B16E08A9182958F700E94FB
:1051700092280E942A1488818F700E9492280E948F
:105180002A14115088F7DF91CF911F9108950F9342
:105190001F93CF93DF938C01EC012E968A918F7031
:1051A0000E9492280E942A140C171D07B9F7DF915C
:1051B000CF911F910F9108950F931F93CF93DF937A
:1051C0008C01EC0125968A918F700E9492280E9492
:1051D0002A140C171D07B9F7DF91CF911F910F917A
:1051E0000895CF93C82F892F0E949228803311F001
:1051F0000E942A148C2F82958F700E9492280E9400
:105200002A148C2F0E949228CF910C942A141F9359
:10521000CF93DF93D82F162FC42F82958F700E94C3
:10522000922820E04C2F612F0E941617182F8D2FE7
:105230000E94922820E04C2F612FDF91CF911F9187
:105240000C9416171F93CF93DF9320E046E060E69F
:1052500089E491E00E94B117CFE1D1E116E0988195
:10526000412F682F892F0E940729C03191E1D9076A
:1052700021F4DF91CF911F910895C83111F41F5F80
:1052800088E72197ECCF9091B3419830BCF4E0913E
:10529000B141F0E0E755FE4B80838091B1418F5FD3
:1052A0008093B1418091B14187708093B1418091E9
:1052B000B3418F5F8093B34181E0089580E008950A
:1052C000E091B141E81BFF0B3197E770FF27E755ED
:1052D000FE4B80810895F8948091B3411816BCF478
:1052E000E091B241F0E0E755FE4B80819091B241F0
:1052F0009F5F9093B2419091B24197709093B24169
:105300009091B34191509093B341789408958FEF69
:10531000FCCF1F920F920FB60F9211240BB60F9273
:105320002F933F934F935F936F937F938F939F93AD
:10533000AF93BF93CF93DF93EF93FF938091D469A3
:105340008F5F8093D4698091D46983708093D4698E
:105350008091B7419091B84186FF28C088EC91E4D4
:105360000E944D1E882349F08091B7419091B84129
:1053700082608093B7419093B8418091B7419091FA
:10538000B84190FF13C068EC71E484EE91E40E9490
:10539000801B882359F08091B7419091B84181607A
:1053A0008093B7419093B841109215408091B741D6
:1053B0009091B84187FF28C086ED91E40E944D1E70
:1053C000882349F08091B7419091B84188608093DB
:1053D000B7419093B8418091B7419091B84191FF06
:1053E00013C066ED71E482EF91E40E94801B882374
:1053F00059F08091B7419091B84184608093B74152
:105400009093B841109215408091B7419091B84166
:1054100092FF19C08DEB91E40E944D1E62EC71E485
:105420008DEB91E40E94961B882369F08DEB91E44B
:105430000E948F1B8091B7419091B8418061809309
:10544000B7419093B8418091B7418F73D9F0809163
:10545000CE699091CF6990628093CE699093CF6925
:105460008091CE699091CF6990618093CE6990933D
:10547000CF6981E08093EA7D80911540813011F4FD
:10548000109215408091D469811168C080911540B7
:10549000823049F08091397D882329F08091397DCF
:1054A00081508093397D809122428F5F8093224288
:1054B000809122428C330CF451C0C1E0C09317405C
:1054C00010922242809121428F5F809321428091ED
:1054D00021428C330CF442C0109221428091204230
:1054E0008F5F809320428091204288318CF110920E
:1054F0002042809125428F5F80932542D0912542A2
:1055000060912342809124420E94331A2D2FDD0F97
:10551000330B8217130694F4C093254280912442E2
:105520008F5F80932442809124428D303CF0C09361
:105530002442809123428F5F8093234240912542F1
:1055400060912442809123420E94101A80932E423F
:10555000809120420E94491A80932D4281E08093DD
:105560005301FF91EF91DF91CF91BF91AF919F9147
:105570008F917F916F915F914F913F912F910F90FC
:105580000BBE0F900FBE0F901F9018951F920F9299
:105590000FB60F9211242F933F934F938F939F93A6
:1055A00081E0809316408091B641813089F58091E9
:1055B000084081508093084080910840811128C0A4
:1055C00080912942809308404EB18091347D909122
:1055D000357D880F991F21E030E04F3F11F430E016
:1055E00020E0822B932B8093347D9093357D8091A6
:1055F000347D9091357D892B59F41092B6411092EB
:1056000002408FEF8FB99DE090936B0480936C0400
:1056100081E080930B0A9F918F914F913F912F9141
:105620000F900FBE0F901F901895CF93DF9300D06F
:1056300000D0CDB7DEB780911740813009F046C069
:105640000E9416258093467D9093477D20912A42A3
:105650004CE251E0BA01EAE02E9F60197109112471
:105660009B013695279536952795BA01621B730BDA
:105670006817790788F582E1898385E18A8386E165
:105680008B831C826FEF80E00E94CB162FEF40E0EF
:1056900062EECE0101960E94771781E00E941224EB
:1056A00080E60E947324E4EEF1E482EF91E421911C
:1056B000211138C08E179F07D1F780E00E945F1636
:1056C00061E080E00E94DA16109217402496CDBF68
:1056D000DEBFDF91CF910895B901660F771FFA0100
:1056E000E61BF70BE817F90720F482E1898384E1D0
:1056F000C5CF620F731FFA01E61BF70BE817F90716
:1057000020F482E1898383E1B9CF220F331F220F76
:10571000331F421B530B4817590710F481E1F2CF96
:1057200080E1F0CF2FEF40E068EC87E00E94161791
:10573000C4CF0895CF92DF92EF92FF920F931F9301
:10574000CF93DF938091154081118CC0D12CC2E0A2
:10575000CC2ED4E7ED2ED4E0FD2E11E08091FB6934
:105760008230F1F580912C4090912D4080938142C0
:1057700090938242D09214400E94F10FFC018081EC
:105780008093134080918142909182422091024007
:1057900021110AC08C3FF1E19F0739F5E0920340E7
:1057A000F0920440109302400E9460229C013695C2
:1057B000279536952795D22E7091D56970933442EE
:1057C0001092D5694091FB69423009F4FEC1A0F402
:1057D000442331F1413009F49EC11092FB693EC06F
:1057E00080917F4290918042C1CF883C20E1920716
:1057F000D9F6C0920240D8CF443009F4F6C108F47B
:10580000E7C1453051F720917F42309180422F5FB0
:105810003F4F20937F423093804280FDDECF9ECF6A
:1058200040917F4250918042FA013196E0937F424D
:10583000F0938042682F6370623031F1633009F475
:1058400059C16130C1F0F901FF27EE0FFF1FE1558B
:10585000FF4F45915491822FFA0109958091FB6980
:1058600081117CCFDF91CF911F910F91FF90EF902D
:10587000DF90CF9008956093FB698093F7699093D0
:10588000F86970931F40EACFD22FD695D695D6955A
:10589000C22FC770EFEFEC0FE73078F4F0E0ED5A6D
:1058A000F34D0C94E03EA42C8D2C5A2C922C9B2C66
:1058B0009E2CA12C2DE060E005C00E94F10FFC01A0
:1058C0006081262F2093D269D150DF3108F03EC08D
:1058D000ED2FF0E0E259F34D0C94E03EAC2CB02CEF
:1058E000B42CBC2CC42CC82CCE2CD42CDA2CE22CFE
:1058F000E62CEC2CF62C0B2D102D152D1B2D212D0F
:10590000292D342D322D3B2D432D492D522D572D30
:105910005D2D612D672D6B2D6F2D0E94F10FFC0108
:105920002081C9CF60917C4220917D4226170CF0E6
:10593000C9CF2DE0C7CF22E062E0C4CF2CE063E006
:10594000C1CF2DE06DE0BECF22E0B5CF422F86E380
:1059500092E40E94841082CF422F84E492E4F9CF33
:10596000422F82E592E4F5CF462F64E472E486E3A9
:1059700092E40E948D1072CF462F66E372E484E4B5
:1059800092E40E9473106ACF462F62E572E4EFCF73
:10599000462F64E472E482E592E4F3CF462F62E599
:1059A00072E484E492E4E5CF462F62E572E486E394
:1059B00092E4E7CF462F64E472E486E392E40E9427
:1059C000A0104CCF462F62E572E4F7CF1093D56953
:1059D000462F70E060E0F1CF022F262F44E452E41E
:1059E00066E372E4CB010E94CC1038CF1093D569E6
:1059F000C73061F480918E428A3041F480914342F5
:105A00008B3020F089508093434228CF022F262FDD
:105A100050E040E0E5CF022F262F42E552E4E0CFF0
:105A2000462F62E572E4CB01CACF462F66E372E4EB
:105A300082E592E4C4CF1093D569462F70E060E010
:105A4000F7CF022F262F42E552E466E372E4CA0143
:105A5000CACF1093D569022F262F50E040E062E5AF
:105A600072E4C0CF1093D569022F262F42E552E48D
:105A700070E060E0ECCF462F70E060E084E492E4F8
:105A80000E940E11EBCE462F70E060E082E592E4BA
:105A9000F7CF022F262F42E552E466E372E490E04E
:105AA00080E0A1CF022F262F44E452E4F6CF462F08
:105AB00070E060E086E392E4E3CF462F62E572E4B3
:105AC000F9CF422F86E392E40E94FF10C7CE422F07
:105AD00084E492E4F9CF422F82E592E4F5CFC6E365
:105AE000D2E4C20FD11D261B4A9149832A95E1F7C2
:105AF0001882B4CE822F86958F7327FD8054217033
:105B00002713B0CE480F511D87FD5A9540937F4211
:105B100050938042A3CE40917F42509180424F5F8C
:105B20005F4F40937F42509380421092FB69609197
:105B30001F409C01217033276217130609F092CE93
:105B40002091F7693091F869369527953695279514
:105B5000BC01E6E0660F771FEA95E1F76627262B82
:105B6000372B81FF05C020937F423093804276CE51
:105B700080918742909188428093894290938A4293
:105B8000809185429091864280938742909388428B
:105B90008091834290918442809385429093864283
:105BA000409383425093844220937F4230938042BB
:105BB000C9010E946022892B09F050CE0E942E114B
:105BC00080937F429093804249CE0E94B61346CE86
:105BD00020917F42309180422F5F3F4F20937F4240
:105BE000309380420E94B61339CE882351F08091C1
:105BF0007F4290918042019680937F4290938042B1
:105C0000ECCD10927F42109280428091367D8823A5
:105C100019F010931540E1CD1092EA7D1093D569EB
:105C2000C09215401092397DD8CD0F931F93CF931A
:105C3000DF93182FD62FC1E001E0DC1728F4DF91A5
:105C4000CF911F910F910895111105C08091F442D9
:105C500081608093F4420E94932310921540009338
:105C6000EA7D0E949A2B809115408130D1F7CF5F59
:105C7000E4CF4F925F926F927F928F929F92AF92FA
:105C8000BF92CF92DF92EF92FF920F931F93CF9329
:105C9000DF93CDB7DEB72E97CDBFDEBF0091FB42BD
:105CA00010E0102F002700271F708091FA42082B68
:105CB000480100931B4010931C4043EF642E42E4C4
:105CC000742ECE0101965C0107966501F3012191C6
:105CD000D6012D936D01A817B907C9F7E0901940B7
:105CE000F0901A40E016F10668F5F801EE19FF0988
:105CF0007F0180E00E946029823009F05AC0EA9456
:105D0000EF2809F056C0043011050CF452C081E0B0
:105D10000E94602963E08232C1F485E00E94A323DF
:105D200061E083E00E94A32363E080E00E94152EDF
:105D30000E94FF1A81E00E94321B63E081E00E9412
:105D4000152E0EC0E01AF10AD4CF81E00E94A323E1
:105D500065E083E00E94A3236BE085E00E94A3231B
:105D600069E081E00E94DA16D5018D915D01F301B1
:105D700081933F01AC15BD05B9F780911B4090910F
:105D80001C408093194090931A402E96CDBFDEBFE1
:105D9000DF91CF911F910F91FF90EF90DF90CF9007
:105DA000BF90AF909F908F907F906F905F904F903B
:105DB00008958091F44281FF14C0809118408111B0
:105DC000CFCF63E081E00E94A32365E083E00E94DF
:105DD000A3236BE085E00E94A32381E08093184019
:105DE000BFCF109218400430110534F5119501957C
:105DF0001109000F111F0A5F1F4FFF24F3948F2D0D
:105E00000F2C000C990B0817190780F45524539494
:105E10004424439483E0E82EF12C052D052C000C3E
:105E2000110B8016910660F4682D88CF60E08F2DED
:105E30000E94CB16F394E3CF93E0892E912CE6CF0A
:105E40008091F44281608093F4420E9493231092E7
:105E500015404092EA7D0E949A2B80911540813036
:105E6000D1F70E94FF1AC701801B910B880F8F5F2B
:105E70000E94321B5394D1CF20912F42022E000C4E
:105E8000330B2F5F3F4FAC01249FC001259F900D26
:105E9000349F900D1124019708F40895EFECF7E07A
:105EA0003197F1F700C00000F6CF1F93CF93DF9337
:105EB00083E090E00E943C2FC0E4D4E018E01E8311
:105EC00083E090E00E943C2F1D8381E090E0DF9111
:105ED000CF911F910C943C2FEF92FF921F93CF9381
:105EE000DF930E94552FCFE9DEE1FE0114911123CB
:105EF000F1F03196849122968F3F29F484E690E068
:105F00000E943C2FF2CF84910E942C167E01F70153
:105F10008FEFE81AF80A8E2D8C1B811720F0115094
:105F2000C10FD11DE2CF84910E942516F0CFDF91E1
:105F3000CF911F91FF90EF90089520912F42022E54
:105F4000000C330B2F5F3F4FAC01249FC001259FF6
:105F5000900D349F900D1124019708F4089552E09C
:105F60005A95F1F700C0F8CF1F920F920FB60F921B
:105F700011240BB60F92BF92CF92DF92EF92FF9255
:105F80000F931F932F933F934F935F936F937F9341
:105F90008F939F93AF93BF93CF93DF93EF93FF9331
:105FA00088E080936B048FEF80936C04DFB18FB92E
:105FB000DD2309F492C0ED2EF12C97012150310917
:105FC0002D233F21232B09F088C09091154092305A
:105FD00049F4109215408FB99DE090936B04809323
:105FE0006C0455C010E000E08FE1B82ECC24C394BF
:105FF000D12CC02FB0920204C601002E01C0880F20
:106000000A94EAF78093010485E090E00E949D2FB6
:106010008EB190E0809590958E219F21892B31F44F
:106020000F5F1F4F0530110521F7C5E080E0D695C1
:1060300009F049C0CC0FCC0FCC0FC80FC83208F004
:1060400044C0D6E910EA80911E42811110930704E2
:106050008EE591E00E949D2FD150A9F78C2F0E94D0
:106060004329882359F081E08093B64124E632E346
:106070002093034030930440809302408FE180934B
:1060800001041092154080911D428093397DFF914B
:10609000EF91DF91CF91BF91AF919F918F917F91C0
:1060A0006F915F914F913F912F911F910F91FF90B1
:1060B000EF90DF90CF90BF900F900BBE0F900FBE70
:1060C0000F901F9018958F5FB2CF8FEF8FB99DE023
:1060D00090936B0480936C04D1CF8FEF7CCFCF92E1
:1060E000DF92EF92FF92CF93DF93A8E4BDE726E023
:1060F00036E1D7964C91D7974F3F61F150E0DC964F
:106100008C91DC9790E0D6966C91D697613099F59A
:10611000DD966C91DD97EC01CC0FDD1FCC0FDD1F00
:10612000349FF001359FF00D1124CE0FDF1FC25DAB
:10613000DF4BD896CD90DD90ED90FC90DB97C88238
:10614000D982EA82FB82E25DFF4B8E0F9F1FEC013A
:10615000288B658B2F5F1996223159F68091D16972
:10616000823020F51092D169DF91CF91FF90EF90AE
:10617000DF90CF900895349FB001359F700D1124AA
:10618000EB01C25DDF4BC80FD91F48894213E2CF34
:10619000FC01EE0FFF1FEE0FFF1FE60FF71FE25D82
:1061A000FF4B1082118212821382D4CF83E080933E
:1061B000D16981E090E0A0E0B0E08093DE40909370
:1061C000DF40A093E040B093E140CECF1F93CF9348
:1061D000DF93CDB7DEB76C97CDBFDEBF11E060E0D7
:1061E000812F0E94CB161F5F1730C9F78091327D37
:1061F00081FD37C0809130428230F1F1833069F007
:10620000813079F520E046E061E089E50E941617CB
:1062100070E060E082E090E022C020E042E061E0D7
:1062200084E50E94161720E044E061E08AE50E94C0
:10623000161720E046E061E089E50E94161770E03D
:1062400060E082E090E00E94F52570E060E081E08F
:1062500090E00E94F52570E060E090E080E00E9410
:10626000F52566E081E00E94DA166C96CDBFDEBFB0
:10627000DF91CF911F91089520E046E061E081E435
:106280000E941617ECECF2E467E18291811102C0E2
:106290006150D8F76F5F89F420E045E065E08DE458
:1062A00091E00E94DE1985E00E949D1620E046E004
:1062B00061E081E40E941617D4CFE62FF0E0EC54A1
:1062C000FD4BCE010196DC0122912D932A2F281B34
:1062D0002617D4F345E00E946A25E8CF7F928F927B
:1062E0009F92AF92BF92CF92DF92EF92FF920F9365
:1062F0001F93CF93DF93CDB7DEB76597CDBFDEBFDA
:106300004C017A01CA0140968B01041B150B6817DA
:10631000790710F000E110E040E3BE016F5F7F4FAE
:10632000C7010E94C8248DE28C831D822FEF40E0BC
:106330006EEBCE0101960E94771740E3BE016F5FBE
:106340007F4FC7010197800F911F0E94C8242FEF34
:1063500040E06EEDCE0101960E9477178E0C9F1CD7
:10636000C12C8AE3782EAC2CB12CA016B10688F093
:106370006596CDBFDEBFDF91CF911F910F91FF904A
:10638000EF90DF90CF90BF90AF909F908F907F90D5
:106390000895BE016F5F7F4FC501880D991D0E9452
:1063A000F525DC2CD694D394C0FC21C040E2BE017C
:1063B0006F5E7F4FC5018E0D9F1D0E94C8247C8A91
:1063C0001D8A20E04D2D61E0CE0141960E94771795
:1063D00020E04D2D62E2CE0101960E94771720E069
:1063E0004D2D6AE88CE70E941617C394BCCF20E0BD
:1063F0004D2D62E9CE0101960E947717F6CF8130CC
:10640000A9F028F08230F9F0833031F1089588ED59
:1064100094E184BF909368008AE990E08093260A13
:106420009093270A8AE080930206089588ED9CE104
:1064300084BF9093680085E391E08093260A90934F
:10644000270A8CE0F0CF88ED25E230E084BF20936E
:10645000680080ED91E0F1CF88ED2DE230E084BF5F
:10646000209368008BE692E08093260A9093270A97
:106470008DE0D9CF84EF91E00E943C2F81E380939F
:10648000600980912F420C94FF3183E00E94FF311C
:10649000E0E2F8E087E594E08087918783E08783F6
:1064A0008681806C868380E8858384E690E00C9406
:1064B0003C2FCF93DF93109260090E9445328CE00D
:1064C0000E942A1490E080E00E944223CFE0DAE6A6
:1064D000899182958F700E9492280E942A14FE0151
:1064E000319780818F700E9492280E942A148AE737
:1064F000CC32D80769F78AE00E942A1485E090E040
:106500000E94422384E00E942A14DF91CF910C94D0
:106510003A32EF92FF920F931F93CF93DF93109233
:1065200060090E9445328CE00E942A148AE00E9491
:106530002A1480E290E00E944223D0E0C0E0EE24E2
:10654000EA948EEFF82E2091D1692E9DC0012F9DE7
:10655000900D112480549C4FC817D90708F4AAC085
:1065600081E40E942A148AE30E942A1480E20E9495
:106570002A1486E392E40E94C72880E20E942A142B
:1065800080E20E942A1482E40E942A148AE30E9474
:106590002A1480E20E942A1484E492E40E94C7280C
:1065A00080E20E942A1480E20E942A1483E40E945E
:1065B0002A148AE30E942A1480E20E942A1482E5A7
:1065C00092E40E94C7288AE00E942A1483E50E9470
:1065D0002A148AE30E942A1480E20E942A14CDE041
:1065E000D0E001E010E020918F4230919042C8014C
:1065F0000C2E02C0880F991F0A94E2F7822393237E
:10660000892B09F07AC080E30E942A14219758F759
:106610008AE00E942A148DE40E942A148AE30E94D0
:106620002A1480E20E942A1480E692E40E94C7287D
:1066300080E20E942A1480E20E942A148EE40E94C2
:106640002A148AE30E942A1480E20E942A148EE609
:1066500092E40E94C72880E20E942A1480E20E94ED
:106660002A1487E40E942A148AE30E942A1480E2F2
:106670000E942A1480918C428F700E9492280E945E
:106680002A1480918B428F700E9492280E942A14B3
:106690008AE00E942A1485E090E00E94422384E070
:1066A0000E942A14DF91CF911F910F91FF90EF90DC
:1066B0000C943A32CE010E946E238823E1F0CE0181
:1066C000C031D10508F0C0960E94F12880E20E94F6
:1066D0002A1410E000E0CE01800F911F0E94A8282C
:1066E00080E20E942A140F5F1F4F0430110599F7B2
:1066F0008AE00E942A14249626CF81E385CFCF9387
:10670000DF93109260090E9445328CE00E942A14A7
:106710008AE00E942A1482E50E942A1481E40E94E1
:106720002A148DE40E942A148AE00E942A14C1EDE2
:10673000D5E589910E94992889E6C13DD807C9F716
:106740008AE00E942A1485E090E00E94422384E0BF
:106750000E942A14DF91CF910C943A32CF92DF92AB
:10676000FF920F931F93CF93DF9300D000D0CDB74C
:10677000DEB78091094090910A40A0910B40B09102
:106780000C4089839A83AB83BC83109260090E947A
:10679000453289E090E00E9442230E94E92280E095
:1067A0008111FECF10E080910E6A882361F00E9473
:1067B0000C14E1E0F0E0EC0FFD1FE10FF11D908102
:1067C0001F5F891310E00E946B298F3F79F513300A
:1067D00051F70E940C148A3029F501ED15E591ED71
:1067E000C92E99E6D92E0E94C722F82EF29480EF86
:1067F000F8220E94C7228F29F80181938F01CE16BB
:10680000DF0689F78DE190E00E9442232496CDBFF8
:10681000DEBFDF91CF911F910F91FF90DF90CF905E
:106820000C943A320E946B298F3F99F289E290E0F2
:106830000E944223E7CF8F929F92AF92BF92CF9256
:10684000DF92EF92FF92CF93DF93C2E0812C912CE5
:10685000540180E090E8A0E0BB278A539748AF4FEF
:10686000BF4F6C017D01C80CD91CEA1CFB1CDFE189
:1068700061E0EBBEF6018791882369F020E04C2FA0
:106880000E941617682FD1508FEFC81AD80AE80A4D
:10689000F80AD111EECF80E2880E911CA11CB11C28
:1068A000CF5FC630B1F6DF91CF91FF90EF90DF90D0
:1068B000CF90BF90AF909F908F900895CF9388E72F
:1068C00090E00E943C2FC0E08091B641813019F0E9
:1068D0008C2FCF91089582E390E00E943C2F729913
:1068E000F3CF8FEF0E9491166BE080E00E94DA16E2
:1068F0000E9459328FEF0E9491166BE080E00E9457
:10690000DA16C1E0E1CF2F923F924F925F926F92E1
:106910007F928F929F92AF92BF92CF92DF92EF922F
:10692000FF920F931F93CF93DF93CDB7DEB76C9792
:10693000CDBFDEBF8091EE4220E1829FC0011124D5
:106940002091ED4222952F70822B20E032E0A901A8
:10695000481B590B4F8B588FDC01D097AB8FBC8FE6
:10696000D12CC12C10E0E12CF12CE4EB2E2EEDE724
:106970003E2E2FEF31E0F901E81BF90BE98FFA8F7A
:106980000E9486166FEF80E00E94CB166FEF89E0C1
:106990000E94CB166FEF8AE00E94CB16F6E0FF9EB6
:1069A000C00111242FEF40E061E0895A9F4F0E94FF
:1069B000B11721E12F15F8F0EF2DF0E0EE51FB4C6F
:1069C0000C94E03EF434383549351036163620360E
:1069D000F93564352C35A9356A3596364D36373755
:1069E000323555351C372D3709E026E042E065E0A9
:1069F00080E00E94E2176BE080E00E94DA1680914E
:106A00005000897F846080935000809150008160A5
:106A1000809350008895809150008E7F8093500025
:106A20008091397D8111FEC2109215406C96CDBFC8
:106A3000DEBFDF91CF911F910F91FF90EF90DF901C
:106A4000CF90BF90AF909F908F907F906F905F900E
:106A50004F903F902F90089508E023E344E06EE1CB
:106A60008BE2C7CF08E02CE243E067E081E0C1CFD2
:106A700008E026E147E168E189E10E94E2178091A0
:106A800030420E947D1887E00E94321B0E94E6304F
:106A9000B2CF08E026E246E26CE08DE00E94E21709
:106AA00080911E420E947D18A6CF08E027E346E3AE
:106AB0006DE28EE20E94E21780912B420E947D18C7
:106AC00080912C428E5FEECF08E026E246E26BE139
:106AD0008AE18FCF08E026E246E266E286E20E9483
:106AE000E21779EF872E72E4972E512C01E0652C86
:106AF00054E0752E67E0A62EB12C20E241E0662D11
:106B0000CE0101960E94ED23D4018C9190E00A2CD5
:106B100002C0959587950A94E2F720E080FF26E66B
:106B2000402F672DCE0101960E9477176394B1E044
:106B3000AB1AB108E0E27E0EFFEFAF16BF06E9F632
:106B40000F5F28E0520E31E0831A9108083079F681
:106B500052CF4F89588D452B09F446C081E050E152
:106B6000C516D1040CF480E09601215F3F4FA98D3A
:106B7000BA8D2A173B0708F4826008E026E246E255
:106B8000823069F1833071F166E2813049F58DE13F
:106B90000E94E2172FEF40E06CE583EC90E00E944A
:106BA000B11740E2BE016F5F7F4F8F89988D0E94C1
:106BB000C8242FEF40E064E8CE0101960E947717C9
:106BC000EF89F88D309731F0A601BF018B8D9C8D38
:106BD0000E946E3168E081E00E94DA160CCF6CE111
:106BE00086E2D6CF6CE1D3CF08E026E246E266E249
:106BF000F7CF08E025E144E163E182E10E94E2177A
:106C000080911D42883751F0803F21F08C3321F470
:106C100080E048CF82E046CF83E044CF81E042CF9E
:106C200008E026E246E26BE08AE0E3CE08E021E1FC
:106C300040E16FE08EE00E94E21780912F4232CF58
:106C40002FEF40E061E68DE291E00E94B1170E94D3
:106C50001B340E9422290E941625BE016F5F7F4FC0
:106C60000E94ED242FEF40E062EDCE0101960E94DC
:106C7000771720E046E061E090E080E00E94B117E5
:106C800020E048E061E085EF9EE10E94941708E073
:106C900026E246E266E281E2ACCE20E042E0410F2D
:106CA00061E088E00E94161702E04CEEA42EB12CA1
:106CB00020E0402F69E0C5010E94B117FDE0AF0E52
:106CC000B11C0F5F0730A1F729E0A22EB12C00E024
:106CD0003AE0932E0430F1F480912A42BE016F5FB6
:106CE0007F4F899DC00111240E94ED2442E0400F96
:106CF00020E06CE6CE0101960E9477170F5F2FEF20
:106D0000A21AB20A053031F708E025E244E263E254
:106D100082E26FCEF501E35EFD4B808140E3BE0170
:106D20006F5F7F4F90E00E94C824E0CF08E026E22A
:106D300040E368E280E2E1108FE10E94E2174E2C0E
:106D4000440C440C440C30EBE39EC0011124AC0114
:106D5000425D5F4B3A01B12CA12C552453945A0C3F
:106D6000842D8A0D0E94922820E0452D62E00E9429
:106D700016170CE0912C812C20E0452D602F8CE71C
:106D80000E9416178091D1698330A1F4C501880D46
:106D9000991D892B79F451E0E5120CC08CE3889E93
:106DA000602D1124685E20E0452D89EC90E00E9462
:106DB000B11728C0F401EE0FFF1FEE0FFF1FE60D05
:106DC000F71D80819181A281B381892B8A2B8B2B26
:106DD00061F1F301E80DF91D808999E0989FF001B8
:106DE0001124E85BF248908126E6911120E0A7E0AB
:106DF0008A9FC0011124452D6AE0600F885B97408F
:106E00000E949417BFEF8B1A9B0A045C0C3F09F099
:106E1000B3CFEFEFAE1ABE0AF6E16F0E711C28E099
:106E2000A216B10409F099CFE6CD26E6452D6CE017
:106E3000600F80ED90E0BBCF8091D16908E02BE03E
:106E40004AE081FD02C026E246E262E381E30E945D
:106E5000E2178091D169869525CE08E026E246E2C8
:106E600065E384E30E94E217809131421BCE88E4FF
:106E7000A82E8DE7B82EF50126E286A981112FE212
:106E800039962E163F06C9F7812F012E000C990B5B
:106E9000069639E0389FF001399FF00D1124E85B28
:106EA000F248818146E28F3F21F080814BE08111E1
:106EB0004AE208E063E282E20E94E21720E041E059
:106EC00068E085E391E00E94B11720E041E06AE8C4
:106ED00085E391E00E94B1170FE181E020E042E0FC
:106EE000682F8BE10E9416170150C1F720E042E0A5
:106EF00068E78EE00E94161720E041E068E78CE723
:106F00000E941617812F66E00E94883EB3E04B2E48
:106F1000490E87958827879555245394580E02E784
:106F2000802E08EF902E712CD501D6968C9100E022
:106F3000813009F006E6B5E0B71580F1A3E06A2ECE
:106F4000670C202F462D6AE0C4010E949417F501BA
:106F500087A9202F462D61E48F3FB9F10E94922826
:106F6000202F462D62E40E9416178E8BD501DC96E9
:106F70008C918F5F0E9492286E89615F202F462D31
:106F80000E9416178E8BF50186AD0E9492286E899D
:106F9000605F202F462D0E9416171BC0FDEF6F2E3D
:106FA000670C20E0462D68E78CE70E941617202F1B
:106FB000462D6AE8C4010E949417D501D7968C919A
:106FC0008F3FC1F4202F462D63EC87ED90E00E94A7
:106FD000B11720E0442D652D88E00E9416177394A8
:106FE000B9E0AB0EB11CE7E08E0E911CFCE07F1205
:106FF0009BCF01CD0E949228202F462D64EC0E9449
:1070000016178E8BF50184AD8F5F0E9492286E89D2
:10701000625F202F462D0E9416178E8BD501DE96BB
:107020008C91B3CF8091B741857029F48091B6419E
:10703000882309F4E4CC0E946B29082F0E945E3457
:10704000813009F40FEF0E94872821E12F1508F104
:10705000EF2DF0E0E25DF74C0C94E03E40386B38E9
:10706000873800393B3A583AD938B1380D3ABD38EB
:10707000C1389B3A613A0E3B243A9638C73AFF3AF8
:10708000003109F4B0C300F5002339F0083009F4E9
:1070900058C2033011F0073081F50E9486166BE06C
:1070A00080E00E94DA1681E0809317400E94152B41
:1070B0000E94FF1A87E00E94321B62E087E00E9474
:1070C000DA160E94E630B2CC083109F489C30032E6
:1070D00001F701E09BC00031C1F048F4002309F43E
:1070E00095C083E00830A9F68093304206C008318D
:1070F00051F0003271F6109230428091B7418570A4
:1071000009F43ECCCACF81E0EFCF82E0EDCF083169
:1071100049F0003221F00111BCCF0EE077C010928F
:107120001E42EBCF81E080931E42E7CF0031B1F0E9
:1071300048F4002391F3083009F0ABCF81E080934D
:107140002C42DBCF083131F0003209F0A2CF10928F
:107150002B42D3CF81E080932B42CFCF10922C4291
:10716000CCCF083139F0003209F446C3011191CF78
:10717000F12CC3CFEAE0FE2EC0CF083171F000320F
:1071800021F0011186CF07E041C030E1C31AD108D8
:10719000D7FEB3CFD12CC12CB0CFC6010F96498DED
:1071A0005A8D8417950708F0A8CF50E1C50ED11C61
:1071B000A4CF0031C9F048F40023F9F00830B1F051
:1071C00080911D428093397D64CF083159F08CE362
:1071D0000032B1F780931D428091F442877F809303
:1071E000F442EECF88E7F6CF80EFF4CF8FEF8093B5
:1071F0001D428091F4428860F2CF7EE0F72EE0CF0E
:10720000083149F0003221F0011143CFF02E75CF43
:107210000E94893272CF20E044E062E08FED90E07E
:107220000E94B11761E084E00E94DA1685E0EDE08B
:10723000F0E4DE01519601900D928A95E1F71092EB
:1072400060090E9445320E9443148AE00E942A1479
:1072500089E090E00E9442230E94E92257E0552EE7
:107260006E0191E1C90ED11C60E3E62E10E0809121
:107270000E6A882361F00E940C14F601E10FF11DE3
:107280009081891719F0123008F073C01F5F0E94B7
:107290006B298F3F11F4143051F70E940C148A307F
:1072A00009F069C0BB24B394E98AEA8AEB8A00E05A
:1072B00010E080910E6A882369F00E940C14082F58
:1072C00080ED800F8A3008F076C0F601E10FF11DE5
:1072D00000831F5F0E946B298F3F31F4003249F712
:1072E000A3E0BA1609F494C0012F10E04601800E05
:1072F000911EB12CA12C84018C149D0409F070C046
:10730000F0E1AF16B10418F020E3A21AB1085A9CBC
:1073100080015B9C100D11240A5C1D4B94E0992E9A
:1073200085E0A82EB12C0E94C722882E829420EFDF
:1073300082220E94C722F501E45AFF4FE00FF11F9D
:107340008829808331E0A31AB1084EEFA4164FEFCD
:10735000B40649F79A94095F1F4F9110E1CF0E943C
:107360000C148A3009F49ECF0E946B298F3FB9F329
:1073700099CF10E08CCF0E946B298F3F09F48DCFFD
:1073800089E290E00E9442230E9443140E94BF0FB2
:107390008DE190E00E9442230E943A320E948616BC
:1073A0006BE080E00E94DA1681E08093174083E072
:1073B0000E9443293BCB8FE9800F863008F485CFAC
:1073C0008FEB800F863038F4F601E10FF11D80E27B
:1073D000800F80837ECF0A3309F07CCFBF2C7ACF19
:1073E000F40182913F010E94E32290E09801281964
:1073F0003909220F331F220F331F02C0880F991F34
:107400002A95E2F7A82AB92A430176CF0E940C14E4
:1074100080910E6A8111FACFB9CF003109F4E6C12B
:1074200048F4002309F4A4CE083009F032CEB1E1CB
:10743000FB2E63CE083121F0003209F46ECE29CE46
:10744000E12C0BE0F02E59CE003109F4D2C148F402
:10745000002309F476C0083009F01BCEFFE0FF2EB0
:107460004CCE083129F0003209F013CE02E0CECE26
:10747000A6E0FA2E42CE0031B1F050F40023A9F07C
:1074800083E0083069F080912F420E94FF3101CEE5
:10749000083129F00032B9F710922F42F4CF81E081
:1074A00080932F42F0CF82E0FBCFEEE0FE2EEBCFB9
:1074B000002309F446C0003209F0EBCD10E00CE0E7
:1074C000A5CE003141F1B8F4002309F499C1083088
:1074D00009F0DFCDE12F012E000CFF0BEA5DFD4B23
:1074E00080818150808380912A428F3108F405CEBB
:1074F0008EE1808302CE083141F0003209F0C9CD1F
:10750000115017FFFACD14E0F8CD1F5F15300CF4C1
:10751000F4CD10E0F2CDE12F012E000CFF0BEA5D5F
:10752000FD4B80818F5F808380912A428F3108F4E8
:10753000E4CD1082E2CD003109F468CE28F40111C7
:10754000A8CD98E0F92ED9CD083131F0003209F0FC
:10755000A0CD81E0E826D1CD2091D169227010E044
:1075600039E0222379F0812F012E000C990B069629
:10757000389FF001399FF00D1124E85BF2488181BA
:10758000883019F08DE0F82EB8CD1F5FEACF0031BA
:1075900089F148F4002309F437C1083009F079CDA6
:1075A0000E94AE33AACD083139F0003209F071CD16
:1075B00081E08093D169A1CD82E08093D169E8E434
:1075C000FDE787A9883081F486ADA8E4BDE7DE96A3
:1075D0009C91DE97981303C0D6961C92D697199665
:1075E0005DE7A43BB50799F739968DE7E43BF807CB
:1075F00041F783CD0E947F3370E1F72E7ECD0831B5
:1076000049F0003221F0011144CD08E0FFCD109285
:10761000314273CD81E0809331426FCD003109F466
:107620007FC070F4002309F4EDC0E8E4FDE7083002
:1076300009F02FCD16AA39962E163F06D9F75DCD43
:10764000083109F440C0003209F023CD115017FD74
:107650001BE0812F012E000C990B019710F48BE099
:1076600090E02091D169227039E0412F012E000C69
:10767000550B4A5F5F4F349FF001359FF00D112489
:10768000E85BF248BC016A5F7F4F369FA001379FDD
:10769000500D1124485B52486085DA0118964C91D0
:1076A000641739F0222309F428CD4181483009F0CC
:1076B00024CD019797FF02C08BE090E0115017FF97
:1076C000D4CF1BE0D2CF812F012E000C990B069650
:1076D00029E0289FF001299FF00D1124E85BF24872
:1076E00040858091D169827059E01F5F1C300CF099
:1076F00010E0212F012E000C330B2A5F3F4F529FC9
:10770000F001539FF00D1124E85BF2489085941727
:1077100061F3882309F4F1CC9181983031F3EDCCF9
:10772000812F012E000C990B069629E0289FF0016D
:10773000299FF00D1124E85BF2484085208121113A
:107740003CC068E4A62E6DE7B62EF50186AD841325
:1077500020C088E49DE7DC01DE965C91DE9754173B
:10776000A1F037A9D7962C9132130FC028E43DE73A
:10777000D901DE966C91DE97561302C0D6961C9204
:10778000275F3F4F2216330699F7099628163906C8
:1077900011F739962E163F06C9F681E0D501DE961F
:1077A0009C91DE97941302C0D6968C93B9E0AB0EF1
:1077B000B11CEA15FB0591F7A0CCE8E4FDE726AD86
:1077C000241301C016AA39962E163F06C1F729E0E8
:1077D000289FF001299FF00D1124E85BF248A9CE03
:1077E00057E0F52E8ACC43E0F42E87CC35E0F32E1B
:1077F00084CC24E0F22E81CCD12CC12C09E006CD22
:1078000005E004CDE12C10E00BE000CDCF93DF9339
:1078100081E080932F4280912F420E94FF3180911E
:107820007C008E7F98ED94BF80937C0080916300F4
:1078300083FDFCCF80917C0098ED8B7F94BF80937B
:107840007C0080917C00816094BF80937C0080915B
:1078500041018111FCCF82E080934701C1E0C093D8
:10786000520181E680935001C0930A0A1092010AE6
:107870008091090A8E7F8093090A86E08093000A2E
:107880008091000A81608093000ADFEFD0930104A9
:1078900080E8809304040E941416D09362048DE063
:1078A00080936B04D0936C04DFB91092A000D5E0F4
:1078B000D093A40080E48093850689E48093080631
:1078C000109200060E94872887E3809322428BE370
:1078D00080932142109220428CE080932D42D093DD
:1078E000254283E08093244285E1809323424091A6
:1078F000254260912442809123420E94101A809375
:107900002E42C0931740C0933042109231421092E1
:10791000D469C0931F4210921E4288E780931D4293
:1079200084E6809326428CE1809327428CE3809307
:107930002842D093294288E180932A42C0932B4267
:107940000E9416258093467D9093477D80911D422D
:107950008093397D7894DF91CF9108950E94063C01
:1079600084E690E00E943C2F0E946C2F0E948616B5
:1079700061E08AE00E94DA160E94152B0E94E63030
:107980000E945C210E9487280E9443140E94BF0F1E
:107990000E949D2182E0F82EEE24E394D1E018E0CD
:1079A000CFEF9EEFD92E0DE020E8C22E809115403A
:1079B000813009F421C108F48AC08230B9F71092ED
:1079C000EA7D1092397DEEE2F0E4148A769681E445
:1079D000EE38F807D1F710936B04C0936C04CFB95D
:1079E00080912B42813071F40E94B8186BE080E0E6
:1079F0000E94DA1690912C42990F990F80E09C5FBB
:107A00000E943C2F0E9486166BE080E00E94DA16EE
:107A10000E940A1A0E948728E0920004D09204046F
:107A20008AE090E00E949D2F10936B04C0936C0439
:107A300000937704CFB980915000897F8460809350
:107A40005000809150008160809350008895809113
:107A500050008E7F8093500080911540823059F302
:107A6000C09300040E940D1AC09204040E946F305B
:107A700082E390E00E943C2F739906C00E94431459
:107A80000E94BF0F0E949D218091B641813009F470
:107A9000AEC0D093EA7D10927F4210928042109245
:107AA000FB69D093D5691092D369D093367D0E943B
:107AB000FF1A0E946C1A0E94E630D09317400E9471
:107AC000152BCFB900936B04C0936C046FCF8091DA
:107AD000264290E080931D4090931E408091164076
:107AE000813021F08091024081114AC08091D36998
:107AF000811116C00E946B298F3F91F0E82FF0E0B2
:107B0000E150FD4FE491E0933542D093A641D093EC
:107B1000D3698091284290E08093377D9093387D9F
:107B20000E949A2B80910240813061F48091034041
:107B300090910440009709F457C001978093034047
:107B40009093044080910540813079F480912742E0
:107B500020911D4030911E40820F932F911D8093E4
:107B60001D4090931E401092054080911D409091C1
:107B70001E40019780931D4090931E401092164026
:107B800080911D4090911E40892B09F0A7CF8091D4
:107B900006408823B9F02091327D3091337D809169
:107BA0000040909101402817390751F00E946C1A4B
:107BB0008091327D9091337D80930040909301407D
:107BC0001092064080910740882359F00E94FF1AC6
:107BD00087E00E94321B62E087E00E94DA16109272
:107BE00007400E94152BE2CE10920240ABCF82E3F9
:107BF00090E00E943C2F48CF10920240EEE2F0E469
:107C0000148A769681E4EE38F807D1F78091327DB8
:107C100081FD48C00E94E6300E94FF1A87E00E9462
:107C2000321B62E087E00E94DA1667E08BE00E9478
:107C3000A32380915000897F8460809350008091BD
:107C400050008160809350008895809150008E7F15
:107C5000809350000E94152B8091397D811105C0C1
:107C60008091F44283FFF09215408091B6418130BB
:107C7000A1F410921540E091B241F0E0E755FE4BBF
:107C80008081833041F40E946B290E945E3481110F
:107C900002C00E9483340E946C1A8091154081308A
:107CA00041F284CE80913142882309F4B3CF81E040
:107CB0000E9460298332B9F482E00E9460298232F6
:107CC00091F480E00E9460298D3109F4A3CF80E017
:107CD0000E946029853109F49DCF80E00E946029CF
:107CE0008D3009F497CF80E00E946029823209F438
:107CF0009CCF0E94392E99CF991B79E004C0991F1F
:107D0000961708F0961B881F7A95C9F780950895F5
:107D100087FB082E062687FD819567FD61950E94E9
:107D20007C3E0EF4919507FC81950895AA1BBB1B20
:107D300051E107C0AA1FBB1FA617B70710F0A61B6B
:107D4000B70B881F991F5A95A9F780959095BC018C
:107D5000CD01089597FB072E16F4009407D077FD08
:107D600009D00E94963E07FC05D03EF4909581957F
:107D70009F4F0895709561957F4F0895A1E21A2E47
:107D8000AA1BBB1BFD010DC0AA1FBB1FEE1FFF1FBF
:107D9000A217B307E407F50720F0A21BB30BE40B0F
:107DA000F50B661F771F881F991F1A9469F7609556
:107DB0007095809590959B01AC01BD01CF01089510
:107DC000EE0FFF1F0024001C0BBE0790F691E02D64
:107DD00009940E94BB3FB7FF0895821B930B08953F
:107DE0000E94BB3FA59F900DB49F900DA49F800D56
:107DF000911D11240895DF93CF931F930F939A9DA4
:107E0000F02D219FF00D8B9DF00D8A9DE02DF10D41
:107E1000039FF00D029FE00DF11D4E9DE00DF11D41
:107E20005E9DF00D4F9DF00D7F936F93BF92AF92CB
:107E30005F934F93D5010E94BB3F8B01AC01D701EB
:107E40000E94BB3FEB01E80FF91FD6010E944A3F99
:107E50002F913F91D6010E94BB3FC60FD71FE81F4D
:107E6000F91FAF91BF910E944A3F2F913F910E940D
:107E7000BB3FC60FD71FE81FF91FD6010E94BB3FAB
:107E8000E60FF71F9801BE01CF010F911F91CF910F
:107E9000DF9108950E94BB3F460F571FC81FD91F8F
:107EA00008F431960895689401C0E8948F929F92E7
:107EB000CF93DF930E94613FDF91CF919F908F908E
:107EC000089588249924F401E401B0E49F93AA273B
:107ED0009A158B049C04ED05FE05CF05D007A1077C
:107EE00098F4AD2FDC2FCF2FFE2FE92D982C892E63
:107EF000982F872F762F652F542F432F322F22272D
:107F0000B85031F7BF9127C01B2EBF91BB27220F5E
:107F1000331F441F551F661F771F881F991F881C1A
:107F2000991CEE1FFF1FCC1FDD1FAA1FBB1F8A1449
:107F30009B04EC05FD05CE05DF05A007B10748F061
:107F40008A189B08EC09FD09CE09DF09A00BB10BCB
:107F500021601A94E1F62EF49401AF01BE01CD0127
:107F6000000C08952A0D3B1D4C1D5D1D6E1D7F1DCF
:107F7000801F911F0895A29FB001B39FC001A39FCE
:107F8000700D811D1124911DB29F700D811D112452
:107F9000911D0895DC0101C06D9341505040E0F700
:067FA0000895F894FFCFE4
:107FA600FF0001C8000101010552414D005058343F
:027FB600310098
:108000000106B5064E70F858985684D84C5B8C4BD8
:108010004C3B1C427070384BAE783C0670B958CE61
:108020008CA08D08849B76761908AE58FC58F3997D
:108030009E990AB5960D9E1596BD966262C6CA5067
:108040001C231908AE58FC58E21BE2371100EE5C05
:10805000981C45028CA08411008D08580CA0B5A274
:108060007B9BCBC313E3DB4B43CB3B434B535BBD0E
:10807000B25100E30E1C5016B523110CAE0E93C482
:108080008370FA70A033F0B80E6150F86550C4F0F8
:108090007C30147C3050BCE0C8CCF73008C8CC66CB
:1080A000EBE0D5884FA550F0D44FA550D43FA8F0B1
:1080B000EECBA550AEB87C58AE8CA74C3344983C60
:1080C000A883B5BC84634C6100431300A550EED473
:1080D000D3B87C588C33A3B070E0A550EED433B83D
:1080E0007C588CC378A84E703868F828EEE8B5BC88
:1080F0008860A04E70B85860434C3748ED04711C3E
:10810000EC1F0C1B919CCC9BCCA3203C560630183A
:108110006621463087662F110C1D02C8CC5C5AD0F0
:108120007038CC9704624728707C3014FCE090666D
:10813000281C70381B2E28BC30EB33B898A8E00000
:10814000A383634323387C8338FC6B383C53387CEF
:108150003B387C2338083C8C1BADBC300670FCE0FF
:1081600048711C8C7F0C238914538C2B0441B02341
:10817000F8992C4C3F305166FB610044ED040CC76C
:108180000100D50CCC0F3008999C0CCFB83C580C92
:10819000D91C6000711CEB5924305006CC4F300CB8
:1081A000B19CA6CB091E201CE2153221460100E03D
:1081B000D50CCC3F300A999C0CBBB8F10C7CD80490
:1081C000884484D83C467CA8C46100CC4B30C306AC
:1081D000203C1C6ADB78EE30BF0E66267BA606705C
:1081E00038EE4B3EB75EF0FC56468B300770999CDC
:1081F00051844E7020B8BC588CC50284983CA8E0CD
:108200006D5820091EC8CC6046F070306906787C35
:10821000660FBC6670380EBAF038BA6EB7F04670AA
:10822000B858CCA03846BC30E660C4783C1C420A42
:10823000BD8E60A0587058585870707070E0DCA007
:10824000C44484C44404B1702DD91C610030FF0EB5
:108250004EF0E020F0AE70AEF0A6DB309C3C30A7D4
:108260003C309B685A2E28704E9C103020E84E708F
:108270009C90105C1010A8883006999C3069067894
:108280007CA63C68D5060ECC1F4CA038CC432E28CB
:10829000BC30B606E00C6B90662870387C1C0A1C5B
:1082A0004E70E06228E01908AE581C58F6BDBE4476
:1082B000F64348F62BF6603D02568C33841100B12C
:1082C0000EAE8E301EC63F4CC3301AC6A36E3008A9
:1082D000EE4E702E3C86F313EE66F3EEB8AE3D0222
:1082E000D588387E7E8953065E04467056607CA62B
:1082F0004708FCA627FCA64B3CED08E606E6E6464A
:1083000046FC06E01C8ECECC474C37784C1758E024
:10831000CC8338BC3AEEE2DFCE308E1A3C7E1E4E65
:108320001CAE3A30AEAA3CBECB133CEAF358AE6E5C
:108330001C53CE3A303C46FC6E1A3A3CEA38CA2806
:10834000E044E23349A459A41B49A4E5A43C1E4ED1
:10835000BE4F58E5A4D898D83CBB2550581CDD8C9E
:108360006EB858E065BC8C1BCCA0044841B0336D9E
:10837000BCCE992CF90C8C2F3C580C6765204670AC
:10838000B85888D3C4B83C5804987C58042B492466
:10839000B8587CD804D8FCD88404D87C8498A8E049
:1083A00085BC390C048CBBB85804ED04C4E0B01A89
:1083B00030E61B1C50BCAEC1B0AE4D14DDAC492440
:1083C00065205DBC651C4C752EB85888987C580893
:1083D000983CA81D02B85884987C5804A341B0F971
:1083E0000C3330A7C8CCF91E66DB2DAA8D08F681A8
:1083F0000B1C98B10A30FD70F0B8150A46A809BAEE
:108400008BA3ABDBB3ABA39B93FBA3F3032B23C9DE
:108410001230CFA663B51230903B1D140912309173
:108420000286061D146684E37330D04330CE0663A3
:1084300065169C021D1411B41DB4D884D81B30A835
:108440000629BF30AE06AF19B4D8D91C8C2330E052
:108450001B30D02D149388309C0613841D1411B446
:1084600006D91CA6D88C7384D884E6BD1C090E04DA
:10847000DD14661BD806163066066B1E7E8C177ED2
:10848000A1140CDDAC5D1E307006C7668B307466BF
:10849000D3069B3071463C301A7E3766EB305C4623
:1084A000E80B3065DB307A4636BB30689B301D0602
:1084B000CB3B301A06CF6667B8D8485CA2E2178873
:1084C000D8E88B266637DD1430053B302D23A61CFB
:1084D000D0E51411B46E5606D91C301D1C621F065F
:1084E000970C2B301FE5140912E6161D1411B46EFB
:1084F000060404CC13081C02A65A56BC1AD91CB890
:108500003007E8BAEF6E49241C0C2DB50CE5A46EBB
:1085100006D91CA675B0E9145B6E3DA41DB48E0689
:10852000D91C1C627330CF2D1449246E3DA46EAE4D
:10853000C512AA625830C02D14CCEF8CDBE0B8B85D
:108540003044E86914061ED91CA1143020E8F89CB8
:10855000E213A83060A820045330C848C8CCA066F5
:10856000E34404048449242DA806864C2BAD7043B3
:1085700093C1B01EA114C66FCC4F6914061ED91C3E
:10858000A11409123020E84924B80E41A41DB41CDE
:10859000EAE38E56063C3040FCE0BD1C2012050785
:1085A000204924785A0E43660E7038EE477A30C060
:1085B000661BAEA3AE3CE03020E80C57302006F836
:1085C000A85666A00879B2D91CA6063C30147C30A7
:1085D0001C50BC087A3056D84C1B36448C1B048483
:1085E000D8E80C8F3020E8E09E4EA0A60E3C266610
:1085F000EEEEEEEEE6A63C266606BEEEEEEEEE06ED
:10860000AEFC2E6E0E60DE77DC101E7CFE7FFCBEA4
:10861000FE5FFCBE437E9EBE1F3CEB7E3C1A9EFC72
:108620009CBE603003FCE8D34670CEED28041413E2
:1086300008AE58FECD7DE05CE0D460D0DC6202D7AD
:10864000629362E97CE0C2E223302C1B302ED4A07E
:10865000D57C33E97CE0D414030CA01C98E217D439
:10866000A03045D57C98F6CD7D7B1C38BC44137A70
:108670003076EF76DF7617483C0AE0CC1BAA7339D8
:1086800088E60952D5883ED74DA6251CD91C302036
:10869000E81538004C73B0E22F302DE813B8957C04
:1086A000D91C7B30C30E203C0A2365202B4E203C76
:1086B000D026E806303404661708B0C606C61CD0BB
:1086C0000C1BE21722E866F13A0E30410660304B8F
:1086D00006F3302506FCE61C0A301E6A23666A375C
:1086E000FC0E66813A30CD6A2F3C3E3EA366E030F8
:1086F000610660306606A0301ADBB03C0E660401ED
:10870000AC0C0F1CE22F0E16913E70012053AED818
:108710000C27B0B13E088BC1B0B1BC492444B0A114
:108720001CF93E589DBC981C1D88FC1EBEBEDDA4D5
:108730004E70E5A4D8B0D83CBEC32550704670B08A
:1087400068301E7CA11C0441EEB83CD844D8FCA87B
:10875000D91C78D884D8F04926410CA83080A6E6E8
:108760004EF070B858CC1F0C1B66664C17168C1355
:108770006E3C588C233080464C2F8C23767676BC0A
:10878000588C2B76767676BC56EE3C56EEEE4E3016
:10879000107030FDF0AEF046F070B858E07CD80CA8
:1087A000DD2F580C2B30844D320CDF890C4C3304F8
:1087B000B170434BF8E61F26E865144C19387DBCB0
:1087C000651CC8F84666E8B858F6F62B9DBC410C07
:1087D00004B898A859248C47C1B0302EA84924C1A8
:1087E000024E28E8A89868E0FC5C0AB8AAA8E0B0A5
:1087F00030E83AF6E3E030107030FDF0E0000000C1
:108800005AEEEEFCC6E6E6C63C06BC5CEA5A505C94
:1088100030662B22E399C63AC60E3006C3A6E67A26
:108820005ABC1A30F6F63C58FC0E3C3A301C0A3C56
:108830005AB03AE07AF30438BC585C98FE9526FCAE
:1088400010D0900EEE7E93EE0C31237EDBEE7EA3F5
:10885000FE13081C78221BDCEB1465238C27787E22
:108860006881228CAF88DB780EDC901E6F080CC705
:108870004E6E56DC5050087B0C5F0C1F0CE30C1F37
:1088800008330423780E561C561750DB7E63EE7EA9
:108890004B9C78221BDCEB9443E030D066FB20E05D
:1088A000D400980278A26838BC983C28E01CAE58E6
:1088B0000813044E6E56DC90688DB8B8580C2BC95E
:1088C0008C89B68CB551884EE80CDDB641A48A4936
:1088D00024DD20792419B46A1C0A301D623F0A2B5A
:1088E000AE9C58636E1DA4DD8CC1026E601CCB383B
:1088F000BC58780ED91CE9501C622B62BEDCDBA28E
:108900000C471437D4A250DCDC8C5BBE1FDCEB8C34
:108910001BD013D0DC4C9BD47F1EBE2F5467DCDBF6
:108920008C1BD013D0DC9BBE131EBE5EDC0C135020
:10893000BEE0DCA0760C831C6247A29C622FA222C0
:10894000230AA2501CE0169CE0D2D268AED2D228F4
:108950004EA846F070E0D91C78D808D8F0AB781C47
:10896000221BDCEB6206569C622BC6DC14DBA05695
:1089700013860EDC50BEDE774277FABEE3A6426F66
:108980007E07A6FAD31EBBBE2766EBE31E0C13BE02
:10899000AE0C83A550E854670CAD2355BC410C1DAB
:1089A000024EE860E078E05CA01E0C1B9C131C22C9
:1089B0002B62BEDCDB0C83144742F21F0404D00B95
:1089C0007676130456DBD45F8C2F543F3E63BE5340
:1089D0008483B8580C2B410CFD8A4EE8203077E098
:1089E000689D2244781CEA31B60EB8AAAE3C68F8FD
:1089F000AAAE3CA838AAAE3CE8387C4AFC2878FEEF
:108A00003B09B8B8D84C578C47D8DE3EFE31B8F396
:108A10004484D8063020665746F07038566637D9F9
:108A20001CA6E853D91C230841B0CE6DB81902B872
:108A30003C5806F804A0965C1427D4B6E30EF62B37
:108A40008C63DC541F66E333D4144FA6E32E8A3ABA
:108A50005B0E0A061C2A4F0E7E8E9C0ABA60E0AEA0
:108A600056E346A38C431B66239A3A370C1F4E737A
:108A700084762B0C4B069CA206BF1BEE608DB8CEF5
:108A800008D528EEE9502E0EA0B8BCEE7EE6C6FE54
:108A90001BDC508C752A5CF65B752C552CD4DABE29
:108AA00026E37B661FD4EB46BE3F752C552CD414B1
:108AB00047BEE3D4141FA2E39CE04C437E9EBE4716
:108AC000DCD4E3DCA07E83A28C1BD013D0DCA26BB1
:108AD000552C4C752DF3BEB6AE60EE5D1E5C4C930E
:108AE000063003562FC6FB462746FBC68606A6372A
:108AF000D4BEE31ED3752CD4143FBEE3A2D414EB32
:108B0000D61B1C501CA63033A6E00D2AC6A6C6A64E
:108B1000F306F6C70BE0DC201FD4EBA0E0A28C1B11
:108B2000D013D0DCA2E0A01E7E7E43ED28D91CEE3F
:108B30002526DC10FEE0DCD0D07C70D91CB07C7027
:108B4000061C4AD36A2775B0AB3020DE7E2320494D
:108B500026E8D309CA008CB3F12E461AAEBCFA1A25
:108B60003A30E63A303CC61C3CA2BC02F6F6DE6B5C
:108B7000F6277CD90E7CAE0819BCF90EF6CF75CA63
:108B8000AE5851000E389C0A983CBEAE2838FC26E0
:108B900084E6C67C287E7E677E01CBCDC63000EEA3
:108BA000CC4371CC66250E22C8EE66A30B000000F4
:108BB00000000000E55CBB6100A3E55C8838FC6652
:108BC000E6876B1CC4E666664B095010841CEE01F8
:108BD0003041A478901C8C476A550E4DA43DA49D4D
:108BE000A48C1F7CAAB18CC1B0041D1425FEA55015
:108BF000EED44B4670B87C588CED02B070EEF0E0CD
:108C00004EE8286AB3B83C58A020BC30C1FC1CE038
:108C100000105B504B903BF3D023BD8E103C064CB4
:108C200023308006708C83AE1CE2EEEEEEFC5C50CE
:108C3000303CE6E60E9CF83C5842A65844D91C301D
:108C40002006861CB86AF3AA6A37C6E8A8B8D3F823
:108C50007E60BEB03AE006B8588C233055737C581D
:108C60004C3305BCEEE91BB8580CDFB05A3C06305B
:108C7000667E679CD0FE431CD03EFE53FE470658DE
:108C80000ECD90EE87B00EB85830505E7C067C302A
:108C900076B1B5BCEEB85CCA46A80C2BE21B1C2210
:108CA0009C5858CEBC30147C301C50BC5870305985
:108CB000E2B858E0D8A686251CC1B030E02D1404D7
:108CC0001D1030E09C58BC0E66483D3A44251C1DE2
:108CD0003C984D14987A30F6453AF6F6167A3016E6
:108CE0003C5804D89CA298A2580C9321382B4C5184
:108CF000370C33BD386520A30CB5374CC9370CB7DA
:108D00008CCD378C8F5E7B3091AEFC9C425D1CAE6F
:108D10004D32C1B0711C9DBC110C1D028C1B0CB3DB
:108D20001538838C6B4CF53B0CF53B4CC9376520F3
:108D3000838C653BD32D38DB4C41370C3381346554
:108D400020A3203C0A30836A7F3031E82D383B0C69
:108D500081356520C3B8FB0C3B8C678C1B4924060E
:108D6000A6A6B8A6A803B8F8E806A6F13B4924B819
:108D70003C0E8CA730CD8C2FD91CD532AAAEBCA806
:108D80009858889858653A4C5330AEAAAEBCA80C97
:108D9000571B301E0C0B668CF39C98D844D8581C7B
:108DA0003001AAAEBCA8C1B030D02D14A83060E804
:108DB000D53649249C98D848D858D91CBD1C090ED2
:108DC000042021386B4C778C5F0C1BBD3865209BD1
:108DD0003030E81B30305E172EE83CBEFCE8953A98
:108DE000BEFCD056E82138430C1BBD386520BBB80B
:108DF000E04936BD1C1314201538BB3020A8A8A8A4
:108E00006D7CDC100E304C66CF21B0DDAC49249C6B
:108E10009858B81CD04C1B1CD0AE7CA2813A65205F
:108E20009B3057BE5E2B2666DF03305466E3834ECD
:108E3000BEFC1CD0E81538630C276520CB4EBEFC69
:108E4000D0E81BB8E0301F43301F23301FE8E8E8AC
:108E5000DDAC4924F81C98E8B83C58880898FC6DAB
:108E60001C61001106DCD01C0EB87E584CE706F8D9
:108E7000425646BE47A6E606E6E646A39C98584CF0
:108E80002330804686DDAC4924B80E8CA76686E682
:108E900083DDAC4924B80E30C8E0C8CC3B66E32083
:108EA0001938436D00C1B020492495BC110C9C9821
:108EB000D84C3B4C1FAEBCD1A6D84E5CD070AEBCDB
:108EC000FE6D076645023040E6C8CC6D0266DB04E5
:108ED000B1703C30E866FB59364924A5BCB8D88847
:108EE000D8A84E68D91C1538734CD13E957CB35D1B
:108EF0001C8498A84936492478EEAB7C4A68251C26
:108F0000D91CB81B0CCB6520E36D7C06251CB6BBB9
:108F10001C307F6A93303A6A73302E6A53302C6A61
:108F20003378EA1FAA0A3C68EED91C21B0B30000CE
:108F30000000000049248C931C78EE4B255068B843
:108F40005884986D1CB83C06300F6A291A86D91CC3
:108F5000DDAC492478E0DCA01CF2251866301E1C2C
:108F60006ACF78581598EE8FB858F83C9C580C5F2B
:108F7000B80E95BC110C810A4C37587C7048840C93
:108F80002B88B0A11C44B8D80C23584898589C583A
:108F90004C4B1D3C4924980E1DBCB80E86813A8C62
:108FA000537C560EB858AE444D32587CA11CB8586C
:108FB0001C98BC580C5B30E61BD03B3A30E617E0FF
:108FC0009010589C583532F8E6C1B04CA066664CFB
:108FD00013061EA1143020E8E060B0303360B030DA
:108FE0003A70EEEEDADADAEEEE7CE041A4584DA407
:108FF000EDA4D8E05CF84A0EBEBE175031020E8CCC
:109000002248E30130028C043EAEC242880480BE96
:10901000202C51C0202ECC0DA241A9AA84F902C453
:1090200050020D3384537FBC3F00000004DC78778E
:1090300077A50400DC4E0DC0AD804070097E441061
:10904000226323144F8CCCC30DC912942379D33FD0
:109050000030004100E45C480640200180840B3071
:109060003417E33B03614413D323C1903331FAF443
:10907000E4D2CA44F24DD4908823743880DFCFB351
:10908000F3BC6C759792E288CFD3CE4060C1562175
:109090001E168C74E8237655D4B87088323931D5D1
:1090A000D193F0E04D472E1FB82F2C89617420C258
:1090B00040844410A0363513834E847F64D84E55C7
:1090C000E88080D274124C1BE360A307800F28CC89
:1090D0001B31841C91DC3E01FC279EC001316D8256
:1090E0000FEEFF13DFCFFBFC27D90F9E1BC43013FD
:1090F00072813CF7F73CF743182F2EE388A4033C1A
:10910000000010D544483012D070C5713003B0173C
:10911000470C3C12C470CC030D8BCF8002470C4D22
:10912000F348CCC44C7888871F871EC715335F84EB
:109130008F2341C0084013CF4688CC00253840CD4E
:109140007512080A0D21334073C4044383C700F825
:10915000B1C44CFC72FC85BFDB87C4040C232031F6
:1091600023715CC00E193400C6848914C3703CD1CD
:10917000F3CF90E150CE6192DFF120A955A34A15BB
:10918000A82A166262403C8777F8480491C33833B6
:10919000C3400431F3B0F7C9C4E4C88DBBCB34700D
:1091A00038E013130741C43C7324232378D1C43D12
:1091B000215E141F13CAC53884C4AC737C7CC8B547
:1091C0001012024080D844C84417612520B33D20C6
:1091D000C623FCECD36EC8C1EC0B5420F944001537
:1091E0004F1534551823FBF73284FC4C018B8773E1
:1091F000E1F81727FF0113C760D19278AF17C603B4
:1092000094D754508F8FF450E4E5A41F659A3D8A9B
:109210006BDFCB3C02CA23A3CA8DC94D8842132001
:10922000668633F3ACFC18FE43A28D0B11A2CA83F1
:109230004813144140001733CC0C0CB26D33847DBD
:1092400003C74F3CC48314F3303D14CA20CED191E0
:1092500010CC3F3CC03EFD2EF2C6F1EE98127337A3
:10926000D673F4480C30CDC980CB3483D88F2072AC
:10927000CA2033DEF32003C48A6D1458608219A813
:10928000C5878C047931ACCCF07340CC1EC97667AD
:10929000F2355B43440B1D38CF7ED0C162733F0A69
:1092A00001630E80B8B3007C8E3C05B0F4D203108D
:1092B000BB0030CD0058885CC574351A37C3D2ED79
:1092C000E2D03010A2633C03F10C4D0CE1E8CF304A
:1092D000FD1107723C7012948ECB9025A18C23094E
:1092E0001C480F8A036AC214130FE30300A3388BD0
:1092F0002AA04C03C431CF0C0CC02C0200DE0AE2C1
:1093000038FC494000C0001D841057195F3DC44E11
:10931000C47FC3FF5DD64BD524CE0358C8CA19629B
:1093200081D117FB420808B2338443F5FC414CCC91
:10933000125328C634B952B9CE0350C400C846F2FD
:10934000CE7FE00932713233F100402233870C8C3A
:109350002CC5C40123EF0B0725F653843401339049
:10936000CC4C04E415AFCECC013931C710733303B4
:10937000188101C831313E1E080700F2C38071FC1C
:1093800063C5C8C4AC85332246E31F3B380720833E
:10939000DC0741FC13C33F6F88F8DDCC5050D57318
:1093A000444C18C04C58F8F883CC7132C3C10C0738
:1093B0000692BD78413BC4BD8F1304B3F810FA1870
:1093C000F3274ED1C7C7C7C7EBA48C080081ABE316
:1093D0007B48B13013223AC467233F437632168864
:1093E000C0F0303F32516308408F12F357B0804BCA
:1093F000F0CC0CD3C0C4DBD8567F5D34F2430503F8
:1094000041460000020103044247000027242120B6
:109410004348000028252200444900002926230053
:109420004540000F800000981E19B0456C63AB13D7
:109430000D08B0C964F0B8C9640EB01D6088C96475
:10944000CBAD130D08B0BEF053ABB063840F0DB0BD
:1094500071643BADB0BE001D606902AAB03560D337
:10946000A5A6A6B035603102B21E18B00EBBAFB0D3
:1094700061603B930201B05EE0930F030151848869
:1094800008080176008435928C031201595A860827
:109490001301215E8E0913015184338E1301A99E9D
:1094A0008F141301715E8E0114015184AB9705096D
:1094B0001601910E008883900505023007455A94E5
:1094C000130200418A940103012E8603355A810C50
:1094D000034E68A8E828E08F141398F0E0840C038A
:1094E000410C511E900C03318A87120C0308CD5E8B
:1094F000CE0C03C15294130C034E2868A82B980C71
:10950000034EE8090299100F039586922D04B005C9
:1095100066870504715E84011207995E84011289D1
:109520005E8C0504A18A0000BD8A8513047D5684E3
:109530000E05870E0548015A9E1205140E05B550FA
:10954000B8E81102981E05B0296A96040175BCE0BE
:1095500094030106B0B162BF0306AEAEAE2BB12DCF
:10956000181E0548B0296A833F030635586B9809D1
:109570000688015A940E098823831206B0ED66BF4F
:109580001306155A833F13063558C30065A68F147A
:10959000079208B0C966930D0888CB8713098481A8
:1095A000568C020C8E0CB0156E870F0C88CB96056E
:1095B000041341743B8E01050DF9709502902D1234
:1095C00051842574BB86060FE03009999C1508610B
:1095D000004106982F31B02D62922D105184080859
:1095E000D578CB8B0301100182880325BEBEBEB0A7
:1095F0001D606666B869603102851310CC2308EDE2
:1096000004B10E94100D0F1210810E842D12B03182
:1096100066900F1413A50E0000751E982B310E0CCA
:10962000B0CD6E981413010C38EE238C03128CB558
:10963000514E70EEE8B902930803B0FA1BBEE8B3CE
:109640008910A06964EE3A460BBE3C1898F01B8E58
:109650000412F552840E12BD2A8E14120D9E9E1213
:109660009552890313015A8613295AAB4E2172ADC4
:109670004E88DB8705124E655A930F0351846B8E1B
:1096800001145184438E091351848808E17A851AA4
:109690000913555E94121113B0F9629413130081EB
:1096A0008A8E0F4552AA14134950356043AB1413E8
:1096B00049501D60B92EAD141398A0BE589BAF142D
:1096C00013495061607B981E3031E16E850E0F1496
:1096D000795A97050916BD0EBF304D18455ABF1966
:1096E0004D18A55ABF303C18E956BF303D3C1825EF
:1096F0005ABF193D3C18055A993E3C18F8AEB8E8D7
:10970000AEA8B902BF193C18BD56BF303D18195A52
:10971000BF193D18515ABF303E18C556BF193E18E3
:10972000E156001D92910518830504482394030F08
:10973000B0E57E8E070913D13E8E0F0188ED0471CE
:109740001E86060F0184BB00009D7CAB0000201C20
:10975000E2E2E283B87CD84C1F481344D83C98A876
:109760004451064DBCE27F410C8C3B8498A8448553
:1097700006880CCB53410C04840C1F08830498A862
:1097800009B8634EE6BCAEB90C004A545C6FD6CA49
:10979000767D4D453C8C92989EA4AAB2BBC2C8CCA3
:1097A0003AD1E0E7EDF3F901097C0E2B14242D32B8
:1097B000353E4763545A6B717C82881A91993245C1
:1097C00093779E28A4A620ACB94F30C8A3DCE761EC
:1097D000EC4209FC600EC01F2E52575CB265696DE9
:1097E0007177883792989EB0B9A8C1DA1582D0D621
:1097F0000EDCE8EF1A14E208F6204CFC286B2A0075
:10980000C88C2409E71892C29EA3E7274DE0489E22
:10981000ECB83C5808987CA8E04E70F8E085B5E0BC
:10982000FFA0B0BE001D6070E0FA174EA05CF6A06D
:109830006636761B26E0F61B4E2B4A6A56D4D4E0D9
:109840004A545C6F0820F66D7132454F61ECDCC004
:10985000A66B982A3A47ACCA63887C82987DAA2B6B
:10986000D67654DC1A20E80E777C0E0E999357308A
:10987000F3FC42F96052280114E237EFB9B2B2E0CA
:10988000141F1A3E155CBBD192FCED453CC8094D36
:109890002EDAB0B9A8C19E2DD677A48C716535D0CB
:1098A000E7FDBCEEC10295BE69CC886B825A23F0FD
:1098B0009D585C0EAEF0AE6E70D494CBE0A55043D4
:1098C00032EC4E70783C0602E01CEA603CEB4CA4A3
:1098D00091EE6E98AE6150AEA0FEA03E337EE000E9
:1098E0002800D58818B550B902B550B5504E70381B
:1098F000AE7828B868F8A8AEE8E0A04E6E60EEE05A
:1099000047710E834140424348700E0078464567D8
:109910006075E00017141110534C0F00A8869C725C
:109920005259911C1815121A515CCF96A94E9D766A
:10993000565A901B19161305575DD085AC4F9E984B
:10994000505B08000C0C0C00555E07770C0C0C00EB
:1099500041460E4E5155593A617E0E5E2D2B2A2FEF
:1099600042474B0052565A2062257F00373431302F
:1099700043484C4F53573D2C631D9A0D3835322EBA
:1099800044494D5054583F05643C9B243936337E3E
:10999000454A08000C0C0C00653E07870C0C0C882F
:1099A000EE61501BDA26F6EF1D64989417D44AFA3C
:1099B000EE58AE0EF09C4A5CEA271C505C0E0A4A38
:1099C000EEEEEE5C262666421FFA06E247FC4626CD
:1099D000E21FFC468C13BE70981D60580E38A60618
:1099E000DA661FFAE7461AB160F08898AE8C5385A4
:1099F00050A0B0EED33E1BBB85508C97A0B03E7BF1
:109A0000CB8550EEAB630EB07BF8615070B0EE5377
:109A1000630EB0CBB8AEF86EB7CC6F4E70B8D84C02
:109A20003FD88C27AD7062C102B8AEF86E6760CCCB
:109A30004341A4E5A8BD8C834E70B8D84CA7D88C00
:109A40003FAD70641BCEB0EE8F2BEE702BCEAE0010
:109A5000B0A8AE58711C98AEE0B0A558B0AE4E702C
:109A600078BC46063C68E078BCAE300560061972EA
:109A7000EE38A02E6EFE433E2F385E3E537EF61B20
:109A800056765CE2174E60EE0EF0386E334C810B6A
:109A9000C90ACEF0AEE0CE7EFEBBA118CC60B858AD
:109AA0004C608CA00841B0B83C58084898FCA8E02D
:109AB00046705CA0D4D4542FCE58E09CD251B5A3AC
:109AC000983C98FC58B83CD88C132E0C1B2E2EBCFE
:109AD000F375583005755830087558300758B8BCBC
:109AE000D80CA0C4D8584E30FFD8BC0E7CA0BE60A5
:109AF000F1585B657387A1C90B3F8F15B01A30A66B
:109B00007E677E777E8F1ED8BEFBA6DBE0D8A6F3ED
:109B1000E0D800A6EBE0D80000A6E3E0A95C98BC82
:109B20006D1EA95C88CBA95C08ABB83C588404E0E6
:109B3000044E70783C5A70AE38EEAE0EF0386E605F
:109B4000EE0C134EF06EAE7BD55C542B1C52F0E045
:109B50004EF0D460AE7038DCDCDCDC93D55C544B6A
:109B60003CDC5010F070F03BD4C7AE7038DCAADC9F
:109B7000DC7C94E36B300870AEE0DCA05C38521CF7
:109B8000AEEE6FAE0E7038D494BB5CF260DCE09C3D
:109B9000D4D4F2EBE048A670851458C15C4E708EA8
:109BA000783CC6B0C67F08CEAE584E3CE6BCEE78D8
:109BB0005A7AAEC39806374C098348E07806BCEE63
:109BC0005A3AAE5878E62BBC1AEEF0EEAE0C3306DD
:109BD00033AE2E6366E3AE70FABC1A3CE638EE3C58
:109BE00070662FEEF098EE41A4CC17266E78063CF6
:109BF000063C063C686E4435BEB8584898A8E0005C
:109C00004E1B4EBE5C501B2E7AD898463E5ED81C2A
:109C1000D4763654E3EEEE6BD86EEE4B2687D86ED4
:109C200026DFAED80E23D8AE2BD8AED86E9E5E5BA4
:109C30008E1E263BD8FCD86EA66E264B66CEBE1E68
:109C4000D4D4C34EAE98EE2E76767600CB2E7AD84C
:109C500098463E5ED8065E139E0ED8DCDC8E132E30
:109C600062F354CB98AED898FE1B66CEAE5C4ABF6A
:109C7000EEAE5C0EE66B3A5BC62622DE6EFA604EF6
:109C80001EE0C6C36E63424F66EAE32EFAAE4ED8BC
:109C90004E5C50EEAED8AE332E7AD898463EFA23BC
:109CA000D8465E139ED85EAE6E2E2BD8EE66D85C7C
:109CB0004E13228EF32EEED4D4D3AE98C1622EFA78
:109CC000AE5E1BB5A23ECE6EEEEE0EEE5A0EEEE688
:109CD00013BA4E9C4217AE8E4E6EDC50CE5322CE3F
:109CE000F34EEE94C963D4CABBA63BC3FEB7F6A736
:109CF0000E8E1CEE8A5C4A9766061B36E04E22CE1C
:109D00003EEEC21BAA260EC223EE2EFBDE338A6E67
:109D1000262EFB6A626B7E5BEE865A5E2A4EBAE0A6
:109D20004E709ECE68B8A606A8E07E78EE68B8A60B
:109D30007EBB4E7078FED8B8DED8E01D648CB5626C
:109D400098941FD44AC9622EFAAEDCCED86ECEF6F5
:109D50006026E63B66EE1ED44ECF66E076FA3B36D2
:109D60007E13484623B6AE932EF0BEF01E06FA8E42
:109D7000FB2EEE66DB8EB0B5604CA0FAA00EF81D8F
:109D8000620E6964EEB03D60556469620E556435DB
:109D900060696475624E5C2650E04ED88564EECEF4
:109DA000E05C4ED01050D050105090D0D050D050D9
:109DB0005CE0FAA00E8E2626065C4647D4941BCEA5
:109DC000E066D34EDA8C93DCD4239D642BDC9D6457
:109DD000D4D49D640ECE95620E9564DCD417DC95C8
:109DE00064EE4EEE93CA0A0ACAEAEA4A8C330E06B9
:109DF0000E46E04ACAEAEFE0BE6E8ED8988E4E2735
:109E0000980EE026CB5C626EA5622EFAAE045E135D
:109E1000081E1A6ECEE673CE5E7FDCD494856B2668
:109E2000DBF568A3B9685C336E66AE333A8EF32E09
:109E3000EE66539CE22B62E24F225C23AEFAAEE266
:109E40006B4E5C6A0E1C500C13A66E0E4C1B096008
:109E50008C1BBE1E1162228EF32E543FEE66D4EE92
:109E60000BEE4C2B2968AE6EDC909CFA9BDCE23347
:109E7000628ED89883268E7E9BCECECE626E0E0CDE
:109E8000396153AE7EF32E7E982BD8988EEEEEEE8F
:109E90000E6ECEEE2798AEE066CB8ED82695626E1B
:109EA0005A5E0E0C1BE1644C1F0160416AEE5C902F
:109EB000D010905010501050905050100B4E54979E
:109EC0007A103AD4E7543F148F94CF54FF9CD05C5F
:109ED0006B9050D05010D050101050905CEEE000BD
:109EE000D0501050D050101010D0D09C8B1CD0D01F
:109EF000101050D0509010DC2B5CD0D0D01010D06F
:109F0000505CDB5CD0D0D0D0501C9B1CD0D0D09CFF
:109F10006B2EFAAE8964B861500EF85EBB06BAF6D5
:109F2000330D62E6EB66EE5ADFE64FBE1EFEFE1E06
:109F3000FE1388B85E2EFAAE08DA77D164FA1B9861
:109F4000FE072E11622EFAAE3E5EBFDAABA606E623
:109F500083461BA6080E5E5A5C8A62228ED8988BB6
:109F60005CCE62AE4E4D6E422766EEE3D8A5608BA6
:109F70000160B32EFA0EAE0E26E6B35E57AEE56470
:109F80005C4EA60E6E3B08CB54F7D43E26DB738E98
:109F90007EF3982EBE333E6EEED4940BAE8EEAEA7C
:109FA000EAAE9CD086C6E35C8EEEF568A56CFAE35B
:109FB000D4BB2E9C822E8EB5680C376E8E6E2E6EA4
:109FC0001CA56CFA3B8EDBEEDB8E235EEF665E0C2F
:109FD0001BBE00B5600CCBD164496098FE356AA603
:109FE000EEDB8E29686E5C1B2E62F34226DCE08C71
:109FF000A04ED8B968EE75620EB968B03D60EB004E
:10A00000000000B0094648167616810B70C15A014F
:10A010000C10080120040114010401140120051290
:10A02000120F120D050D0F1219200C0F13140E0F25
:10A030000E0518091314050E140E150C0C10120938
:10A04000160114050F1514200F062012010E070526
:10A050001001030B090E0714121920010701090E44
:10A060001905130E0F12010D120F0D08B060303AD2
:10A0700070BC5C50100EC1B0AE307A0656A856D3F4
:10A0800049240CA08DBCF10E2170B8F0B00E4C2309
:10A09000BD701BB57069708D70B00E356069704C05
:10A0A00023B9701BB17081704670F84C1F48EB0EDD
:10A0B000B835606970AD7081700E626970A9708D7D
:10A0C00070F04E70F8280D729D585CEE615060EE95
:10A0D0006670EE38D494B34E70138CA0BEBEBEE052
:10A0E00025601B1D60A550F05CE0D4D4D4D4D460AE
:10A0F0004E7078BC26DCD4EB667038A05CE0217032
:10A10000B5701D74F0BD700EA970EE4E70EE6162F8
:10A11000842170B1700EA970356081648C27B57090
:10A120001BBD700E3560BEBEC9643160A970696028
:10A130008164A9702EFA0E0960C9644D60FE89031E
:10A1400005608C60F088B9706BB0FA33FE238888A4
:10A150005EF00E35608964B80E3560D164316005FB
:10A1600060F00EB8AE6160FADF0ECB8C1F88E08421
:10A17000E0AE88FE13485EF0B0FAA00EEBAD74E3DB
:10A180002E0E7AFE4B480C338C238488445CA60642
:10A19000E6B177468FCECE235C62EE570C0785641E
:10A1A0000EA6AE3D7A0C0D633960AD746ECE5C5A6E
:10A1B0005E26E6433ED454D3EE3D7AD84E3ECE6B77
:10A1C000AED8221ED8AEAEBEEB1E2EAE8ECE93D82B
:10A1D0003ED86EEED454B3EEBD606ED8469CEEE130
:10A1E00078EE132E62F38E42FA1BDC9B0CE389643B
:10A1F0000160A9640960D16449601E0560B05ED841
:10A2000098464D60A606E6A176B176DC6654EB5E14
:10A21000B5608C3BBEBE696431608C2B6964316073
:10A220004C87696466660075608C3F4E5C66503D85
:10A23000604C13BE0C60F0E04E6E5E546F94EFD431
:10A2400027544F14679CD09CE0DC90901090509065
:10A2500010505050905CE09094F3631C5D789C50DB
:10A260005C109CE05C5D789C50DCE05C5D785CE0C0
:10A270001C5D781CE00808AE0E2EBAFE43880C1B4D
:10A280008C13485EEE4C457B8C2BAE0ECECE4E5CD6
:10A290001050EE66F62F661B268EEED898EEEEEE88
:10A2A000CEEEF69F8EFB2EEE66DB4EEE98EE4C1B4E
:10A2B0008ECEEE8E5B2EEE98EE4C0BE6F7EEEB8C30
:10A2C00047884C1F48734463840CC38C1B842B88C1
:10A2D0001B8564436E8E00AD743B26F6278EB32E2D
:10A2E0006600B5604C5F98EE66006960696449601D
:10A2F000D8AE0E263B6EEE3BD454B726E36E4EEE40
:10A30000E178EE133E8EF32ED4CEEE549BD88E8E93
:10A310004E5C50D89C90905B8A8ABEEB1ED8AE4EA5
:10A320002ED88E1E62ABAEFAAEFA0B7E661E8E9BE8
:10A33000980C4F8C3B396023B0D898464D60F0D1D3
:10A340006449608C13F08C13BEF00B5ED8AE98AEEF
:10A350000C1F8C1F866EDAC3D8A5600C7B8964D174
:10A36000644960016005600C8739604CA0BEE04E16
:10A370005C6A560E8E0CA02300ED64FA0D63B04C9F
:10A380009F0E1E4E5C66D01D604E5010D0D0D01077
:10A39000501090109C506960F60D62E01CA09C6EFD
:10A3A000138E26F34EAEEEEEEEEEFCA0A2E0CED47F
:10A3B00054AB139C42E60D63B0221FDAEBAEA24E03
:10A3C0002E5C105CEE22270D622EA2F3A637EEEE75
:10A3D000EEFA9BAEB04A1C5090B562B0064E3055B6
:10A3E0007C067C30E04924B83CD88C1F881384D884
:10A3F0007CA8E0302D9C58A051B698DCD0CB06C08C
:10A400001000000000800000000000048080042094
:10A410000020030001080CC41431000D320003CCED
:10A420002B28900210003314900130021028400CA9
:10A430004070A2015039980332900004800000005F
:10A44000C0000580000000005002420AC035003004
:10A45000300000DC000C8A04000068CC39000000E9
:10A460001AA031C1030230B9C040000C00008C00BA
:10A470001303C680088000B32100000850C80032D2
:10A480000800088000080800040001D9200C80C8DA
:10A49000A024933920000000C38D06083068000313
:10A4A0003000F30125000840009013900343A64DAF
:10A4B0008E0C307003190000000003000000000043
:10A4C0003000030000003000C3D0000004C0004290
:10A4D00000380C20153700F7CA89886FC8CB02F303
:10A4E00033840090D00300000240D95555555505DE
:10A4F00095657116695AAAA9EAAA2AAAABEFAE0312
:10A5000054285A3FEFFCE3C38B000BEE2A1E80FC5D
:10A5100000AF02542196A9C091EB95E5286ABB05CE
:10A52000550AC467A25A0A99872352F51188FE4F2B
:10A530008D13EF6E4D0CBA3833CCCC2000002CDAE2
:10A54000555555551500155515005555154055557A
:10A550001515551510001000000000000000100037
:10A5600000401040101560D50CEBD10C448A12123B
:10A57000FFDA8C88221341418B63680C8859206272
:10A58000800C302003C0083E2CC100AFC4C0F8BC12
:10A5900007B3CE204F11138087FC110AA08A8028B0
:10A5A000B820C938808C02FEECC17FFB38FF40C266
:10A5B000BBCFE3684E4C4CBCFF4E5CA80300953902
:10A5C0002292DDDB4B2FF470010F3FFFE12040F2C0
:10A5D00004C631E2C8C8FF310AC88CCCDF8720012D
:10A5E00009C9BFF3EF0B1220131124C40889E01B23
:10A5F000484322C4008F24003E46402C26233C3F83
:10A60000800314D0E76361134F1344343619314D7E
:10A610003B442A400129924FFE51D23C70212838F8
:10A62000CCFC3E400C04506029064CDB60F74E0128
:10A630000C002554D8F36063F7F187AAC1FF8DE3BE
:10A64000224BDC7136EE03C5084A8E288C927410BA
:10A65000CD0420812BCEEF8983040040B74FB00793
:10A660002010224988B04ED24F861258EFA11D0FFC
:10A670003BC0323C3F11CCF21C6F974072FB423D15
:10A68000B51F02300004E3844B12F4760BA2788CE1
:10A69000B30948006262173B0202862D52B8FF11CF
:10A6A000E25E5D50B2C46D0A100C403040866831E5
:10A6B0002658594D241452330029410718240720E5
:10A6C0002900A48002C0C4808CFB0B9522000B786B
:10A6D0008E00AC928400A75423CFF8092044F630B2
:10A6E00043C0B5EE5E298FF0735A2323CEB4001118
:10A6F0008C3CCC0B480C4442BC90393E9320082142
:10A7000000203D460000040040000010000004044A
:10A710000001000001400000410441B915376CFC04
:10A72000D1170304C3CC500C0C330860C4CCD0CC7C
:10A73000800411230A3FC6C80080FFBF78EE8A3F1D
:10A74000034C0322CC3401304C21002330108028EC
:10A75000C33062E2500005C01088C0FCA30438C5B5
:10A760008424B34DCDE02B2F043C123028DE40383A
:10A77000647D1374C6374208403EF6030000C140B2
:10A780002194C83E312220022085006B84CEC8046B
:10A79000599D5316097D7F71D8C532E1463B8038FB
:10A7A000133040C785224E5523DD0E054F4490CC13
:10A7B0001CDDBFB88B44A074125022129130970355
:10A7C00000767FF74C17DF8445CE98F2D949140202
:10A7D000C42012513222C900048C4A3B4BFC800336
:10A7E000050B0051482B0E31EC502DF0DF38C8130B
:10A7F000ECCCD8513D300451FBC73EF37F0CD00C5C
:10A80000441348AD7056390C51844E584488A18089
:10A8100095BCF0B3D5888A3E23E6D7ABAA0A704D23
:10A82000A47E7C81BC8D8CB0AA39887309504E5BA4
:10A830000CDF98EA2DBE0AFC4DA459A4AA0A582997
:10A84000A48A41A4CC57980647662F022762130AB0
:10A85000AEFCCA7004B00A8AB0CA70E5A47CE21FDC
:10A86000F6B362BF62ABF62BF61BF67F0C5B980A61
:10A87000468D8C59A498AA58081304B00A7C060F78
:10A88000662F02EF62DBF5A8B0AA70E5A4EA987023
:10A890001CA18C98622362626E6258B06A775582FE
:10A8A00046FC708A980A29A4BD8C6ADB20B07038F7
:10A8B0009C5898700E388E8E1CB63FB6DCDCDB02DE
:10A8C0007B4AF01C6A101C02BBA666700A4EF09808
:10A8D0007CAA698C70389C98F0467078A6682E66C1
:10A8E0000DBA6670EEF0EEC34670781C10701C0A4C
:10A8F00038E039883E37FEFEFEB183980A7CAA69AB
:10A900008CFC4DA4AA58B00A4DA4AA0A70E5A47CF8
:10A9100022DDAFE078E64E30C058708370383E9349
:10A920001CEA277CEA2371841B5584C606B0666F37
:10A93000E07EEEA0FEDC58B098701CB0FC6A6F7C24
:10A94000705584DE7985AB00000000000000000037
:10A950000000000000B0702E70380E3B55849870D7
:10A960002E58AEF0E07858EE8B1598EE810A4CEF39
:10A970000C27D588671CB1182BCCC3A918AEBC30E6
:10A9800076767627D588437AFA851406DA1A300661
:10A99000098366E64670787066BCFA38D884D8F0C9
:10A9A000BA3A301C62027CA23C0E3A300A7E27EE94
:10A9B000EECBEE3C7066EEAEF0EEBC663FEEAEDC8B
:10A9C000901C3B3C2606467078A6681C02C4BD8CD1
:10A9D00009B81D02B8463C584484B0E06259A66EDE
:10A9E000E0C461A4CAD844D885A43C0AED1ACCA01E
:10A9F000D5886A66A08CE746E000000000000000F1
:10AA0000386B3823380338E338C338A338FCE00008
:10AA100038E038933873385338333893387CE03C17
:10AA2000E07CE07CE03CE086EA667038CAE086E6DE
:10AA3000667038C64B42EAEAEA22E2E61FC61BC647
:10AA4000360A1B261B62620A707C3020FCE0AAC317
:10AA50007CD80CE92F758879A085140CCD071902D4
:10AA60007CD80CD12F758841A4F80C83E6DDA9654C
:10AA7000504C1346261366E8DD8CFBE61F26E8657E
:10AA8000144C1938655026E8E55C75067858EE8751
:10AA9000CC1F41A4A1A48584CDA8884E66480B157F
:10AAA000981CEE1B0C7B810AAE668F840C731B888E
:10AAB0004E704C47CCC98F41A4F8CD84E844B044D3
:10AAC00070198C4C27B066CB95A47CAAFC61A47C41
:10AAD0000A4CA9A76550E62398ADA01D0245BC11FC
:10AAE0000C711C2DA84CAFE0390C0860BC580CA0B0
:10AAF0000498DDD83BA188B030C570CC1F4C1B79C1
:10AB0000A055C42DA87BAA0A584888F5A898AA5829
:10AB1000334E59A48D8C986ACFE0AA8A700A7C3093
:10AB200083FCE0AE1C8A700E7C3080B31DA44BCC3D
:10AB30003F4E70F84666E8467038AA0ACC57E213D2
:10AB400022E21322E2132228E04CC98259A49DA4D8
:10AB5000AA0A29A4AA5839883E5F488C337EFEFE93
:10AB6000FEE3B0E098EE4DA4E5A41C6A4F06E64E65
:10AB70007005BC95BCCE581C0A59A43988FCEE98C7
:10AB80007C1D88EE7CEE6A461746363606277676BA
:10AB900013266A698C980A84F5AA584A174A4A23E8
:10ABA000666262E6E6E6E61322CA101C0A986D8C1D
:10ABB00098E0B9844C1187AE41A444F8E633E5A887
:10ABC0004C3748655026E8DD8E30DADADAEEEEE012
:10ABD000B02BB03A707A258CF3B02BB03A707A254E
:10ABE0008CA3B02BB03A707A258C53B02BB03A704E
:10ABF0007A258C3A3A3A7CEEEEE0B0703C467CE046
:10AC000066BC1C3A3076F6E7E23FEAC3666AAF03F9
:10AC1000222222227B9C229F224F3A3A301C22275A
:10AC20004E4C7F488EA9186EBCCB3A3066AF7A7A0C
:10AC30003C1CE044448641A4CC3FC6BC584C1B4D50
:10AC4000A4E5A47C82E2DFE237E2AFE223DDAC934D
:10AC5000F68384763CAEBC9C98161C66673C0E2935
:10AC6000A48C29A54E70AAE03C0EBB59A4A3E2E730
:10AC700036C736C739883EA74C2FED1848234C3BC2
:10AC800041A44DA4DD8C4E70E0E5A4884B7D9C98DA
:10AC9000CCBF4CAF4C9BCB5C42EE2B0E4E701C4A93
:10ACA00033AA7C8E8ED33C58681598EE9B0C1FC43B
:10ACB000934C7B8CA758B8E683B85898BC30E64BC9
:10ACC000E0C81C0A1DA4A37D9C8411007EFE4B8D50
:10ACD00008063064069B8D901C0AB8E6B38A636A46
:10ACE0008686A644D190EE60810A4670CC2FB85873
:10ACF0004C83B80A38AAFC0EF8FCAAE8AE0930ABBF
:10AD0000EA0130091E04CC7F4C6F06984C8D900CE4
:10AD1000870ABD8CC102CC330A0238BC3A30A6B6D1
:10AD20003A30FCE64738AACA0C4B8A3B384AD3086B
:10AD3000EE41A43DA43DA4AA0A559CEE530C3BEA67
:10AD400049A4E5A4D6E63342EAEAEA22E2E697C657
:10AD5000EAAD3CD86A8C8346425366985846704B9D
:10AD6000C63673A2A2B3AA62620DA48308AD3C8466
:10AD7000D8064891900AD8662702331B061B04AAFE
:10AD8000464223666262E6E6E6E61322CAE641A48C
:10AD9000EDA47CC63CFAFE8D8C59A4CE7C8D8CE54E
:10ADA000A4D8840C1388D88D8C980A7596190856E7
:10ADB000A08A16CCC3468B02A6588C3B84980638D2
:10ADC0004A4B0638AACA237D900A499646BBEAEA4E
:10ADD000868638E2AAE2270DA48B462222421B6611
:10ADE00053A2A23B047D905841A470986627023379
:10ADF0001B061B08AA0DA45697E6567FE68AB0AA42
:10AE00000C1322EAEAEAE63C8D8C9825961C903CCD
:10AE10001E98EE6A21B0001CF61B101CEEEA3CEAFC
:10AE200023BE2F7B3CEAF358845C4E7050FADA9CC8
:10AE300030583A30E6575CDA22A3E5E200D0881CAD
:10AE40003A308C97E63A30C61FE663E60EBC427C89
:10AE5000A67CCA70BCA6F6F6F6A33A3A0E303C1EA3
:10AE600078AE7E3A3A306A677E8E8EFE2F4A2F4445
:10AE7000E34A97BC631C06461F4EE030DF0647C618
:10AE80003C020ABC059AA6FCCA221C70BC0E98AEF5
:10AE90007A30EA8304D88C1B8408D86A3F8E8E0CE3
:10AEA0004F4A777C8C173C019A4ACF48B09C108C53
:10AEB0009F0E3C7A7AFAFAFADAFAFA9C98FAFA9C35
:10AEC000901CAA08E0781C101C0A70383CE6359AE1
:10AED000D5883ED37C62588ACAFCCA0E4DA459A4B8
:10AEE00098EE6E6E1CE5A46E1C6A578E8E986258A2
:10AEF000E24B4A871CCE7C0ABCA34ACF4670CE7C6C
:10AF00000444E0441CCC1F4C3BF80E38AA7CEAEB0E
:10AF1000C8E247C4EAEAEAE66FC628AE4A7CE8F827
:10AF20004666E8890AC6369B4E7048D3C44CA0F8E2
:10AF300046E8CC5795A43C0AED184435BEA918DB69
:10AF400036AF335836C7369903CC1F4CA349A43DBE
:10AF5000A41DB43C3E6B980E4670110C1B19088C56
:10AF600060D91CB8492676C321067858EE319EB8C0
:10AF7000AAA81598EEA19268B806FDBCEE3BB80EE3
:10AF80000801AC1B95BCB806EEEE787CEE0CFF78A1
:10AF9000AE3CEE1C4DA459A4C1A46E1C6AA06E1C4C
:10AFA00058EE8D8C1C98EAA0AE4670855201AC0C10
:10AFB000604ECAFCAA3C7EEE1DA0EE3F706E85502E
:10AFC0000982705838EEF0982606C3E08E85506EE0
:10AFD0000801AE41A4CC2F46CA4602B8AAA8E08C0C
:10AFE0009F061CC3300B0604B898A8A63CB0FC1CF6
:10AFF0001086BC5C221B29CA30E6D3E000000000AA
:10B00000382338F338C3389338633833387CCA3C34
:10B01000B3FCCA7C933CCA7C737CCA3C537CCAFC9C
:10B02000333CCA7C13CAF01CE03CEA7C23D588225E
:10B030003803389338633833380338D338A3730070
:10B04000385B3833381B38EB38BB388B387CEA3CFC
:10B05000EB7CC2D63CF0AA0A6E701C1BFCEA7C7327
:10B060003CEA7C537CEA3C337CEAFC13EACA47F0B6
:10B07000983EAE4670E011A0EED3A5A461A47C1D5D
:10B0800088E6132E698C980A3C1C2376DCDC76E378
:10B090004E70786E682E70E638E66670E6F0E6264A
:10B0A00066A7E6AEF04EAAAE38AEF09870384AF019
:10B0B00098A9A6980A4329A44685A47E58FEC74CA1
:10B0C00013C809824E1C70786E700638EE2F30C09F
:10B0D00006A04EE0CC8795A43C0AB18C41AA2DA8CD
:10B0E000669FE68BE841A4CC2FA1A4D84A2709503B
:10B0F0001B29A4EDA47CC4483BFCCAAED851ACD8F3
:10B100008AAE06B7662F02976A833CC9AABC08308C
:10B110007A76EF3C7E45AAA3583C0A4DA4EDA49C48
:10B12000D08D8C98E041A4AAD8A1803C1BD588D8AA
:10B13000063F6660021F62607C8ACAFCD83E67D800
:10B140003CCA7CD8447EFEFE1348E6170A4ED8E07F
:10B150004E70381CCC17E20AE01CAEE6BD9E5A26A3
:10B160008F263B301D7C44D1026666FC084DA8C585
:10B170000278101C0A703988E62709503BD5883EB2
:10B180006F4DA4E5A47CE21FF6D3B06ADB11A0EEFC
:10B1900009829C101C3020F0B070660A38D88408F0
:10B1A000D8F04E70786668C4B18C0180BD9CC10235
:10B1B000CC53AE0EBC30E04DA459A4AA0A707C302A
:10B1C00021FCE0C6C2A0BB1CCCB76262627186CC17
:10B1D0008F1C23A237A2A22FA2E0A2A2A2A2A2AEFB
:10B1E000E06EE0469C5845A4AE58707C9C98E61CE6
:10B1F0003084FCE0C98C8ECE5C581E99A49EFE5B08
:10B200003E3EBBF5A891A4CDA883FE95AAFEF75CAF
:10B21000224BFC261CE2CF8D8C8B22A70422170820
:10B220008DA4300F0C2391A453F5A82691A48DA4CE
:10B23000CDA841A459A49DA4698C7C698C0C63FCA5
:10B2400061A40A4DA4DD8CF846E8C502FEFE37CEA7
:10B25000DC95A4BB5C62439CE2B790FC5DAA628370
:10B260009CE26FD0BB8DA4FEFE33FC261CE20FD007
:10B270001DA45378EEA091A478CECE68C330F0AE72
:10B2800058782366CECEEEE798AEE0F8261F66E04B
:10B29000044E6EA05CE070CCA795A40C133C52D871
:10B2A0004A431BD5883E33E6DF09503359A4E5A451
:10B2B0007CC4488AD80EB0CA70AED851ACD832AE71
:10B2C000724B06AF662F028F627BAEE3A9184EAABF
:10B2D00058AA0C41A4B0AAD80E442BE5A84C3F7242
:10B2E00098121B0ABFAE707C066550A01C4C60A66D
:10B2F000E8B00ADD8CF8E0C41BC488CC27E5A403C1
:10B30000AABC3A30F6EB3A3076EF7A76E11B488CFD
:10B31000A91A7ABBA24BAA626266700A387CA27C28
:10B3200082E2FB2222A0F62BF61BF64FEACA8DAC76
:10B3300082E25322223BF6ABF69BF68B29A43CCA51
:10B34000E0E2EBE2FF36EF36DF8C258F8DAC8DAC83
:10B350002237484C6029A429A48C173988ED1AE2B9
:10B360008B8DACA253AA101C66700A38FCE0A27C3C
:10B37000E0E22FF66051AE7660EA8DACEA76DB0350
:10B3800004781C10581CFCCAEE30BF26AED8666B81
:10B39000D8AE7070383E437E1E1C6A237C6AE74A32
:10B3A0007F1C8A8AA6B63CCA087C7E137CF03B0CC4
:10B3B000234A3CB33CD84670D8E0B083D813AEFCE7
:10B3C000EE707C1C0A3988E6CBD5883EDBFCAA0EE1
:10B3D000584DA4E5A48A1CDA7C0AFC6AB74A574691
:10B3E0001CDA707C0EB0EE730C33466E8D8C3B987D
:10B3F00008231C980A7C8B3020061CF86AF3B8E0FE
:10B400007F61626364650060060405010C1D7E0DAA
:10B410004EF05C90308C3C0EE5A41CEA5730051CC5
:10B42000426AB7C1B06B3CC1B0E02B6E30051C4224
:10B430006A9F9E301F0C23E8BE3726BE1FE8EBE054
:10B4400020DE6DBA5E270C71B049241CE5A43C8E49
:10B45000D91C7C5675B0AB3080A330C08B0616303B
:10B460003A66AB302C66A3302E66F7304006B8D86B
:10B470004C5F8C4FD8DC101EDE7E3353D8E8302072
:10B48000DE237EBE7E70E8E0163020069730600630
:10B4900073A6D844D806B03070A646A0061B4E5CF2
:10B4A00090101C30663322E3303A5B3C56363B0E3C
:10B4B00041A4C1A41C426A60FC5C021DB48E9C586D
:10B4C00006164670307F66851DCE0E1C7C66DD8FAD
:10B4D000FC0E1DB48E9C58467051B473E0200C6075
:10B4E0004C3FC8CC37486D00CC603080E666FBE04E
:10B4F00030107030FDF09C4ADC909C905C901C9069
:10B50000282828E049246E1CCCE5A66EC9A6381C64
:10B510003CEA6D591C387C0EF87C0AAE28B87C0ACF
:10B52000AEE8787C0AAEA8AE9C9868E0E6251CE6FA
:10B5300056069C58B87CD804D83CA8F6F62F468707
:10B540008CE70C23300BE08C273077E03087E0303D
:10B550001C66273054E09D580CC92289BA84B898DB
:10B56000A82B88B898A80CA78CAB307F069C98E6CF
:10B570008D2666AF652083B83CD808D87CA8D92032
:10B580007924BD2025241D0239B478FE37FED91C4C
:10B59000B81B09B8469875B031B8638C41BB41A45B
:10B5A000198C4E70D92041A41E8EE5A41CEA2B6E86
:10B5B0008DA41E46700C1B29B8E05CA078A0FE7B11
:10B5C0009E60FEDE7E5B8C4BFE301A31B8B37E602F
:10B5D000FEE0D4577822AF145762DC5058D4A099BB
:10B5E000A4130C778CC37EB77EA7C314B794A70CA3
:10B5F000931CA0301B31B878F65329B83BA08DA41A
:10B60000042BA08DA4088D141D02301C9C5899A6F3
:10B61000307F66937846977EFE2F410CBD8AAE8DB3
:10B620008C29A44670AE68633E236520E3AE99A4DE
:10B63000BE008B1E41A459A4BE1EFC1CD08D8C7E66
:10B640000723781E9ED91C5EA0BEB8E3301FE830E9
:10B6500020DE7E6F1E3E5E23E8BEE346F07068E0AB
:10B660005ED3B8580C373CD888D87CA8469C98063E
:10B67000307F667F781CEA3FDC10FED91C1B09B8BE
:10B6800061B6851CDC10FEC1B051B6C98C9C9870A7
:10B6900041A41E30F19C5899A4B09C5899A4AE7E48
:10B6A0006815BA4E705C105CD0100EB8B03C06FA4B
:10B6B000FA7C4638BCA606583C28E0E6174E7009CE
:10B6C000503344A180AA70040A4DA4EDA4D80C27DD
:10B6D00004D8330804D88D8CB00E3988E603D58899
:10B6E0003ED7AA0A704DA40CEB08EDA47CA24BAA8D
:10B6F000626266700A387CA27C82E297E2EFE277AF
:10B70000E263DDAC4BB0E60F700C4B41A44E70E829
:10B7100028DD8CB8584CA0D5885FE27FE217365FF1
:10B72000364F59A4E5A47C22D7E38DAC0BEDA47C65
:10B73000563C8D8CE5A41C4AEECE8D8CCE7C63E508
:10B74000A41C4AEECE8D8CCE7C1BA6FC586E1DB47C
:10B750001C980120C3AEBCD91C0C733A3A3006A623
:10B760003C2EEEB9BC04D5124D140912D91CB9BC3B
:10B77000CE3C061EA114B81CD0E8661EA11463A618
:10B78000EE1C1084101C421F02889C1BDCDCB6EBF4
:10B79000E6161FDCD64E94602213E2B6F30EF88C48
:10B7A00017B858B0E0EE2798022398AE4EF0E0CEDE
:10B7B00070989801207B0C3FB858B0AEBCE06E4D3D
:10B7C0009CCE0592810A4404040C4745A4E5A45983
:10B7D000A42B6E2DB46E66E66ED91C4CD9B0D9126E
:10B7E0000C23EE58EE04D80C23080408D8E0BD1C46
:10B7F00018120F0D20E000000000000000000CB93E
:10B8000062204038238038C4F800C4039D1033D42C
:10B8100010D0CC0C0011802C2E122151C04411717B
:10B820003333809043A21A1F0035802093C1477F95
:10B8300020C4A3612032E2CCA3C838491C524981FC
:10B84000304443C8C64304224B1204F1EB003038A5
:10B850008431000000A00091869B8CE3321070D0F0
:10B860002A8348F420B806B3F836E2C90F0A92805A
:10B870003D86330033E3C94D03DC50C1832303000D
:10B88000440400300C00C07C373B280C0A5359CCD0
:10B890008A6892C4BDCC0431BD4C0C0E04E2A07881
:10B8A00038E00326143003DA203E180470483C4B7D
:10B8B00040E000002920CD9C84FC92EE2E4F87C0F2
:10B8C000804CE14430D00F461263E483E0384E10E0
:10B8D00086E1330334141258D131B2348A104D400A
:10B8E00004C0A0A20894D3206A153E053D0BE132A6
:10B8F0002138FCD7913944E6109943648E7A557209
:10B90000B4EBE27EAA2FAEEF8804E9AB701248C414
:10B91000C87675C4BED2C4D03CC8E4E8E2E1121ACD
:10B920003180CB4E02C258F8F06F8E0808A57D6DAD
:10B9300041C308EA1433A4015FE083F2604382004C
:10B94000C02C50CE0743710E6E4C8FF7C40C0D0601
:10B95000211895C54C4851A37B8DCE8DD7D40C139F
:10B960008A5A851332020C836C3854C8030C2CDEBF
:10B97000D1C404F37FC49C46D74D41334CCC3C0F1B
:10B980006195D01805C2D2A0C47A84C1E3121ECD3D
:10B990004EB838910C51A57DA23EBE8C3DD2704F61
:10B9A00060813B152E2DF67C3C70BC08A456179484
:10B9B000824F240AE00A40330108CF23F240F808FE
:10B9C000BA08D92008553CE038ECA8FA0C5021C43C
:10B9D000722208C7805E0808CFE1608E388E16623A
:10B9E0000B622F880833C20F01E7A0080328232227
:10B9F0006060FE084B0087B8C3913F2759227B0047
:10BA00000400008C00444400C820CB0DC4CC8C281A
:10BA1000C404008C0C4AFA0011110088093E06404B
:10BA200088508FEFB82BA0880F0260824D3180B90B
:10BA300008E01A12CF000522EE0741338C3C00418A
:10BA4000F0F3DFD43ACAD5C843078D40F3F3004979
:10BA5000515BECD038508380486C28C91C1132806F
:10BA60008C2CCE8CC094688C8B3B003040FD0C49F4
:10BA7000520D500D40145D55373324C34902C3188D
:10BA80004A4C50D8821B6449133184331103820419
:10BA9000D0C03C09CC4B0EE0394F8EBBB33EBE0745
:10BAA00049EFF1E22100414403880F230F051024E0
:10BAB000F3F30F015540C544CD03013C13FC0C4882
:10BAC000E4EEAE11E1816ADC861EE11086D2ED2340
:10BAD0008788181116CF704444301ADC878313B856
:10BAE0004C01847421983DCDF02034C9E0868D014D
:10BAF000008580438D30C40C208103604861F4FFD1
:10BB0000000000004C71B204FCE0180143C461BCA9
:10BB100013D30422336110447C7C4CF4217B0C1F32
:10BB200042FCC4C470D7F14CCCE3313821E310306F
:10BB300081F11008040CC2DEF228DFF9611C20300C
:10BB4000D50148E23A7B1D76D411D30434F777351A
:10BB500000B1C4714C2C48F0C74F128D33C2FD0D9B
:10BB60003131A0301310B1108010200B030A302A9D
:10BB70000A3204AC608A38CC3C23C2CC4C800A32F6
:10BB8000C1141333F18E22020C2222327131E443AC
:10BB90006ACCF771203937EBFCD4DF4C312DCE1055
:10BBA00032CE880C41CC30830236DF5B91D1B8C1F4
:10BBB000E4008D3C4D0F140E4A4C2007AA71DB5156
:10BBC0001DA342A0C3FB102632B21ACA083200BC21
:10BBD0000C008F0002D0805EC834233310F30F7343
:10BBE000DB2E0DDFCFF152F7D84B123A30000FC5E4
:10BBF0003043CBC810240C3341B4E43F000E004066
:10BC0000193F0097013B01C60A430AD2057C01D2C5
:10BC100001520A19008809B409AC0D5B0D630C16BA
:10BC2000016907F7037206B20E6205730E3606ACA1
:10BC3000080B0A7B0A85010303AF02B5068600B133
:10BC40000DE403490F530F5B0EC30EBA062D085FB8
:10BC50000E690E2F08050F2C0F350173035703C013
:10BC60000C0400AC009D03B809A300E306A20B2F4F
:10BC70000AFC00F7012001290132023C02CE066CC9
:10BC800000009319050B0C030B8045628432200ED3
:10BC90000306201418052D8D0F0F1213010B80556C
:10BCA0006A8E0306201418052018032D851A09131F
:10BCB0001001C870F868385C581C0E38AA28B044C7
:10BCC0005D5C385CD8284C9B5D1CCC274C09820DF0
:10BCD000FC0E0F20120F0F0DF1FE80BD6A981209A5
:10BCE000040D0581408001620DFC04151020060C36
:10BCF000F1FEBF0705124E78BC067CC6007DC68EDD
:10BD0000130110A9D09868F8F67B0DFC0B051903F8
:10BD10000F0405D9FE009D0E809D66BF0E0E3D18D6
:10BD20000B802D4ABF0E0E4D180B805D4ABF0E0EC4
:10BD30003C180B808D4A870E050C01F9C41379C499
:10BD40000C1B06434E3005EA6DCC66A606E0980F44
:10BD5000140179C40C1B2E53468D8C9C985606F505
:10BD6000C4B94A851A09130C068889E8B08BBF0547
:10BD70001A0913C15C4E70783CC62B0E1B841E3012
:10BD8000107046F0A1144E708C60DE9C7E7E2726DB
:10BD9000D4E30A061E5C422FFAA6E30E8EE0E1C44D
:10BDA0000459A4EDA456E63F3005426AAF089C58FA
:10BDB0001C38FCAA0A7C28E04E703830081C901C05
:10BDC0000A838D150E0179C40C600B801162940FEB
:10BDD00012010B80696660B0307CDADAFC3A307CA4
:10BDE0000B00E00B00E0D05C3066603AC60E300617
:10BDF000A075227E477E59F37E19637E0D4EEDDAE3
:10BE00003CFE4E66A63A5C105C223730C6E3692ED3
:10BE1000D05C30C6D7CC2B71CC66D3550E7C1C3091
:10BE2000060E7A30EA592FA6D3CCDD0E5D1C4CDF0E
:10BE300071CC66BFE92EBF0E0E3D3C180B80714AD7
:10BE4000F80E30E82BF80E3000E6AE6150600E566A
:10BE500037300306E3AE8D080626D3E07E7E895395
:10BE600060065E46FAA056607CA647FCA62FFCA69C
:10BE7000B5A2E10A814081C866BFE6856813A36662
:10BE80003168C66687E61568D34BD05C30E613E0B0
:10BE90007CE046E098E0D91C788C2B84D8842388F9
:10BEA000D888D8F0492660A0D91C783CD888D8FC1E
:10BEB0009B81130F100B80096A0B80F96A0B802598
:10BEC0006A0B00CD9E0286C6E0BF0E0E3E180B80A8
:10BED000C54AD91C30126A5F78D88C1F881384D861
:10BEE000F06330706A63411C30186A9D7E4EF00525
:10BEF0007E78E2D3411C4CC76100D1441BC17E193E
:10BF00007EC676C3A5D00C60C6762330EE13469667
:10BF1000864686AE0E7C0A85D026E61C4E8223A677
:10BF2000A2A2A21F26E386EA02AA0AEAEAEAAACAAB
:10BF30002AE0856813E0A6062658D944E0EB5D1C8C
:10BF4000214687010C060C0312B830FF3CEEB94ABB
:10BF500087010C060F14130B80FD6600203C56066B
:10BF60009CE23BA0005D1C21463087E099050B1444
:10BF700005070B801D6681408488ED64BE58300241
:10BF800089408808AD402570BE981D608CA7FE1FB3
:10BF90000E5B0E300555703BA00EAE00D164EE89ED
:10BFA0004C690208A140257088A393100C03100B64
:10BFB00080696E9807120C030B80C162863E3C18A4
:10BFC00015C845CCB87CAA3CA845CCF5C4CEE871D0
:10BFD0001E5CE6A616E61376A6E6E6E6C6A6D4142A
:10BFE000A3E09828C488C4FD7E3E4E302C5808300B
:10BFF0004070387CE0304070387C063CA6BCF0E0F5
:10C0000059A413A63040562B3001B6166660A5D051
:10C010000CA01C4A2A704E5CAA0A7C9C4AA606F018
:10C020007C70383CA606BCF0FBAE0E7C1CAAFC0E55
:10C030003040562B3001B6167030EF06383C662380
:10C040007666471C4A2A703866F308AE0E7C1630B6
:10C050000156BF0670F038665BA6360670F038668B
:10C060001B062B1C90D0061CE076173670383C66F9
:10C070008B3001763F2BEDA45626E66630075A1327
:10C080003AC6F306E6BCE2667CE62B4E2E1CEA8539
:10C09000D04666064B66861C82A0A2A27BC666A519
:10C0A000D046A063044E70F8EECE71C8700439D04B
:10C0B00006B0BCA6700C1F08B30C60783C06B03C00
:10C0C000063C068C3BB958BC70B95A3C70E06EA077
:10C0D0005627FAA6F330030C1B6608468EAE608D19
:10C0E0000A304056A03001B616E0041308081B04BD
:10C0F000044E7038DC901010102884444E5870386C
:10C100001CFCEADCD0BEEB59A4EDA48A1CEAAB0A05
:10C11000302C6A1F48B3885E5BBE980C23AA3C1B78
:10C120007CAA581C6A3005426AF78A985E630C2B19
:10C130003C58BEC37C1C9010CB2E5F1C38FCCA7CC4
:10C14000288C6F0C0B0CA0CC23D5886A41A47B0CE7
:10C15000A0986815980EEE734C670C771C9DA47C14
:10C160000E7C0AFD1A0DFC0E010D05D9FE83051289
:10C17000140507884B8305120C031201840B80A160
:10C1800052E54C0CA0983C063C4C3B0C17060C139B
:10C19000463CA63C9C4A0EA04E2F8C7B5C628E6671
:10C1A000665C1BFAA642EB8C13BE600D544924F862
:10C1B00028AEE8B5BCFD5A064C2B48B03C06CE7CF8
:10C1C000A6FCEEB0FC061C0201D08408CEFCAA0A34
:10C1D0007CEEEDA456E6C6762697CE7C4C1F261341
:10C1E0006603047CAA0ABCC6BCEE8CC3B07CA6263F
:10C1F0005F0C4FA646BC26BC703A4BA626E6EDD097
:10C2000063FCEEE626E6EDD00C604388983CAA7C01
:10C2100058E0CE7C0698E6B07C463C70B0FC70BC22
:10C22000A63C66063CF0E09301051601130B8099CD
:10C23000568891D04E70F80E300255701BB5A2AEE4
:10C24000BCEE514C4E70783C06F8C4FE1388CEF616
:10C250001348A67C9C4AFE1348A63C583154BCEEB9
:10C260008940A808B156BF0E0E3D3E180B80A14A6A
:10C270004E75F0EE600DFC0E0F200412091605F14C
:10C28000FE8C06130F1049F0F9C40B80E6E956BD89
:10C2900056585D1CCC604C6060B03AE08D0F0F12B8
:10C2A0000D050B809D5A8215131405074433901415
:10C2B0000507480B80594200BCA8E04E0070446856
:10C2C000780605BCEE59DE785E3E683C06660401E1
:10C2D000AC0EC1B01C0C0742271D145BAE012063DD
:10C2E0000C77AEBC4D14DDAC4924E304B1BCC36E85
:10C2F0006EC9A46E085346F059A4E5A459A4046677
:10C300008E060404D91078065830301C622B30B0E9
:10C3100062275613B6D91CB8B81C101C8C3342B80F
:10C32000302DE876B63CA23C3E1E7E7E8518492420
:10C330005DBC99C844785CE291DF3084CC2766EB21
:10C34000B371CC663F785C62683DDE309366FBC8B3
:10C35000CC2FC8CC0D541C101C02784CBB426F76FD
:10C360005B6267A21C10101C021776A268C34E5CA9
:10C370006244D302FDDA3668F6F65BE2E21FF6337A
:10C3800078562268E201DAFE435CE2234830F02B63
:10C39000C1B0BD1C03011420050D101419DDAC083B
:10C3A0000170650E4E9C90CC67601B7A1F7ACB881B
:10C3B00059C8550E1CA020E2F9CFD91C7858492441
:10C3C000300501ECC27012C38700233BB313BB0DD1
:10C3D000549B8CE378068605BC95BC66866608018E
:10C3E000AC4359C85B785C42688859C851DE8CEB15
:10C3F00048C393011405070B80ED520000000000B4
:10C400009805160113883398140507843DF0B0068B
:10C410003C2606F9FBE6C622BC70067CF03DD04EF9
:10C4200070F8AE708C2F38EEB94AAEF0E048F9C41F
:10C4300046C10238467CA65849F0DDD4B0E622FC5D
:10C4400006023DD08A983C0A05CC98420C172E0A69
:10C45000F9FB4EB07C5CD070FCE090051601130B2C
:10C46000803D6A4CE57A040D7CF57A0B80694606BE
:10C470007038F61366663C1EE0D09C30583A1C3A81
:10C4800030E63A30C64FE63F5C50D0D0F19AE60E27
:10C49000BC427CA67CCA70BCA6F6F6F6E33A3A0E1D
:10C4A000303C1E78AE7E3A3A306A677E8E8EFE2F22
:10C4B0004A2F440B4A97BC430E98AE7A30EA830465
:10C4C000D88C1B8408D86A3F8E8E0C374A77BCFD07
:10C4D000E24AE748B19AE6C532308306CE3C56665A
:10C4E00037B85CE2E2E2313238FC9CA262CF1CA297
:10C4F0003C28352EE0DCA0DCF2C156A00EAE1C724A
:10C50000CD564EEB514CD1C8E653D144E0C4F57E34
:10C510007D6813BB664670385C5228A658BDE0BEE5
:10C52000EF983CA6BCBE580948EEEB86983C7038A4
:10C530000EC67066E6386E33EE773A6E5F300406EC
:10C54000983A7EB75826371568A30DFC0E0F2013B6
:10C5500015030820010C0DF1FE266F29E60948EEAF
:10C56000DB33D1C8E62B4670F828B8EE4670CEF023
:10C57000F1688E1C527C706944E86E754CA8987006
:10C5800038F6274E70AB98267038463C05688D709B
:10C59000CE0EDC52BC702626694468454098803D2A
:10C5A0006A84050B800172840C0612038443930194
:10C5B0000C0612038801C8E6B5A2DC908C133E6815
:10C5C000BDD00881F08CA1C34E70780666263DC2AE
:10C5D0005AEEAE3C700698F00DD0A6065870CEF01C
:10C5E00070088C6366700201D030FF8D8CA658985D
:10C5F0000E0DD0A65870B0662F704EF09B0C234ED7
:10C600006EF0C102847E1788B0FC580670BC9C4A4C
:10C610001CBCF004738C060C033EA5E8B07E7E2B98
:10C6200089F63E8C1B78EE55F2BDD07DF20DFC12E2
:10C63000050320140F0F200C0F0E07F1FE920803C4
:10C640001010018408B5E00CAFCEBC06B07C8C2F76
:10C65000A63C707C26E6CEFC0AEDD0AE7C0E980699
:10C66000CEBC4630FF063B3CAA8D8CB03C0698E61B
:10C6700071D8849803920803130E09884349EA830A
:10C680000512130E0904B5E00CA7B03C51D8CE3CFE
:10C690000E889826587C9C0A7C1C0AAE7098E6EDA1
:10C6A000D0B0AA7C0EEDA4AEFCAE8D8CAE7C0E7C20
:10C6B0006A93846262901C622751EC02AE8C2FFC5C
:10C6C0000E888B987C0AFC66588C9BB383051210ED
:10C6D00010014404B9E049D8987C0EFC2BEDA45914
:10C6E000A4AE7CAE8D8C01D098663758AEFCAE738C
:10C6F0004C6030FF8D8E8C061A1305120B807D4A1C
:10C700005ABC1A203C06B0303AE62366DF461AE0EF
:10C71000411CF53E30EFB616666F3001B670387CBE
:10C7200006562306B66666E09819050B1405070B36
:10C730008005427924B5BCC10208D8284E2E687005
:10C7400088C4651C0488ED0600000000000000009D
:10C7500000000000000000000000000000000000D9
:10C7600000000000000000000000000000000000C9
:10C7700000000000000000000000000000000000B9
:10C7800000000000000000000000000000000000A9
:10C790000000000000000000000000000000000099
:10C7A0000000000000000000000000000000000089
:10C7B0000000000000000000000000000000000079
:10C7C0000000000000000000000000000000000069
:10C7D0000000000000000000000000000000000059
:10C7E0000000000000000000000000000000000049
:10C7F0000000000000000000000000000000000039
:10C80000810F1418F8EECE7EFE595A15C89C58397F
:10C81000B69209040D052E009170A56CBDCC06469C
:10C82000BCA63CF0BDCC26BCF0883E4E5859F08CDE
:10C8300053C1B01C4E901A987C5875B0BAD33020B2
:10C84000E8B03000E6E6C67EE3E8B0DCD00EA11426
:10C850004924385E285DBC8001529CC22B387C661E
:10C860003B0D54663002C61306F5C44E708CB551AC
:10C87000EEE8D5CCA6A62FB5BCFD5AC1B0BD1C04B0
:10C88000091220050D101419DDAC080170B902DC85
:10C89000901BDCD0FE84480453DC501BDCD0FE042B
:10C8A00044848404040E30407030BF0638661B0890
:10C8B000634C537C66B5F7EE7CE6FCEEAE0E3CA610
:10C8C0003C263C0E0C7F7038AED86E1788D8AE2E42
:10C8D0006F8C1B6E582DD00CE7A6067038FCA60690
:10C8E0007C7026E63DD00C6F4C278C5F83CE7C6637
:10C8F00037FCEE4B84AE0E3C06704E6EF00C278C6F
:10C900006B8485D0C6A686A6A5D0469330EEA62613
:10C9100086065C424F9B880C2FB0BC16DEBCDEF353
:10C9200076E30DFC060C2014191005D9FE0DFC064B
:10C930000C200E0F1420060F150E04F1FE1C3040C3
:10C94000704C57AE0EBC06387CA6BCF00CA04E2E28
:10C95000BC30BFF0E09208030C0504884383051245
:10C960000C05048449F08808E9D48CF9FB8C7B4ED3
:10C970007001C898A658CEBC06B07CC6E698A6063C
:10C9800027C6DB0686A6467098C60658CEBCA6C645
:10C990003CAA8D8C98E63C0AEDD0987C83B07C460E
:10C9A000707C707CF0CEFC0AD9D0CE7CAA0E84EDCF
:10C9B000A4F0664BB0561C2A13886A1CF0AE7CAEFD
:10C9C0008D8C8C60A293A63040562B3001B6166633
:10C9D0002F70383C06A2A2A28CAFAEFCAE88338C7E
:10C9E00006121510A068A5E88EB05A580881F09874
:10C9F0006E46262642EA4E7078063DC3BDCC46BC44
:10CA0000F0AE0E3C0A3DD0BA3CE6A670A638EE70F9
:10CA1000EEF0DA3C66A084A63040562B3001B61604
:10CA2000661FA5D0668C27887B981205160113888F
:10CA30003B9812140507843DF0B0588891D0B00699
:10CA40003CC61306BCA606BCD870E63C4626832628
:10CA5000E698A658B0FCA61C223DD098EEDB9214B6
:10CA60000507843B920516011388DC90FE95E8C10A
:10CA70005C4E70783CC6A660E6B006978C730DFCE1
:10CA8000050E04200F0620060CF1FE66A6C686BC25
:10CA9000A6BCFAB0FC060DD07AB0FC70BCC626BCB1
:10CAA000F0AE7084448C57A67CA63CA6700488B374
:10CAB00008849B90011713070512484B85160F0D2C
:10CAC000070512448491D0E6136670063C063C06C6
:10CAD000B958BCB958063C0627883C70B00E3CA635
:10CAE000BCA670840404B07C7038EEB07038EEF0F0
:10CAF0004C33B07C70CEF0B03C66603C048C7F8CD4
:10CB00001B661326700C600CEF3C080C9B700E2DFE
:10CB1000D0B0A68BAE7C0EB0E622FC06023DD08AD9
:10CB2000AE0E3C0A05CE94100B050513844B811400
:10CB3000100B0505138889E84E7001C8FCFA1E7EAB
:10CB40007EB0FC70BCA6063C463C7080C15A941076
:10CB50000C031284438114100C03128889E8B03C42
:10CB6000A6F5C4CEF07C06F5C46EA05A233003C6E9
:10CB7000B01D60EEB94ABD1C20051212DDAC0801E3
:10CB800070ED8AA188C1B0BD1E492404CDB4734E96
:10CB90005C90D0D010309C6262BDC06B49A43DA4B3
:10CBA0008A3DA4E5A4581C22071CAA588CDF6AED14
:10CBB0001898EA6DCC3010701EA114D91C7E9EBE50
:10CBC000B8BEF37EBAFC8518F90E46F070B85CE288
:10CBD000E2E24660E21BAE4BAEBC067CA63CA63C45
:10CBE0005EE0000000000000000000000000000007
:10CBF000000000000000000000000004320605E80C
:10CC00000000000000000000000000000000000024
:10CC10000000000000000000000000000000000014
:10CC2000000054000000009001000000042AD08899
:10CC300022282280008051018045028001C05504D5
:10CC4000C02422006024110054005001400500243B
:10CC50000204100D2002C05000000C0C00E0344F04
:10CC6000C8834F8A4F3C372C8E20C13B08E16810A7
:10CC70000D204E064065F3B8144DBFF48308922290
:10CC80000159C91D744FCC78E4452FC2F1020054FC
:10CC9000D450C1D8C430FD3A06FE876130164E41EB
:10CCA0008660434BC43D898BBBD1D3BB031011516C
:10CCB000D100034035312DE212133131D5C172500C
:10CCC00031E04C0005D10444151E50455D4C762FD3
:10CCD00003005C000000194207C9C4004066021648
:10CCE000F6460522501012B4CD460A001900740011
:10CCF000318F4F40384454F37F2B4147888714E0ED
:10CD00004331410F3C4A349009941140314166301F
:10CD1000CD2823514ECA60CAC01F8FC2E72F080119
:10CD2000B60501C2C8105D07FC2210301100FB04DB
:10CD30002244448C738748E0C4073D03A3064AA4F9
:10CD400080C1084B31C1142013044B03D60F1B02C2
:10CD5000023D0CC1E724E20051086000800000524F
:10CD6000D147842000923374CDFD6405C1111104B4
:10CD70000004F04020800661761402C404640012AE
:10CD80000012EE450D0511A0803900102148410028
:10CD90005238B18C40225015F70500549C0B0060AE
:10CDA0000020409A25CE660040050002205D3EA985
:10CDB0002686E8B534D00C004033C14149C223A3D4
:10CDC0007463C71333CDEFD27188521027BAD2E300
:10CDD000C4B84EF9F3B5A78448F623C2BAA24521D8
:10CDE000A28D6CF63300004E32C884B83260301D1C
:10CDF0000100104CE98608B7203B2AE10E0019001B
:10CE00000008804278001A0A820280078F442200BC
:10CE1000215410E1417004001D65155D2275F3B8C1
:10CE2000E322C140244354689FA88F2F638F854B12
:10CE30008B3D1F4FBCA244C05C357A9F2B0896D413
:10CE4000C515724F45A1214505910921A130E24444
:10CE500029BD290000603C981F8E04884668819196
:10CE6000089282470BA9C55401110002008620A236
:10CE7000833C683D40964089240204500189800724
:10CE80003A8A500A640200E8C0A48C0800006000DE
:10CE900080C1612444020555582C00146001800EA5
:10CEA00000040F80996110440009001073CD003C0C
:10CEB0007D840900500011C8000049C01D000074A5
:10CEC00094D4CA63114113480DD4000051DC70980A
:10CED0001913000000000000000000000000000026
:10CEE0000000000000000000000000000000000042
:10CEF0000000000000000000000000000000000032
:10CF000000804A0C00404613912302090D54171D5E
:10CF100053B58F34215E94A01611043630C5D10C60
:10CF20000080938C20000802F01246CC800200148E
:10CF3000482734878189904020227082815389025A
:10CF400031057041D43D5124230060080000601079
:10CF50000215828F8403800080427218468451C477
:10CF60004820514800511110204241B420B02C00FB
:10CF7000F0514CD008550B3C00094048A4803E03BA
:10CF800052098180487F314103FC038000A0104298
:10CF90000451019D4400480420002800E0D43022C0
:10CFA00000008640040480620208117C1F0000001B
:10CFB0000088488851C41004C14B02824022380CBA
:10CFC0008838C693C014400854000003000C184071
:10CFD00081124404C000C0000454E0440030809337
:10CFE000CCCC4406F5BF5A318CBC41400484CC40C3
:10CFF0003708C25EF501D4080C00000000000040B4
:10D000001A24005D0B6E08060F380B670B5F02D702
:10D0100002E202EA02F306340407010002C102C878
:10D0200001790089016E0122011701350B010423EA
:10D03000040F0B440CE5056009FB00EE09410054A8
:10D04000006902D0007A007100610000850D0914AA
:10D050002018032D83322020050D09142D9410175C
:10D0600013C5DA810D0C010C0341E68D0C010C0394
:10D070001289E6930D0C01120C03C9CE00000000CA
:10D08000000000000000970F0404A140F944694823
:10D0900063C1B0981E7E3570DDAC6564983102586E
:10D0A000300370C158CE6152814084D54CF88C1346
:10D0B000B86ED330200C3330188C1326E6A18804C8
:10D0C000B17022D91CB8C6E86564ED8A389C4AE084
:10D0D0003E3E3E8A1E4E62EFCECAD47EC31E4EAA8C
:10D0E000E05830107030FBF0E8E0850D0914D96885
:10D0F0008E7C5E61446948BB6ED9708B85140104D7
:10D10000D968754C694843C1B008F548656498EE24
:10D11000B94A97130C0312514C04E5449B86010C49
:10D12000031295445B514CF8BC6944FEA0DC50E00E
:10D1300097130E1512514C68E08940A838A0FE1BC9
:10D140005C8A0E9E1EB1644E46D95C5C19688D7077
:10D15000CE0E5C7CEACED95C5C4AFA1F4E5BA00E18
:10D16000665C1BFAA642EBAE0E60E099040DB8BCFB
:10D17000D844D87CA8E0990D04B8BCD848AB0E8E32
:10D180008EA04E5C504E4E9C3E3ED05C4140603C7A
:10D19000E00408E0DCA046F098067038F6136666F6
:10D1A0003C7E60BCA6BCDC100EC1B0AE5C900E46EE
:10D1B000F03C70380C435C04F2277CA2E370D91C6D
:10D1C0008EB07C7075B06E8E5E4B5CA2A39CA2AFDD
:10D1D0007AD30CE361009CD2BB9CD2A0C1B0DC101E
:10D1E000FE04041B300B3C0E1CF86A1FBEE3B8495A
:10D1F000243E616A856869547008A968E60670383B
:10D200001CFC6A6A1E6A337E7E98A658B08148ED7F
:10D210004E6954BE3E0165DB000045DA00000000A7
:10D2200000006954F693E0DCA01CEE982670380EDE
:10D23000A0F2A65EEBA6728940387C323200003242
:10D240001F12EF662792B2939260981D68A6049809
:10D2500070CE1C42F0861E81487E98C6BE6066EB8A
:10D26000F613263C5E9E9870380C134E7098532629
:10D270007038A670A6F066A60626AFC670B0F0BEDF
:10D2800033E0300870A6DCD09C1E387C4A3CEE604F
:10D29000A6BE60A6067038BB8940387C4666E6A606
:10D2A000260E4B361CE2172AA6496870383E607E6F
:10D2B0001C128B1C42F0935C0A6029FEAB05140122
:10D2C00004D9CE93190104048DCE980D0C010C03E2
:10D2D00011E6B2310B0C03DD48449828E0B4320B60
:10D2E0000C03DD4848AB940B0C03DD48846B8414BD
:10D2F0000B0C03DD488823514CAD72754C46178EDC
:10D3000030020C6BE01CA01C50509C30057217665C
:10D31000884884DD6C0C0BDDAC4E30200EB8B8B8FC
:10D32000662F7EB86623D888D8E8492438D91C9C53
:10D330004A9EF9447E3570492659CA85683389402A
:10D340004EA8E0454A93000099CA08C1B04944007C
:10D35000B9620058894068F858A8B80E4EA07A60A3
:10D360006E1F8CA0A84E2828A82828E8E828E8A83E
:10D370002828E8A8E04970136BDD48A00E3CAA7C81
:10D38000C6A670663004062B301246BA9A4EA6BC6A
:10D3900001700EB01A9A70DAA5709A7C2B816CA07D
:10D3A0000E0E4924389C0AAE284A7C0E4E5C50D0A2
:10D3B00010101090504E5CD0905090DC4140AEBCAC
:10D3C0000E389C4ABC70BAA57070BC0E4E1CD010B2
:10D3D000903A5C49404E5C100E2BCE7A1A23AE7CFC
:10D3E00006B0A6705A0170BC30120EB0BA5A7A66F6
:10D3F00006237AA646FCDA3C5CAA7C0EDD48694628
:10D4000094030512120F034843850D0914051344B4
:10D410004E7D4070CD6C49503C2EFCBB8514010400
:10D420001405134E7E708140EEB5A258CD6C448435
:10D430004950704570380EB0284CD3492478AECE90
:10D440003010956078AE68CEF0AE5C4E138A0A302C
:10D450001095607858B075604E3004583A3024BC4E
:10D460004960709544A0EE1FA01B2D60B02560EEB2
:10D470003961216CC4F57C856813E061481CCAF9E8
:10D4800072E0AEBC0EA01C30120A334A2356134A77
:10D4900016E004E0DCA005688EB03E777E4970138C
:10D4A000730950EA0A4BAE3C0E1C12D1501B84ABE0
:10D4B000D8EE271CD2D3D54CB540EE4D704E1C5043
:10D4C000501C0A1BCD4290901C0AD36E816C4E0EEC
:10D4D0008D70CE4EFD50A0980EE09ED95C4D70131D
:10D4E00063D95C8A8A4B30030455701B616A8A8A4F
:10D4F0008A1ED95CA04E9C909C0A931C3C0A73A087
:10D500005C99704E5CA5700E0E60E00E695013EBD6
:10D51000D95CDE7098067C6627B00E2B6670C15809
:10D52000CED95CFE23A03E2B6E6D50234C670BD9E9
:10D530005CDEA05CFE138A0EB0FE138AAECE5E6F78
:10D540009E2146307A66FB61020404981D5C5AE114
:10D55000080698467CA6BC58E01C987038E09713E3
:10D56000783CE64EC67CC63CEE514CC4780ED1E207
:10D57000B1640E681CE260CE3C58B96C6100CCED21
:10D5800057080C7F44E544CCCFE05CB5708C171C89
:10D59000D85346F0987CB95844CECC37FE2BA03EE9
:10D5A0007E538C2B2D548B234970630460B1702201
:10D5B00008D91C495C638ECC4FE01C214CCCF55C37
:10D5C000A0CCCF6089406C9BF89CE27B4970CC1D5D
:10D5D00070CC4F89403031E8F9561CF8EA23A8385E
:10D5E0000E98BC62EBCCAFA2023C580CAF0844AE24
:10D5F000F544CC47214CE05C115C3B6046F03013B5
:10D60000716487138474348575358676363718824D
:10D61000C21283C37300230B36363636363636369F
:10D6200036134B237BFBFB6B53306E66FBF1568B43
:10D63000030F0C039170E5EE995ABB05D40D5449C4
:10D64000248142115AB95A855A0DD49170A56CA003
:10D65000F9CE73AB8C374C73195C061C62131C42F9
:10D6600062315D33D38940F81C0CFFEABF4EA82815
:10D670009B4C8FB570A88C1B281368580C2555F34C
:10D680008C178C1F883B842B4CD73032155CA08CB8
:10D690002FA6FB415E66134660315C315488E54C31
:10D6A000AB8C9F4C8F0C1F0813042D5404434C3734
:10D6B0008C370CCF08A55A044C1F481344989C4241
:10D6C0001C4258C3155C044C374666B64893367600
:10D6D000DF1C862233A24C47C62B629C86A24431B3
:10D6E0005C4CCF3154BB4C778940A838700C255521
:10D6F000987CB958B004F544987C70AEF0C8CC7BE7
:10D7000008488C2D55C8CC3BE01CF55C46F0983C95
:10D71000A02660F61348315C7C26BC588CE54D6130
:10D7200000987C26167616577038AE98F038AEF012
:10D73000986E4971F9560CA04C43C8CC60A060208B
:10D74000E0CCED57E006983C0CA03CE03C0C173CCC
:10D7500058E0302E0C1B303DE830128C1B3004E8B2
:10D76000195CD95C065E3E4C1B3E234C17E63030FC
:10D770007CB6163C761B301FE8E67EABE0A0C1B05D
:10D78000600C495CD95C6EE00C2B5E4BD43B5E13A5
:10D790001C4C135C2BE01CA05E0EC1B03E04885CE8
:10D7A000421B3EC3EAE0DCA07EBB830491704C4F79
:10D7B000D8C9705C422F3E33D8885E3EFED91C78B3
:10D7C00068786860E0EAA09C9A5E339A509C029068
:10D7D000DEDE1790D95C13D07EF3D0D0D0D0D0D07D
:10D7E000D0E0DCD08C7F0A9417904C276210135045
:10D7F00050DC0210CA683828380AAE28A046F0E08B
:10D800009401030D0C017D681B796666A65E3E5887
:10D81000C4440D54E0C170843D6404CDB47B758C68
:10D82000E06564E04871682B65644164E04544EB61
:10D83000B068CDB42BE5AC88138478703D64E065A6
:10D84000443B8CE5AD3D6413208C758DE020843322
:10D85000985E580D54214C492498FE2BCC6F1568C6
:10D860004330FFCC3766EB235162203C560630181C
:10D87000662D5A308766D3309366FBC8CC6100FBB7
:10D880004E9C90CCA7601B7A1F7ACBF55A894858DA
:10D89000C17085641385644B1C20E2B78C73E54C22
:10D8A000300671643470C28412C300133383533B57
:10D8B000DBBBD14413037966E168E09C83016442D9
:10D8C00049621B985E3E4962E54C2B3008716480CA
:10D8D0003482C2848712C300CB033B3B6333538B38
:10D8E00073EB1568E365203BF168E05CE17084410F
:10D8F00062F168C1B008ED48B3447168008B294EED
:10D900008568668698663315C84D68CBC658E02092
:10D9100030F1CC256366E3E0E008017201EE884156
:10D92000DE9870C4F57CB058E0000000A09C4ED09A
:10D9300090CEFBE0B87CD88C6089028D0C011A195E
:10D9400018300289407D4070514CE83888084D50AD
:10D950007C46EE173A70842689400EEE6B8899500B
:10D960002B301AF1424E360ECFAE7C466860094825
:10D97000B0300446068C1B66367066A658851406C1
:10D980009806678826260613848568238C97A188C5
:10D99000C1B0BD1C0E0F20120F0F0D38F8214286AA
:10D9A000C626704E7EF0C6704EDC90901090F0044B
:10D9B000A96858B0C6260E2568869806B05568989E
:10D9C000A658A670660638D87066D8F026ABC67022
:10D9D0002658B0F65BF04670780E98702658AEF078
:10D9E000B09C629F0948EE173AD87026D8F0BE3F27
:10D9F000A6667006388BD152982B148140CD6C2EC0
:10DA00005899501BB5A2A0DE1B8E0E70984E5E3347
:10DA10000ED164AE734E9C501090D05010D090AE8A
:10DA20000E874570380EB00E286B8606B05568C656
:10DA30007038FC1CAA0C2F0A3967134A7CF026A602
:10DA400004A568A6A6E0A6496870381C3E607E1250
:10DA5000B3E0067038F61366663C46FC0606E051F5
:10DA60004C4EF0E0DCA030C0085C905C0E13664EBB
:10DA70007078067BA60670383EAF7E62A0FC5646E4
:10DA8000EE770CA0A398496870383E6F98A658E0CE
:10DA9000894833D144E07EA060B03AE06954F69BF7
:10DAA000982670383C05688D70CE0EBC555CD91C2C
:10DAB000B83B4C604EBB514C894038339870384667
:10DAC0003C0E0430059C5A109010DCDCDCDCA0FA23
:10DAD0005A13229AF33A0C534C2BC8CCA023CCED0A
:10DAE000576627D4BA73945BFA5A5CD0905CFA46B6
:10DAF00026139423FA10C3FCAA0E60E086011405D5
:10DB000013514CE838288140EE8349701B4E5BDC92
:10DB100050AEFC1E1B261FE6EBBC89403CA8E8E08B
:10DB20004EDC5050501090E084E80444D828E8308F
:10DB300029E8E0EE514CE8380E4E70AE68A0E09750
:10DB400013140513417013339E048D501BB5A24D61
:10DB50004C98DE1BA08E28E0B432050D0914018418
:10DB6000887B850D091401843B8514010401888498
:10DB700044417013CBB87C1C50600691704C23D884
:10DB80008813D8492430260213A222D888D88C7B47
:10DB90008662271CEAEA0604E948E2B308A3068C79
:10DBA0004FC9705C4267DC906B095060AE3C0E134D
:10DBB000FA4C47DCD0A25D6C6E4BD91C9C10D0A2F5
:10DBC0007CE89CA2BB8C608C603020616C30414C46
:10DBD0001B3050616C304D6E5851B6B6A31C8C7F13
:10DBE000A25390909C5D6C6E167693D090BBA2CFA2
:10DBF000302F0C4B664C73B8D848D81B4C3BE84BC5
:10DC00000EEE0E0EEECEEE0EE0CE30046944A0E035
:10DC100081400E3001A0A65C4636616B7606138A01
:10DC200066F3E0A0A01CE0DCA04EB2CEEE4EEEE02B
:10DC3000F16804E09C23E09C08A0C1B0AE707C5E5B
:10DC40000EAD5C0C60D91CF8F8B00EED4A7E7C1A63
:10DC5000FA5AA57013150E0D0F0E141505170504AD
:10DC6000140815061209130114B01A30E83ABEE37D
:10DC7000E09806C44924B8BCF6F6F6A088E004C5CE
:10DC8000703059D866F31BC570301E0C1BCC8766EC
:10DC9000DB2308C570302DD80C1BCC1F66D3C458AD
:10DCA000A60658E030107030FBF0A838238940F801
:10DCB000D8E0AE8444BC0E30121C0A776A53A0CA66
:10DCC0000A374A881B563348234ADF0660AE3C0EAB
:10DCD000E00E4E7078EE894078A0AE8E0E68E09728
:10DCE00013100F1413514C28E060FCB07CA0EE0E12
:10DCF0001CD09050A636369C133AA2F38E76E3AE33
:10DD0000BC0EDA3CDAB0BA5A707A9A4E5C109C417A
:10DD100040AE3C0E3C5A4E1C50D010509010AEDA23
:10DD2000CEFC70B01AE05D1C0C13C88498A8150CCA
:10DD3000711EE1688CD972E0C97020E0894038A07A
:10DD40002E2E60E000000000000000000000000037
:10DD5000000000000000000000080B6CBB8CAB0E44
:10DD60004E70B89CA2A8B5708C1B585B4C43C1B0D8
:10DD700048042BA16C044484617604588940594CB2
:10DD800038580CC76C2F4C517EDBE8F8D84C4D76D8
:10DD9000D80C1F4CC34670B83CD80C738C674C57DA
:10DDA000D80C7BC97491704898A828E8381CEA57A9
:10DDB0008CA30568EA274E907BF83CFECFFEBF603F
:10DDC0003D5BCC4B3B4E36682B854044E804D8A8DD
:10DDD000288940BD6C88044408844484608940F8E4
:10DDE000D88C3BD83038E8FD7E0C27D8D57E5848F3
:10DDF0003031E8757A980670389C62CFF613666603
:10DE00003C1EA6067038AE7E1B4E23267038AEE050
:10DE1000DCA05CEE5D7AF237B2EEEE7CD37C0630AD
:10DE20005EA61C6A873C5CB27C0E4EB2EEEE521BC4
:10DE30003CD31CEE25510E917004E6C61CEA4BE063
:10DE400008F174A8E8557E3C305E6A478E8E8CBF20
:10DE5000CC87A3FE97C68C7F4C6FD844CCD3655437
:10DE6000D0F0F9700D7EC6A16C49240C37B8D844A7
:10DE7000D8A8AE6841683B8DE2F174A8E8CC9974EB
:10DE80005D1C0C330498A809B8BC5884983CA87849
:10DE900058EE091E44D5420C676554D0F09888BCF2
:10DEA000983C589974E020F97098BC584C93C1B0D4
:10DEB000BD1C14090D051220010C01120D20534543
:10DEC000441333C17098BC5846F06666FB610098F5
:10DED000DC1044E05830F1CCFF66EB2030264C2BB0
:10DEE00008FD7046CC9F66EB987E4B4C1F482B4834
:10DEF0008C979170A56C6B2020441C583C1C0A49DF
:10DF0000CA30C36A8B2E4C4544000D54654400460C
:10DF100066CC3766EB0D54411C4C5F9C985606301E
:10DF200072665F4CFBD57E8C6B480D7CCB4168BB29
:10DF300098E3970F0E0D0C01514C88C4084860857A
:10DF4000684B2315684389400EDB6631687038E6FC
:10DF5000463C0E8940F9740E630C474C3F8C271CDD
:10DF6000C217D5764C43F8D88C1B58E058AEA8E8B9
:10DF70003038E84C60E00C132049244CA7CC091F32
:10DF80008C8B91704C37D88C53C502603D5BC97443
:10DF9000F90C9170048498A82860A05D1C98CD9E0F
:10DFA00058B8EE514C6C9B385888989CC2285D1C20
:10DFB000089842A84B4D4C38580484D91C783C89A9
:10DFC00040A8FE63084E2B00E080E02E6889CE4C0E
:10DFD000EBA56C33587D6813DBDC90F091708CA757
:10DFE0006148D6F970736576817ED968C97071BA57
:10DFF000D57EE976008B93CBD3DB0003320D14CEB4
:10E000000000000000000000000000000000000010
:10E0100000000000000000000000000004000000FC
:10E0200000006C454C54434D613076314C4C8C4C67
:10E03000C1CC34CAAAF4BD031FC60F60481110003A
:10E0400066C4781400404503401794EB00D4DF28E1
:10E050001B505047BB402060CD3D3930B30FCCDC66
:10E060004B45DA6707C225523BE40D172330723364
:10E07000300173171992E4E3C4793F7D6055402461
:10E08000A348451455922000508E404ADEC7B14245
:10E090007CF45845324211EDE291008482183D62D1
:10E0A0001F2246E435C9C708060B94B8FC3838006F
:10E0B0000400020000C07503700D700EC07999CD88
:10E0C0002144688C43D910FDD3B31F8E505448713E
:10E0D000300DD21847374FA8C3E0129BC4139A489B
:10E0E00043315140140AA790161A425812250507C9
:10E0F00029C05104E961838D01501188137A71564A
:10E100000080008018642B00006242E4C615594864
:10E110001122B05884214406012921804253B16D57
:10E120004D79CC4C3C7220125843C53149500611F0
:10E1300036063D6474670E11D01311F643423C3E1F
:10E140005190798704E5501A90281C3EE16288F4CA
:10E1500054B848C554429F0C0388D434242344F255
:10E1600025D28109C71972A2320444064DC1405D0F
:10E170009C371CB6DD05353DD50E91263405A61C11
:10E18000040000000050AAAA5645851700069754BF
:10E19000CC998911501ED521961D5B33B72DF316EE
:10E1A0003E7719A53409564948885810C210C00452
:10E1B000914520A1BF00E353659537581944293E86
:10E1C000393D501CAA504A92A43442826DD5F227A0
:10E1D0007F17CE091D12C7C44521481C9311EF3388
:10E1E00052043033002134C623334E16DB03830C34
:10E1F0008040CF1708042E12308010011F0004F059
:10E20000005050605B1294719219441A681820E40F
:10E210008111732E51556463F4782414576CF98B73
:10E22000C8843851445398464100C080724C06D18E
:10E2300054587410000004BC600A0664D978675C06
:10E2400015CDD4F479B92790C444030AF5B70B006F
:10E250008419356F23B2967C84E1336A844D124968
:10E26000CD3A57333300601F288AA82014585154E0
:10E2700084469A8F868896862C26A619685C8051DB
:10E280001DA01835109015047F850914C2808618CA
:10E29000554C09EE9F488D763112ED113E24EE4328
:10E2A000DE5422D1C4DD6625291E6D36DF5C0709E8
:10E2B0005684F52F6017F2F3C92F10050EB0E40055
:10E2C000D4644280818877CE08D907773035213AE7
:10E2D0000004744025CA00C000C0003010CE99C5AB
:10E2E00070D4E03F4F1F1610D8239810837030036E
:10E2F0007F3CC745C405403EC11F34DE01F237FCF8
:10E3000065BD1FE556C86AC2BE84C0D5260232204C
:10E31000990FD365550000000000E4DBDF31D55FC5
:10E32000A54E458C539531BEF4617C1C0F553C6362
:10E33000134C7C428772483200D44B0852E8D43BDD
:10E34000858100E561462545102EA32F6192F48753
:10E35000EA0000000000D44C786C333009D95757DC
:10E360009D83357303E17F541319DF2C724270488B
:10E37000F5601CF11D6D0B1ECF01C13581952C522E
:10E3800047828002B226FC5FF03B073FBE930987BD
:10E3900012DA311F4E3030565B05853C8F46104AED
:10E3A00002FCF4B3398AD6461379D53003000088CD
:10E3B00001D5AC4BA6C5F82D15E3B97866D406DCBB
:10E3C000C4805107BE57C0500C94531B0100D56246
:10E3D00081719009D8D108CB7EC0F383013B4738C7
:10E3E00063304C4561FE89344D7D7F24CE57FBE47C
:10E3F0001D40B70D9315ABF6665D665456FC0B8851
:10E4000000F8615044FE1348260E7676B5A3D91C59
:10E4100078D88484D88C1326F046F009C886E64B59
:10E42000309EA62BA058F142CC2766EBA3D91C78CE
:10E4300058203C56069CE21B4EAB3012664761C822
:10E440006686A568E330C4064FC64ED0A646263C75
:10E45000A3E6761C4E906AC6FB303162276A13A68B
:10E4600062AA3C26048C2B08A07E60585D1C98BCD8
:10E470009CE22B0602A2E6C602A23003622F1C42D7
:10E48000136230088C270C237B0C134630555EFC3E
:10E4900006BC30E61BF61B2E03068C2FC16813C387
:10E4A000A60EA05A7C1AFAFAFAFA56233C3AFCEE67
:10E4B0001A46BC26260E55C4604C61008859C8789F
:10E4C00028B86898A859C4EA005ABC1AB0303AE68D
:10E4D0002366DF461AE0BDD065F04C2FA18002DB39
:10E4E000CC3F4E70B8584C7BCC6795A43C0A59A4DD
:10E4F000E5A4D88C1744A180FD188A8514064E70B7
:10E50000CA685878A6C6026A6DCCB05E3C062B5D20
:10E51000C4C830DA7004B07C0E01D0EDA4AE3C6605
:10E520007F7098AE59A48D8CAE7C6606FC5843046F
:10E53000987C1666C3084E70980E78061BA66878FD
:10E540000E59A430C08D8C4DA4468D8C4E587078D9
:10E550000E4C23C4BD8C783C667BEDA4D884D88D4A
:10E560008C29A429A4AE0E584E70780EB8BC5884DD
:10E57000E0DCA0DC1050121C8AE5A43C5CF2CB7EEF
:10E580000F02FF1C8A4DA4EDA47C6A22D398AA69CD
:10E590008C0A588C574DA459A4468D8C980A29A4EE
:10E5A0001B1C6AF5A89B623C5888821B59A4468DA7
:10E5B0008C42D762101C021F023BA666700A4EF006
:10E5C00098AA698C7038989C50F09806467078A686
:10E5D000682E063B6670EEF0EECB4924F85A5EE8F2
:10E5E00030BF2684A80E78AE66CB70380E4670AE6B
:10E5F0003E8B1C8C137CEA330EFDBC95BCB88C1F83
:10E60000884B781C0A29A429A4B8AAA8A1801C397F
:10E6100088E68F0C2F59C4F0000DFC03080B13156E
:10E620000DD9FED5883E434670AA680A4DA4E5A4DC
:10E63000AA704670785816468386FDBCEE4B66B8C5
:10E64000FCEE0825AC1B95BC780EE3D1486E2B5927
:10E65000C42E1659C41916D1486ECFA3D1489D486F
:10E66000FE738BD1486E4BBBD1486E439D48FE2351
:10E67000FBD148CB4E3E304C0EB87E5B81C806784D
:10E680003C06B9586E63AE6E7F3A3A3A3A3C7038FF
:10E690000E8E844E70F8E030546E9B305A6E736666
:10E6A0006E53666E33B5A20EA04E3E7EC37E7EA034
:10E6B0007ECE7E574E43EEA0663346F6A0BEE04EB9
:10E6C0005EE76EE0CE7E1B5EE0E0DCA0DC5EEE1F6F
:10E6D000237CF2F3AE5EEE1F237CF2F30E03E0A583
:10E6E000CCBC0E4670AE6881F04E70789A66AE680B
:10E6F000304070AEF03E55F04E7084B07E7E7E2F7E
:10E700007E89F68801C8E6B5A286B0668DC61C066D
:10E71000A54FC678A6063DC358B0FC06707C26E619
:10E72000F002223DD0AED8E63C7006023DD0B0E605
:10E730000CC38604304006A5D00C49D1C676431CD4
:10E740000A6AA5D049D066B0E6C67038A670A6F0B1
:10E75000986666776651ECA606704EF09866BF8D97
:10E76000C68451EC8C276688D326E67022FC06020C
:10E770003DD0A658B026E6FC063DD098BCA6588CE5
:10E78000A3BA44DDD47AFA9A983C0698767FA60616
:10E79000BF0DFC060C2013091A05D9FEA5D00C9755
:10E7A00098762BA5D00C5F98E63CA6B0FC707CF068
:10E7B0005DC40A3EE6B006A63CA60667BC704E7075
:10E7C000F8FE2F66A6067038EE472DD0983C66AF4F
:10E7D000BB0000000000000000000000000000007E
:10E7E0000000000000000000000000000000000029
:10E7F0000000000000000000000000000000000019
:10E800009CC2FFCC574626FBCC2F5DC4243C71CC68
:10E810006653309066FBC8CC6100839C4262E2A5DF
:10E82000684E9C90CC5F601B7A1F7ACB5DC4E01071
:10E8300071CC664FA5689C228859C87BA568D91CF5
:10E8400078583012662761C8CB30C266AF46F08C6C
:10E850005B59C8BDCC66E627652073BCF05DC42952
:10E860003C26662F8865C82B49F08804E9D48C2B98
:10E870005DC47E3E4E70088C2B4540061BF9C430AB
:10E8800018A6C6B07CEEBCA686A6061F04A666988F
:10E890003CC658B03C0671D84E70B87CD8040C13F6
:10E8A00008D8BCA898668DC77C0EEDA4E601D0AE52
:10E8B0003C58C69C584E7051B41C53BDD0C1D85E54
:10E8C0003E2DE0DDFCB1C0BDD04C1BE9D071F0B0F5
:10E8D000FC700602385AF051FCAAAE3C58C9C099E7
:10E8E000C0980A01D098AA0A5841C480E68741C45A
:10E8F0004C5780E6AB708D8C987C0EB004D88C138E
:10E9000008D826CABFAE3C580AB066577001D0413D
:10E91000C4808D8CAB0C2341C4804B081304980A2F
:10E9200030FF8D8CA156C1D8BDD04CD9C85E7E7E3B
:10E93000FE39E098EEB5F604DCD01EB07E7E2F08DE
:10E940007E29E331F40C533E85E0B05E3E7095F0D5
:10E9500059C0B0CE46CE6E6E68BDD071F04E7078A4
:10E9600058B0FC060201D0EDA48A0456705C0A0679
:10E9700076265766D88C1B086AD86A6A98AACAE7AE
:10E98000AA581C4699C4B0A1C46AB0664F7001D0A1
:10E99000EDA4A1C4B30C7B46A1C45B0830FF99C4AD
:10E9A000640530FFA1C469D095DC0C554AF9FA38EA
:10E9B000BCA6BC288804E9D48C434E30913CEEE9D7
:10E9C0005ACEBC06B07CC698BC1ABCEE4E70385C01
:10E9D000AA581C06BC065F3C0EEDA459A4E6AEBCCA
:10E9E0000EEDA4AE5884C61C6A17881C987C66E697
:10E9F0001F8CAF8CFBFC580A01D098AABCDBE156F7
:10EA00003BB03C263C463C7098E63C0AEDD02E8458
:10EA100049D463BC6658CEFC0A01D0B07C263C7059
:10EA2000983CAA7C5806D3B0FC707CF05DC45E3F75
:10EA30007E2F06ABF0837E7E89F788480DD4CE58B2
:10EA40004E70F80E8C2BEEC3F9FA3DD00698BC063A
:10EA50007F0DFC050E04200F0620120503F1FE6653
:10EA6000B03C065DD8554AA5CC06BCA63CF081F06A
:10EA7000D5CC663002C61306F5C459C42E12000068
:10EA80000000000000000000000000000000000086
:10EA90000000000000000000000000000000000076
:10EAA0000000000000000000000000000000000066
:10EAB0000000000000000000000000000000000056
:10EAC0000000000000000000000000000000000046
:10EAD0000000000000000000000000000000000036
:10EAE0000000000000000000000000000000000026
:10EAF0000000000000000000000000000000000016
:10EB00000000000000000000000000000000000005
:10EB100000000000000000000000000000000000F5
:10EB200000000000000000000000000000000000E5
:10EB300000000000000000000000000000000000D5
:10EB400000000000000000000000000000000000C5
:10EB500000000000000000000000000000000000B5
:10EB600000000000000000000000000000000000A5
:10EB70000000000000000000000000000000000095
:10EB80000000000000000000000000000000000085
:10EB90000000000000000000000000000000000075
:10EBA0000000000000000000000000000000000065
:10EBB0000000000000000000000000000000000055
:10EBC0000000000000000000000000000000000045
:10EBD0000000000000000000000000000000000035
:10EBE0000000000000000000000000000000000025
:10EBF0000000000000000000000000000000000015
:10EC000081C8E6B5A2064540B9CCA6BCA63CF048F2
:10EC100085F08C5BB0FC2670381CEE77709BD5CCF1
:10EC2000A04E70EE59C4EA003CEAF30E4E70AE6896
:10EC3000B01E4E3E1CBEBE33501050903B10BE2B3B
:10EC400010105003BE2B5050D0D3B046FC06F5C474
:10EC5000A3F85E5AE8A878E630C0062663A60670D8
:10EC6000383E334E7EF066A3A1803CD5883E7B7053
:10EC7000AE0E584DA459A4468D8C980EB0E66F7018
:10EC80005DC414218A4E6E56DC90688DB8BC08981D
:10EC90003C28441C6A8AEDA45606303A067B303084
:10ECA00006AF3020469C58DD201C6A4E30056A5B5A
:10ECB00059A46A4C8FEB48783A87783A8DC7B83CAC
:10ECC000D808D87CA88CB5515DC4333B3045663F2D
:10ECD000783A27301B83302B66832666378C7F304B
:10ECE0001A23266627301CD32666678C9F4C435315
:10ECF000F8EECE71C8700439D006B0BCA6700839E1
:10ED0000D0E6172606B0BCA670783C06B03C063CA0
:10ED100006B958BCB95826703C063CE64EA670A60B
:10ED2000F0B02606C78DC60E66176629C6BC069CBF
:10ED3000E2D330901C02AB30316A8B30460217664A
:10ED40009C024B501C62276A136AA6A606C6E6A25E
:10ED5000065E233008465DC46A27F9C40C2F70157F
:10ED6000C8E68DC606F8FEB0C6FB46DE1BA6C6A6E4
:10ED70007079C4AA58B0665F701C980AEDA49C58BC
:10ED8000461C8D8C51B47B4E1C10CC2F6EEB4E4B21
:10ED9000203C56069CE21B4E5330C4064FC64ED054
:10EDA000A646263CA3E6761C4E906AC6FB3031622E
:10EDB000276A13A662AA3C26EE61005DC42E1230BB
:10EDC000FF06F8BC66470EB8A6AEA88DC6B8BC66EE
:10EDD000B5A3840895D0302B06B006273C061B81CE
:10EDE0000A06B8BC13EEA6F30EB03CE630A8AEEEB1
:10EDF000176668A69C583508B0063C260677BC7096
:10EE0000783BF87EFE5F5C10EEAB1C7CEAF33C3393
:10EE100015C83C9C4A7079C40C2F8AB058EDA4AE3A
:10EE2000D87C1C846A1788D8AE987CEA1F8CBF4EA9
:10EE300030051C6A538C2F6A59A40359A4034E70E1
:10EE400030913CEE3B79C46DCCF5C459C4EA00BDA9
:10EE5000E0DC101E46FCBE77E6A670066638EE7053
:10EE600066EEF0BEAB5DC4EE00307A66FB61027800
:10EE7000E8380E38D81CAA28E09CA01C380EF8AA46
:10EE80007CE8AE7C280EE0D4948DC7A0EA73E267DC
:10EE90009846AE283B48084EDDE04E300BAAA0FA5B
:10EEA00060E6133AA6CB3C30030E51C45DC42E126B
:10EEB000B87CD83C30300693302E66370C60A6A65E
:10EEC000E0300D664F302D06E0303A066061DAB171
:10EED000D0AE0E3CEECEFCEA6DCC666686664E3059
:10EEE00007A63AC6F346703CEEBCC66804044CE183
:10EEF000C4E9D00881F08C4BB07EFEA1C3A1F4839D
:10EF00004E70780666263DC2EE4E9CCA1C3E70AE20
:10EF10003C06027098F00DD0A60670B0F07A4670EC
:10EF2000CEAA7C0EE5A4E6AEBC0E01D0C68D8CB098
:10EF3000A626A67A2770AE5B7001D0B08D8C0DD05E
:10EF4000A6704E6EF05DC4F000492438FC7006389F
:10EF5000FCA67C70E04670387CAA0A3C28E00404D9
:10EF600084E9D4983C1C0A0451FC4A2A2AE0306007
:10EF70000698467004261C7C4A300AFC58B8A6A89D
:10EF8000E0D91C78D8E0EDA40616D91C303A6643C7
:10EF9000302C6623302E6661DAE0B1D08E0441A4B5
:10EFA00044CE0637662FA20217484ECA686A054645
:10EFB0000000000000000000000000000000000051
:10EFC0000000000000000000000000000000000041
:10EFD0000000000000000000000000000000000031
:10EFE0000000000000000000000000000000000021
:10EFF0000000000000000000000000000000000011
:10F0000088DCD0FE95E84E705C380AB0AA2845D856
:10F010001388D91C78468C1326F0256C88080404C4
:10F02000E9D40C5B44DDD4CE7C06463BA6265DD8F5
:10F03000705B7C0A556CB03C46BC70C57E256C0488
:10F040004670387C1C0AEDA4563CAA7CEE3BCEFCF4
:10F050001C0A556CDABC06B07C063B86BC065DD843
:10F0600070DA7CE6917AAE4670CE68C1B0E0B07CD2
:10F0700006300B0697300D46DA7C06333017C63E55
:10F080009306301806BBB03C061EA114F87E7E9E87
:10F09000066646F098A6581CB07C26E6CE7C0A048C
:10F0A000EDD098E67CAAFC58CE7C0AEDD098AA5800
:10F0B000CE7C0AD9D0DC101E9E9E1C98AA5804084B
:10F0C00093EDA48A06D91C79B01CCCE746F06A01FE
:10F0D000D0987C6A6F98DE586A8744D91C987E2F36
:10F0E000581EA9763020E805768A48196C4479B014
:10F0F00098DE1EFCDC901E1F5E1BBE5E3C5883ED3E
:10F10000A48A06D91CCC33D9B008357679B01C6AEC
:10F1100046F001D0986A63DE3FFCFE9B0C8BFEDE5E
:10F1200004F3D91C0CE37E9EBEC7F8BEF3A3D91C22
:10F13000B8F8568A063040C64B46F06A196C1B79FF
:10F14000B0980C37FC1E9E3C1E3C9CE2042030F024
:10F15000E6E09CA0443020CC697766E3C666797708
:10F16000E699C8D91C9C6282B8A2F34C1B98F3069E
:10F17000E094339C98A60658A0D88444D84C77C60F
:10F18000A69C58301F6617260698069CE8D09C025D
:10F1900082B8A2F34C5177485576203CF64BA568CF
:10F1A000711C5DC4E01078581A7A7A4E203C5A1CC3
:10F1B0005D001AE000105B504B903BF3D023000041
:10F1C000103C56063044668F788C1B84138884D894
:10F1D000F0A5680C6973517626669FB07C06668C34
:10F1E00023300B4686BC0646F05DD8C97A26667782
:10F1F000B07C0646268C1B300CC653064349247847
:10F20000FC5CEAEE9C300842A17CF6DD7B30088C89
:10F210001F4200957C068C47C1681BC17A7C5898B8
:10F22000A6588CBB796C4A57C1B0BD1C0E0F20127A
:10F230000F0F0DDDAC78D884D8F049246D586100EB
:10F2400030FF66675ACCE3203C0630C366DD7A693E
:10F250007288489806C96C25E8E3CEBC06B07C6687
:10F260002326E6CEFC1C0A04EDD0988D8C0666861B
:10F27000B03C0671D8C97A3008957CE6EFDABC0656
:10F280001C3001667FE6CEFC0AEDD030608D8CB07C
:10F290003C9D7EB07C667766C6E6A658BC065DD807
:10F2A0007C26E633C626E6A658CEFC0A04EDD098A6
:10F2B0003CAA7C58066611F4D3F6278C557B1C06B5
:10F2C000300825400E7E9B9A0507088700D36B3BCC
:10F2D000E3FBEBD323DBB17E75F44670387C0AED9B
:10F2E000A4567626A3617E056C8C1B8413883D761C
:10F2F0006520056C8498F0A568F572796C0AA17B8D
:10F30000B96CB0684829E84670787083BB843BFBD1
:10F31000796C0A5788CEFC0AD9D0B03C26BC70ED77
:10F32000A456768CEBE6556CC6263FAA7C5CCAEEEA
:10F3300083B96CB0FC5CEAC41C59E8056C8498F095
:10F3400046F01B056C8C1B84138898F0C97AB03C7E
:10F35000E6C17A6606265DD8056C8498F0A56869D2
:10F3600072267F556CB03C06265DD80B4666E68853
:10F3700059C804C1B0BD1C07140F201E7E7EC63CB8
:10F3800030033E1B30017EFCE8BEB3DDAC0C3B46D7
:10F39000F0C6E10803A5684E5C10901ACC4F26EB2E
:10F3A00099C8BACB7976300B01ECC3847434857577
:10F3B00035867636370023363636363636363636A6
:10F3C0005B65209300000000E080E006C61C224739
:10F3D0001C8622279C860882CD7EC61C222B1C22DE
:10F3E000DD7B02A29F8C174230555EFC06BC30E0EC
:10F3F000000005CAF3EBE3DBD3CBC303180D14679E
:10F40000308AA630BD8B72201165E34F0B1D10238F
:10F4100050C604A89C60C74C81496A521BF515F37D
:10F4200014124485B60825C6205B15EBA2262A0ACD
:10F43000400C50AD3C362203820F003532388184B7
:10F44000D80400CCC040819010038074D184F5B002
:10F450004DC000A409302333CC5068BB881F88FB03
:10F460000D8C8C84D4CC0035C0A803033C3181863C
:10F4700021F25B38338A1CC3A1362321B22485E8EC
:10F480002ECD8843480C08000638622380C71082BE
:10F49000B02066CDC040FD657EFDF5E6D61831D1C1
:10F4A00018C0A82221727CBCEF43E2F030E363BBBA
:10F4B000EF0C2320EC20ECFF10A2A0802122282AB0
:10F4C0008221C0C3953C412282101102821108CCD6
:10F4D00004002088310089FD0CCF0B1042084991AF
:10F4E0009D3055C3080018E00D7800880350F08166
:10F4F00034242AF102000000000000000000000097
:10F50000C9E0331053FE72482113E20331158A35E6
:10F510001D23C6B0CB28320EF88A423203980C4025
:10F52000102131411204B81BCE392500C520F0044A
:10F5300052D9C408182044D915449146A603153D54
:10F540006D50210009076954011693A150421A4ACF
:10F550001B050452C7AC8EA0418010409A4F5D112C
:10F56000040481004227644114441785A2244348BF
:10F5700061542468441EC98009CD33A1DC50106A4F
:10F58000821041C1B30601194525880333D6404393
:10F59000482331E50800000610D014294304310047
:10F5A000000000000000000000000000000000005B
:10F5B000000000000000000000000000000000004B
:10F5C000000000000000000000000000000000003B
:10F5D000000000000000000000000000000000002B
:10F5E000000000000000000000000000000000001B
:10F5F000000000000000000000000000000000000B
:10F600002134432432A02C3222037A488414111767
:10F61000C54108160E3BD19008DA2308D40C50B827
:10F620000320AAC428201417170E003183AAAE7332
:10F630007F3703F17A18EB40E8C42EE340E044E062
:10F6400088114C2046211420D24F22D41E7F7C8C5E
:10F650003FCF143D4D34004238019D1008E1503237
:10F660000030344E4207C404A89C60C74C81C84097
:10F6700045D3F0D0801231CC44D401412433841BD3
:10F680008E32F62E61200609FD73B40CC10CF38C8A
:10F690002108C44098186081620F848B9EC008279F
:10F6A00008C70FEEC5174060865D2403B731315C93
:10F6B000C744C7CB50005044642384930C32E88C79
:10F6C000683D00088509240A6002040084C0000027
:10F6D000880E841800A3512E4891801E8508048945
:10F6E0004F2F313131B13C1432C3085200000000B9
:10F6F000000000000000000000000000000000000A
:10F700000B801A2838215A84720934015C0504954B
:10F710006824000054180D059034E248C5443411A3
:10F72000140F3113C411249811405844587841C41F
:10F73000084D700CC447E3244571A11991368087A8
:10F74000D0CC54010C8D2B033B0371330F45304655
:10F7500034D6061D20F4E668C8003744C8516C4B07
:10F760004C8C214BDD14E55131D0141E6300C000D8
:10F770004931CDEC56540E954414C339144A34879C
:10F78000064767C5C435C67D44753300E0B41B2306
:10F790002DBC141F595580D10A901110105C9C612A
:10F7A000C4004500148D4105090941465124C9444E
:10F7B0007155591055508296A0968978626E514DB8
:10F7C00085094A4DF5430186E051080816C68CB1FB
:10F7D0009C01B0079E01E6167941C088F20C200515
:10F7E00021A1F70C331654E3D21600000090AAAA08
:10F7F000884077282F3FC5A2474B85F630FF3F88CA
:10F8000000000000010000000200000003000100F1
:10F8100005000100050101000800020109000201C4
:10F82000090102010A0000020B0000030C000004A1
:10F830000D0000050E0000060F0000060A0000077C
:10F840000B0000080C000009584E55543020005899
:10F850004E5554312000584E5554322000435846DE
:10F86000554E300054494D45522000435846554EA0
:10F8700031004164764C31200041647655312000DE
:10F88000416476553220004D6174683144005374F0
:10F89000617431420046696E616E63005A656E7232
:10F8A0006F6D005050434C20520050504355205231
:10F8B00000436972637569005374616E6461004747
:10F8C000616D657331001A1B1B1B1B1B1B1B1B1B54
:10F8D0001B1B1B1B1B1B1B1B1B1B1B1B1B1B1B1B78
:10F8E0001B1B1B1B19007C204275696C74206279FC
:10F8F0003A204D652120202020202020202020207B
:10F90000202020207C007C20496620666F756E6474
:10F910003A20696E666F4070617865722E6E65740C
:10F92000202020207C00171B1B1B1B1B1B1B1B1BD1
:10F930001B1B1B1B1B1B1B1B1B1B1B1B1B1B1B1B17
:06F940001B1B1B1B18003D
:020000021000EC
:10000000444953500A454F460A57616974696E67FF
:1000100020666F7220646174612E2E2E0A4F4B0A87
:10002000505834310A52414D0A4552524F520A003B
:100030001640008F00A60299009E026600950247B6
:1000400003370309031E032602EC02F90451052FAE
:100050000557056A0577050C059104800485048A17
:10006000048F05B104630456045C046A047705A593
:10007000059A05D205A005C204E70504051204BED1
:1000800004C904A904DF04D004D7051604B0049EF3
:10009000049704B704EF05CA054605290522054F54
:1000A000056405710583058A05BA053606080663E9
:1000B00003B400008220160E0F03201604012DE069
:1000C0008E091805084830088B8E0914030F300F6D
:1000D000438E090E0902300244E6B83C5804CC1F96
:1000E0008C2BC4840C5F04C1B0301F682668C668BE
:1000F0001E2B6520610049244E00309D3CFA7EB8DD
:100100003C98FC6D1C3C587EFA7A6F605B0C2F08A3
:100110006B0B133C7A17FCCC8B0C67793C2E381296
:10012000C6C3837711C080703010847434857535F0
:100130008676363700E3E323DB53B300C366666697
:100140006666666666666666666666661B693CAC7B
:100150004CE733FB300A06B34CA7DB5E23793CDE69
:100160002146A3B87CD84C1B441348D83CA8A34CC8
:10017000EF8B4C1B446B485B5E2F6100410EE0D956
:100180001CB8E6F8302006A8B8B856A66617B8A678
:10019000E826E8C6E8BE5E2B6D8CDF005D1C3C588F
:1001A000200BE066D91CB8569C5806E223E2E20612
:1001B000A2263B66F8693C2403DC904C1B7E7E063D
:1001C0007E9BFEB806B8300A664623302F0626E826
:1001D0007E3E23C666E8E6E89C98E8EB5E6BD91C99
:1001E000B8E63020E86606B8B8B8566613F866A6D2
:1001F000E8E6E84924793CC8B01A5A300CBC1A70B9
:100200008DBCF10E8498A8793CDE5D1C1106E0D906
:100210001C0EB89CE2337E7E4C137E7E302FE81C91
:1002200022A6F8B0E21B62DFA0FCCAF61F226656C7
:100230005ABCBADEFA7EF35AF8B0E2736263601E0B
:100240003009065C422FFAA6E30E6EC1B04924B80D
:100250003CD808D87CA8208CB55188EEE8E04E2028
:100260003C063018BC1AB0303AE62366DF061AE0C6
:1002700097050916180508F8AE6D8CDF8C3008005C
:10028000E66D8CDF3A5C005AD070088DBCF10E9799
:1002900005091614030FF8AE6D8CDF8CAE0E9C00B2
:1002A000E21B8902DCE2E7E2D7E05CA01C4EA2027E
:1002B000E2EEEEEE3CBAF2BAA2DCD493300FE6697D
:1002C0003C51970509160E0902F8AE6D8CDF8C4E75
:1002D00000BA1A3CFA1B8902E6EFE6DFE05CA01CDC
:1002E000BAF2F2F2BA42421322A2DCD4A33002E6FE
:1002F000693C51B8AE6D8CDF8CAE00F06D8CDFE7E1
:10030000A600F0EE3004EE465BCE1C58DC9886C3A7
:10031000EE66F3BC463CE09918140F12793CC370AA
:10032000793C43B0CBBF140902793CC33CD88C273D
:10033000D8B95AD8655A840E01793C43B0BC463CC2
:10034000BA6D8CDF6C6E008C9102A902920F793C21
:1003500043705B920F18793C4358AEB0D8AEAEB044
:10036000AED870D3940F0EF888AE6D8CDF8CBA00C7
:10037000BA005BF88458B8AE6D8CDF8CAE00D8AE96
:100380006D8CDF8CD800E00B00A188C1B080B0304C
:10039000063000E6465D003CA6BC300656A87A56FC
:1003A000D3492408000170ED8A0B00C1020B00B98B
:1003B0004A0B0089520B00B5A20B0089020B0019F1
:1003C0005A0B00810A0B0009828814010D201604C3
:1003D000012DE08D1614201604012DE00B00A188DC
:1003E00080E00440CC00F3004D50A631F27F3A6922
:1003F000111B1342A631F27F3D85C2032F0270C646
:1004000000F600534952544EA605C8012F0470C689
:1004100000F400535A3FF653495A453E3DA631A8D1
:100420001997738B9BF37585C8032F00000000009C
:10043000050E04200F062001121201190E0F1420C0
:10044000011212011920060C0E010D0520051212D1
:100450000F120E0F20120F0F0D04090D200512129E
:100460000F120E0F20182D0D050D0F1219150E0469
:1004700005062001121201199812140D201604010C
:100480002DE0AB14010D4EABAD14010D308073AAFD
:1004900014010D30203BAF14010D30A0D8793CD9A8
:1004A000038D090414010DF86150753CD6CFAB09DA
:1004B0003016F3AD093056CBAB0A3036A3AD0A3057
:1004C000767B810A09130D30053B8A09130D301123
:1004D00058F86150EB8A09120D3013ABAB03130DC2
:1004E000301273AB12130D30323BAB03120D30924E
:1004F00058753CD606AD03120D30D2ABAB12120DBF
:1005000030B273AD12120D30F23B810A09120D3078
:1005100007FB85160F0D0DC4483B900117130DC442
:100520008808F86150B80E785150753CD697BF05D1
:100530000D010E0D793CDF22BF0D0904793CD62256
:10054000920DC433930DC4608848793CDFD0BF124C
:100550003E12C448C3923E3C12C493833E3C03C443
:10056000085B832B0319B86150C40888F861507583
:100570003CE5CE96091008048B820118010D120487
:1005800043820118010D030808844884F86150EB88
:100590008D120E1204338D120E0308846B8D151309
:1005A0001204338D1513030888448404753CDFF16D
:1005B0008D1513883B82010D151384843B8D120E1B
:1005C00006888844A3820118010D84845B8E090D7E
:1005D000882B98010D8488480804793CDF428D2AD5
:1005E0000D793CE56793100E1214793CDF49960EA5
:1005F000090D793CE5259319130D793CE5EA94053D
:10060000040D793CE58EB030CBB030F6F6366BB0E9
:1006100030F636F63BB030F636F636F61336F613CD
:10062000363A70DADADA3ABC80E000000000000006
:100630000000000000000D50CA00F6004D4544497E
:1006400054A81B10A5AFCF66A90AA819A5AEAB196F
:10065000B6B2018BA5A8AC0AB6AA87A5BFA5A59B73
:1006600073AC08B997F27F3FA9178EA5A57179A53C
:10067000AC9A73AC17A5AC0AA596B12A09A8157E49
:10068000BA0BCF6F06AC071DF34D5452A5A4C40C92
:100690002F1F10C401F700434D45444954A81B07C0
:1006A000A906A59283F74E4F542043505868124B29
:1006B000638E75691A10101245A806AC06B1874BF7
:1006C00067B1838EB72701A90A73CF661242111A48
:1006D00010101141A819A5AEAB19D07D8F02AC0A3C
:1006E000D0778FE06683F352452EA5BFA5A59B73F7
:1006F000AC08B994F27F3F8EA5ACAC06B98AA5963A
:10070000A594A5ACA597A59509A815AC087EE03BD6
:1007100083F3494D2EA5BFA594A5A59B73AC08BA3C
:1007200091F27F3F8EA5B0AC06BB8FA59554A5ADC9
:10073000BB880A7EA596AC06B25D0BAC0AD01A8FB8
:10074000AD06A596AD09A595B26D04A5A8111A1020
:10075000101140124385CF6FCF0FAC071DF34D54DE
:1007600052A5A4CA1D2F2150CA00F6004D41545273
:100770005801A902A81BF5524C2043588ECF68CFD0
:1007800069CF6AB114CF67A802CF66F74F524445CC
:10079000523D3F8E616883AC024030511140A6212A
:1007A000AB198E2083F152111B1C134240A59DC230
:1007B0000AF4004D5452CF6F02A908A907A815A842
:1007C0001BFC2041204920445420422053458EB236
:1007D0001904F152A5A0F44445543D9B737EB22800
:1007E000CF7BA808CF66F152BFB9CF67F152A5A25F
:1007F000B23ACF68AD02B4279F00B244CF6AE02D71
:10080000829A73F2522C9B73A5B2B254CF7CF152F0
:10081000AC029F00AD02A5BBB262CF7EA808CF6933
:10082000E00B820FA807AC02A5BEA5BD03F152A53F
:10083000926883511140A63175A819A59DAA198502
:1008400074401140A6218ED0926FC2162F3D30C049
:1008500001F4005A5E4E8030754F20537120427172
:10086000054E01AC0485A815F2553D9B737EF256EA
:100870003D9B727E85C605F5004D41475A4FA81530
:10088000F2523D9B73AD047E85CC02F400655E5A46
:1008900081554E80B134CC01F4004C4E5A814F50FA
:1008A00080B141CC01F6005A5E312F4E80301316D4
:1008B00010714331754F2068605371206843710493
:1008C000E061049700B28185024F71214071B4113B
:1008D000C606F50053494E5A81325A7133E04C8AAC
:1008E00042225923E0518B4280B100CC03F50043F2
:1008F0004F535A8132597133E0318A4254225A237C
:10090000E0358B4280B100C004F50054414E5A815D
:100910001242325A71124233E01D8B4023E00C8A9E
:100920007143762259714380B1000B83835871550E
:1009300043715840BD850C558360400D124385C0FE
:1009400008F400615E5A7532717450427622421D7D
:10095000F3655E5AC003F5004C4F475A5034758119
:100960004F5024957195727580B100C403F6005AFA
:100970005E312F57327533753151713051402071CE
:100980004354762171432322C204F4005A5E5781F6
:100990004F504F75754F7175427540744E554E806E
:1009A000B100CA03F300432B71067540754074B162
:1009B00000C202F300432D547154B613C801F50070
:1009C00043494E56E00482B100034F607154714EAA
:1009D00085C003F300432A4F75754F7575717542D5
:1009E0007540744EB100C003F300432FE024021D94
:1009F000F2432ACC012F5B70C600F400504C591210
:100A000013A621AB198ECF6AF84445475245453DA0
:100A10003F8E1245D00F6A71121146D0166A71A826
:100A200000A903A905A9069116911506E04B8C971C
:100A300015B608E0448CCF6FA815A81BFC465820BB
:100A40005254202020204E45578ED0156FCF66A9D6
:100A500006901691157183838397159096AC059532
:100A60007342E1E18E9073909642AD0571F4463C7D
:100A7000583EE18B8FD0406F0DF1619015A631F398
:100A80007F3D3F778E919585CF67A619D0576FC868
:100A900015F40052545312141A11AC069117AC05F8
:100AA000BB9390161141911590960C95959715BC96
:100AB000079500A8050B2036213722382339243A20
:100AC0009016121040A819AE73F34E3E358E85CFA6
:100AD0001911101A10101691149115E12E902DE095
:100AE000DC842A11E17191E16E91E16B91E16891F1
:100AF000CF18289112543827911129911342269129
:100B000010144241379012144290135141901042F8
:100B10009011514136A900E06397AA038503AA0208
:100B2000B1882D29453D2D2A453D0190133C129554
:100B30000C950D2D51901041661000111B1C18458D
:100B4000E0358675523F2C2D4290111243416711BA
:100B50008361433E2C519012412D12424052940E1B
:100B6000A800E00287082C2E543E40372D2F543F1A
:100B70004036E02796850771777185CF17181A10D0
:100B8000101691149115E08390AC03852DAC00E014
:100B90002C842811E0C191E0BE91CF162754124356
:100BA000838351264166B1A2524039AC00E00E84E5
:100BB0007476413AAC00E00584A9028505F4524FF1
:100BC0004F54E03B8F77E02C8D850154523B742BC2
:100BD00054AC00E00586A802850774F155E0208F2B
:100BE00074F156E01A8F74F155E0148F74F156E0E9
:100BF0000E8F850EAD068591979617917385CF0F51
:100C0000E00E0DF27F3D9B737E85CF10103D268355
:100C10006167B4D0433E7690956140566811405765
:100C20001146713C0A1110950C2E543E092D2D2CA5
:100C30002E42403D78858383E00B8E67852E426689
:100C4000B916BA200F909540429715BF099095406C
:100C5000901491157585CF119715012D42409095EF
:100C60007191958504A803103D27362837E0D416E6
:100C7000B300C0452F2320C201F600444946455128
:100C800019A621AB198EA815F54E414D453F8C8E06
:100C90009A07F74F524445523D3F8B8EA9019773F7
:100CA000A801FB535445502053495A453D3F8E12ED
:100CB0004331F458303D3F8E32F459303D3F8E334E
:100CC000AC01E02D800A2322E0958135E06B84366B
:100CD000E06784920683402340222183403440E031
:100CE0007E81254026834040134324E05482BA2B62
:100CF00001F559302E3D3F8E340B242322E06081D4
:100D0000353021E0498636302120244025E04485D5
:100D10009206834030218340E0348626834040257C
:100D2000401343244034762625401343402183401A
:100D3000354276E00C82BB3F052340222140B29E23
:100D40000392027192038F980298037F85072024F3
:100D5000402006124324407442234022744002AED5
:100D600087082142CC212F3A50CA00F3005643A9EC
:100D700004CF6FA815A81BFC4450204350200D2021
:100D80004D2055568EA627D0176FCF7EA62DF16425
:100D9000CF14F27F3D9B737ED0286FCF7DA62FCFDF
:100DA00068A62CF10DD01614CF6BA62AD03C6FCFBD
:100DB0007BA629D0068FCF7CA628CF0FAC04D04EBF
:100DC0006FCF7FF2583D9B737EF2593D9B727EF24E
:100DD0005A3D9B717ED0656FCC0FF60043524F5346
:100DE0005383CE023042CE022342CE0194717194DD
:100DF0000342742042234121744190712241CE71FB
:100E0000A62785CF67A623D04E0FCF6DA624D09EF0
:100E10006FC208F300565361686877139474967430
:100E20000F7591F496740F7591F496740F7591F493
:100E3000757585CF6EA625D07E0FCC05F300565272
:100E4000686175A627741342134090F3977290F26D
:100E5000977190F185CF66A626F3444F54D0CE14F7
:100E6000C605F400444F542142712242407123428E
:100E70004085CF6AA62BD0BD0FCF69A62B74F14D4C
:100E8000D0F114C005F300564531753275337575D0
:100E900085C002F300562D1C11A62EC601F3005684
:100EA0002B920175920275920323222185C802F4C8
:100EB00000565859CE0175CE0275CE03757585C89A
:100EC00002F30055564F90714F917077114ECE70CE
:100ED000754E85CC02F300560DA62BA62AA62BA68E
:100EE000265D85C402F3005644A628A62B7485CA45
:100EF00001F300562A9470947142C8012F2030C02B
:100F000001F30054521117A621AB198ECF6AA91B09
:100F1000FA5A302C59302C5830203F8E13A62477A3
:100F2000F5524F540D3F8EA90567B198A805911051
:100F30007311CE71F7632C622C61203F8EA62B12A9
:100F4000A624CF6F01A81BA815A901FC5E4E205E48
:100F50004F202020204E45578EB117CF7DA622CF9F
:100F600066A801A630D008FFCF67A901A630CF7FC1
:100F7000F2583D9B737EF2593D9B727EF25A3D9B27
:100F8000717EB140C013F3004354AD01B38813A682
:100F900025A628AD058503AD05B2B611A62412A677
:100FA00025A6239010AD015459A62E1130A62590E8
:100FB000105A9300A62EA62914A62412A62511A61F
:100FC00025A6269400A62A20A62E14E00783AC01AD
:100FD00085021304A625A629C00C2F0000000000DE
:100FE0000000000000000000000000000000000001
:100FF00000000000000000000000000000000000F1
:1010000000000000000000000000000000000000E0
:1010100000000000000000000000000000000000D0
:101020000B00D19E000000CBC30000311604011854
:1010300000000000000000000000000000000000B0
:10104000000000000000000000000000000000227E
:10105000020000C0001800100010F223E3F3C4CE19
:10106000201214C16F3C5888FFE6EF080000000012
:10107000006804545555554D1CF1EC4CE30DC03D32
:1010800006CC23E2CCD14F333B3713F22B335354EE
:101090000D4FAB28CF1D48E80DCEB33713DBCF1C67
:1010A000734C456417FC24E2F05112F1F2F2BA28B5
:1010B0000479EF2FD173C3C4FD7D138C14D5CA639B
:1010C00000004C444C10D7050000135422743340E8
:1010D0005513ECC10800C0041122DD0C5430B207D6
:1010E000234C101304C12CD07530002333008C3CEA
:1010F000C300CC074CD033303F30E7E1B40033417C
:10110000220713141335CDD4650D74EC47C9D010E4
:10111000D0109010D01000003000C0348D0110416C
:10112000411114620000116200100044445121007A
:101130000100000100000100100004001000000484
:10114000000000000C0000014000104F02003301BD
:10115000114410410440001033000400014000100D
:101160004F00C40031400C4008C001C0CB1033090F
:10117000009300D330B0330D70000CC002C02CCCF3
:10118000246000800080910C00022000088064131D
:101190000000800060008000024839054C033009DF
:1011A0003005300530D9744967746618DA6F050068
:1011B0000080010044111111511151444404515453
:1011C00044441145114500116200004411050054CA
:1011D0005501454445511415401111144110101189
:1011E000114111111111451404444444044544149F
:1011F000511151041111510450151101448801007D
:10120000141100454444440040555415514540458F
:101210000010454404000050141140141111111124
:101220001111111144101111111111114111114518
:1012300054154544555110620050555555144114EC
:1012400044050014414405005511005445000015A3
:101250005455555541445515010055055541450016
:10126000405541554145004055554105555551554D
:1012700055515555005055550001005555444500F0
:101280000055555555550140555555551100555565
:101290000440150100415455054055555511004174
:1012A0004088014044140100544151504444444199
:1012B00044101101000014444454454414441405DE
:1012C00010044544404511410010101111155144BE
:1012D00044545555114504540440445050411004A1
:1012E0005154515454454545514510155155555487
:1012F00044454540415545555515551511545555CD
:1013000015545504101144455041105555155504B8
:1013100055114405101454554510550445500445C5
:1013200050514414411015551555545555455455B3
:10133000555541551145454411155115454555051E
:1013400011620000451401501100501111000050AD
:1013500015400550115441414154555550555510B3
:10136000054055055550550551554155555555554F
:101370005510551545514455555555555421064060
:1013800044440000004510111144414444041141FB
:101390004410111144100551100501001415155188
:1013A000545515155144101104405511155111157E
:1013B000554410005554151111450404014055556C
:1013C000151144144100545505404400445154053E
:1013D000005114550014451555004444540044541C
:1013E00000441462004444110100404501501411AE
:1013F0001501004511454400000045444404111105
:10140000411444411401105144544451444445454D
:1014100014114551444451105511210000000000A1
:1014200000000000000000000000000034C003E0E5
:101430001839F738F77FF3A2007B00BC00CAF3CF5E
:10144000F81FF845F859F866F873F8A0F8BBF8D714
:10145000F90FF924F93BF958F972F981F98CF9A1DE
:10146000F9B6F9C8FA5FFC470DDE0E280E3F0EB440
:101470000ECF0F5CF3DFFD39FDA8FDE1FE0AFE3063
:10148000FE53FE61FE6BFE7DFE8FFEA3FEB3FEBF2C
:10149000FECFFF540FB7F3AB0B900C350CA40CC16F
:1014A0000CE40D21000085160C0F1308793C2C6804
:1014B0004670F87030C070381CD0F0A04E68A8B0EC
:1014C000E80E4924B8AE4EEED74E9F30C7704E5C42
:1014D000229CD08628E806706048658C015C621BFF
:1014E000A2A230C770AE738705140E0904793C2C94
:1014F000A8898C00900F0F0C0913CC37793C92C44B
:10150000E0793C3BEEA038588C4F0C27693C924C5C
:10151000E733784C270CB3B846FC064924F81E7E06
:101520007E37793C92895270A6A687A647A6B7A6B1
:10153000BF898C5DEE3B0E658C32EE2F58658C2199
:1015400070658C3A898CC5898C50793C92793C1AAB
:10155000120503151213090F0E898C881E7EF87E62
:1015600023B87E37793C92895244793C3BEEA338CC
:10157000580C270C63AB8C9F884844CC1348884395
:10158000084404CC13080898F04670B87C588C873F
:1015900088983CA86D8C9F580C1F04138498F04CBD
:1015A000471348300B0C1F301E06793C65E6534C40
:1015B000C36D8C9F580C174B793C92793C1A0E0FD7
:1015C00020120F0F0D898C884E58793CD36AF3DCBA
:1015D000901E1C793CE5E698E6D63C58BEB31C98B4
:1015E000EA1F3CEB58681598EE1B4C33793C92810E
:1015F0000A5C420A0C23AA62231C29A430C3704E41
:101600005CAAF04D9CCC67B8584C474EE8380E0A9F
:10161000AE28B80A30C370387CAABCF04E705C109B
:101620009050105090105050D058681598EE1B4CA8
:1016300023693CBCC80C17C40E1C1DA4BD8C4D9C5A
:101640000E30C37038BCAA7CF0E0A18888C1B0BD60
:101650001EBA60A67066A638E67066E6F0A3BA60A9
:10166000A67026A638E67026E6F0A3E0DCA0467059
:1016700078E630C0067026CB38EEB33E8F7E5C1223
:10168000DC90905C726B5E725BFC560643A6262B68
:101690004EE0E026E046704EA668793C3BEE43A65D
:1016A0000670264338EE2BFC5606B36686467078E5
:1016B0003CC6BC68860630C070383C1CCA60164602
:1016C000A0A6262746E02B66E6C60A3C0A7CF03632
:1016D0006630C1464670783CA6C6A65ABC1A783C0D
:1016E000066626A666A6793C21A6E066866D8C9FD6
:1016F0003E13664670783CC6BC682626C61B46E08C
:1017000030C00670383E23A626CB30C01E7EC646AB
:101710001F661E46707826467CA63C66683C06A678
:101720008630BF46BC265E1726463C5ABC1A6679F0
:101730003C21467078E67C0630C0704EDC9090FC10
:10174000A6B606167CE6F67CF04E68A830C00666A3
:1017500070383E274E7EF04626E0044460793C3BDC
:10176000EEA038588C13488CE30C8B084C3F04488F
:1017700098F0B833844498F07858FB7858C44C13E8
:10178000C88CBF6B0C1F4EE0B858C40C13C80C5764
:101790004670B87C5884983CA84670987C1CEAA097
:1017A0000E6D8CBAB858259E4924B0E888793C2A39
:1017B0000C27793C954C534924B87C588C1F450222
:1017C000C502793C2A793C3BEEA0A6067026433838
:1017D000EE2BFC5606B38630C00670383C56062603
:1017E0000670385CEA273E1366A6066686A65ABCD3
:1017F0001A6630C0E6793C2E662643A67026064E51
:10180000F0C3E04E1C909C101C0AE5A456E6603024
:1018100005426ABFE01CEDA43C3005426A1F1E1B56
:1018200059A47CE00000000000000000000000005F
:101830004408918C6B30C170385CEA1CBC0A46705D
:10184000793CBA5C6AC44213C81CBD8C4C091FC1E8
:1018500002793C95F858793CAB6BB058793C955877
:10186000793CAB793CA2F0418C78793CA8EE2769B1
:101870003CA10EB05EFE23693CAF1EA0BE1D6160A0
:10188000FE1FEE27693CF3793CA5EE63793C9F1C73
:1018900002D0761613B6F0793CA86838E8F828B07C
:1018A000A8B80E793CB53A356060793C1D793CF2B8
:1018B000EE9B793C6A0E793C1A793CB52626BE250A
:1018C0006160FE574E5C2226260E793C1A793C99BF
:1018D0000E38AEA0BE1D6160793C1D793C79793C23
:1018E000A2A0256060793C1D793C56D85EFE6B79DC
:1018F0003C52A04E3E6EA03D60A5500E60793CFD6E
:10190000EE9F793C56793CA2A02560A550600E79E7
:101910003CFDEEFBF8700648693C00793C524E5C99
:10192000223AA3793CA5EE37B068693C71793C9FB7
:10193000F627693C6A76F0793CE7793C1DB00E7970
:101940003CA8A0BE1D6160793C52A04D6060793C0E
:101950001D793CF2793C1D793CEC793C06A0BE1E19
:1019600060793CE3793C81793C990EF8AEA0BE1DCC
:101970006160793C063ECE63793C0EA0BE1E607964
:101980003CDF23793C5A793C87EE67793C5A793CB5
:1019900087EE27F8E82BF84EEED7793CA858793C2B
:1019A0009558793CAB793CA2F04670B0E8498C2A56
:1019B0000C27498C95B95AA04E5C66503D6030C8E2
:1019C00070382560A5500E30C770AEE80E384E60F6
:1019D000E0B0A84E68793C99E8064870693C00B8C8
:1019E00068380E793C99AEE884B0A8F8280E793CA6
:1019F00099A0BE1D6160793C1D793CA50EB8A0611F
:101A0000604E5C223ABE256160793C060E793CA2AC
:101A1000A01D60A5500E60793CFDEE87793CEC7905
:101A20003CA2A05CFA37BEB626228B5E37FE373A60
:101A30005BBBFEE762FA1B2213667A00A5500E60BC
:101A4000793C99AEE84EEE27693C2A7870F80E7919
:101A50003C994EEE27B08C53AE0E06664870693C3A
:101A6000000E793CA85EFE23693CAFA0B8AE616071
:101A7000096060793C1D793C990EF8A0BE1D61603B
:101A8000793C52A0496060793C1D793CE7793C6A19
:101A90000E793CB5BE1D610E60793C99AE680E7939
:101AA0003CD3BE1D6160FE9B793CA55E680E793C0F
:101AB000D31D6060793C1D793CA50E793CB51D6055
:101AC00060793C06793C1D793CD386BE2561FE7366
:101AD00060793C52B0A0BE3D61BB793CA50E793C1B
:101AE000D386BE1D61FEBB30C970380EB0BE3561F5
:101AF000A5500E60793C99AE6888693CB9B026263D
:101B000026BE77793CB5666666E0A0316060E07914
:101B10003C5AC3793C56A3793C99F823793C990EF9
:101B20003833793CA50EB8A0BE1D6160E0793C99C0
:101B3000AE0EE8384EE0793C52A0756060E0793C2A
:101B400056C3793C352B793C52E32E7A0B30C0706A
:101B50003868F828CEBE1EE8B8BA9CEAEAEABAA805
:101B6000AA8A8A8AE330C070EED8B81A9ABABABA8A
:101B70001CEAE6A8F8EE38E87828BA463CFED8EE2B
:101B80005CE030C39C4330C41C2330C59C7038EEED
:101B9000D8B8D4CE14EBFEAED83B793C52A07560D9
:101BA000A55060E0AE0E58CE23793C56A049606047
:101BB000E030C070B83CA6BCA830C37038BE5CEA48
:101BC000F0E07038E0793CAB0E30C7BB30D0A330CA
:101BD000C08B30C87330C95B30CA434E707828B8A8
:101BE0006898A85CE04E5C22A0E01C38AAFC0EF8C5
:101BF000FCAAE8AE28E0B0A0FA274626765C5A5E3A
:101C000050EE4670B87C0E9CA2467C60E6E6A0AE24
:101C10001C2666E21B4213A6B67FB66F58860646A0
:101C2000B6504626561B26986E466030D070E000AF
:101C30004924F870B80E30D0704EF0F0586D8CAB6F
:101C4000AE5830C07098E8A0BE1D616030D0704EB4
:101C500028E8DA2F58693C3E793C5B30C070F825A3
:101C600060706006481344666630D07038F0EE58F5
:101C70004670B028EE7004793C6B30C270658C08F9
:101C80006D8CC6AE68F8F0E80666693C506D8CC68F
:101C900078A01D6068B80EB86160AE0E58CE49607D
:101CA00009604EBE50503D60606D8C1D30D0707824
:101CB000A03D6030C070B82560A830D070F80E30FC
:101CC000C07038F01D6060793C55B0FED830DE70D1
:101CD00038FED83160606D8C1D30DE7038A6F07E25
:101CE00030C070CE284E900E30D070B8A01D60A8C5
:101CF0000E60693C0A30D0704EE86D8CC6B068301A
:101D0000C070AE6830D0705C4E90A830DE70385E27
:101D100046F030C0704E28A830D070F80E78A01D64
:101D2000602830C070F80E30D07038AEBE1D6138FB
:101D30003D60A550F05C4E22A80EA0B8AEBE1D615D
:101D4000FE2B60693C55B86960AE0E58CE4960E81C
:101D5000B80E1D60B82560F83D60B869604E6690A9
:101D6000503D607030C070F80E60793C62B03D60EC
:101D7000700E30C070F81D60F00E60793C62E806AD
:101D80006660693C36B80EA0BE35612830C070B8B8
:101D90000E30D070B86160F030C070780E30D07006
:101DA00038616030C07078BE2561B0256060793CD4
:101DB0005B78256068606D8C5230D070F870B8A088
:101DC000696078BE2561B02560606D8C1D30D07073
:101DD000780EF0A01D60386960606D8C35A03160B0
:101DE00060793C5BF02560606D8C1D30C070787050
:101DF00030D070B8A0FA23DA50260EA835600960FA
:101E000058606D8C95B0AEA06160B0256068EE46FC
:101E100070B80E78A846703868EE2E7A606D8C0621
:101E20006D8C52A03160709E30C070CE2830DE7054
:101E300038A606F0B0BE256158380E30C070AEA886
:101E400030D07098E8780EB0AEBE1D6128B06888BA
:101E5000084E6830C070B84AFC0E4E1C50A8901C4A
:101E6000029C48021BAE44F08C1F04138430D070D7
:101E7000780E4E5C10A035604ED0256068F80E30AC
:101E800007E66030C070B8AE26AE7038A0BE1D61E7
:101E9000382560A830C070780EE0DCA01CF2525EDD
:101EA0001B669230D070B85EBE1D61FE7384083030
:101EB00007E66030C070B80EB09C02EB26AE70AE84
:101EC00038A0BEAE60267038A01D60783D60B8694D
:101ED000604E90BE2561FE1B88083007E66030D05A
:101EE00070F80E30C070B8A626A670AEF0B80E78A6
:101EF000A06160F82560E83007E6C66030C070B8C1
:101F00000E0C33B0AE9C22A80227693C38B80E4CA8
:101F10005730D070F826AE70AEF030DE7038A03E8C
:101F2000137E46F060693CE2F858606D8C9530D0C5
:101F30007038586D8CABAEA0BE1D6130D07078701B
:101F4000F858606D8C81980EB0A01D6060793C558A
:101F500070606D8C521E30C07078A03D60B0FA4346
:101F60005A5E5066D414EB2560A550F05C58606D45
:101F70008CABB0A0A550F060D44B30C07038D8887E
:101F8000D8F0418C786D8C52A049624EA05C6650AE
:101F90003D6230D07038AEA0BE1D636630C10C17F4
:101FA000267038FC9CA2023CF0A0B0A550584670A8
:101FB00098F068A8E87060E0DDAC0170ED8A5470BC
:101FC000C600F40054564D1110A621AB198EA9007D
:101FD000CF7F773132333435D00BEF0FA815F27F36
:101FE0003D9B737ECF6FA81BA916FF204E2C204966
:101FF0002C2050562C504D542C46F27F568ED01B20
:102000006FCF7B111242CF66F14E31AB16A634BFB3
:1020100036CF7C111243CF67F14932AB16A638BFD9
:1020200046CF68F2505633AB16A635BF52CF69F390
:10203000504D5434AB16A636BF5FCF6AF2465635C4
:10204000AB16A637BF6BCF7EA815F3454E44AB0049
:10205000A800AC00F5424547494EF67F204D4F445D
:10206000457ED07F6FC817F2004E2267B49B111BCC
:10207000124336E02F8864BBA32864B29705F62488
:102080004552524F528ED0A36F042325402467B58A
:102090001443B18402E0068A015431850B6526653C
:1020A00043318509E0118938E00D8939850CAC0090
:1020B00011AD001042850A2383CE053340265436E5
:1020C00061E0150B114024422623424067B552437C
:1020D00026425485CC0FF30050562267B189E05454
:1020E0008727254226B2830125210224424054330A
:1020F00085C204F400504D542267B18BE036872727
:102100002542234026B28501232540210267B500E0
:1021100043543485C005F30046562267B18BE01462
:1021200087244223402743B28601242142234002D0
:102130005435850822111B124365214254553776C8
:10214000585422111B12434376E09D0B1140423636
:1021500085CA08F3002A49212442234025406732DA
:102160006785A9052324E0BA0B403676244154251F
:1021700040374264B500211178B1842463B29001E4
:1021800026274267B50027264354216053B3BB027C
:10219000216011403226244266E065850D225021DF
:1021A000425822114167B18343B2820121023811A2
:1021B0004124422221532642403921284122114103
:1021C00067B18D4322422442B28E0311714D328594
:1021D0000121112141421243022921424029714328
:1021E0002754294371532242767132714D61111B7C
:1021F0001C1646BD59AC05E00785A90522B3350676
:10220000A80522603227CE0637C41A2F4270C600B6
:10221000F50043464954A815A81B1118A621AB196F
:102220008ED016E8CF6F2BFC207E2B2020434C7ED7
:10223000204649548ED0126FCF689900709906706D
:10224000990C70D0206FCF66A61CCF67CF69D02BBA
:102250006FCF7BA61DD0326FC80AF300417E719903
:1022600006917447E021804774920574920485C4F6
:1022700003F300447E719906917448E00A80487423
:10228000930574930485017576507176715071765B
:1022900094705071947150990C85CF6A2B114150F4
:1022A0000C2BA901A902A903A904A807FC4C2045ED
:1022B00058204C4F47205020428ED0976FCF6AA6AF
:1022C0001ED0E7E2CF6611A61FD0DFE2CF6712A6CD
:1022D0001FD0D7E2CF6813A61FD0CFE2CF6914A6D4
:1022E0001FD0C7E2CA10F500424649547733A9808F
:1022F000A907E01A81E02882E03683E0448420CCFC
